:020000040800F2
:1000000070DD002061020008A1360008E32D000821
:100010009D3600086F040008A53B000800000000A2
:10002000000000000000000000000000A101000826
:100030007304000800000000FD010008E937000813
:100040007B0200087B0200087B0200087B0200089C
:100050007B0200087B0200087B0200087B0200088C
:10006000E90A00087B0200087B0200087B02000806
:100070007B0200087B0200087B0200087B0200086C
:100080007B0200087B0200087B0200087B0200085C
:100090007B0200087B0200087B0200087B0200084C
:1000A0007B0200087B0200087B0200087B0200083C
:1000B0007B0200087B020008E13800087B02000890
:1000C0007B0200087B0200087B0200087B0200081C
:1000D0007B0200087B0200087B0200087B0200080C
:1000E0007B0200087B0200087B0200087B020008FC
:1000F0007B0200087B0200087B0200087B020008EC
:100100007B0200087B0200087B0200087B020008DB
:100110007B0200087B0200087B0200087B020008CB
:100120007B0200087B0200087B0200087B020008BB
:100130007B020008810500087B0200087B020008A2
:100140007B0200087B0200087B0200087B0200089B
:100150007B0200087B0200087B0200087B0200088B
:100160007B0200087B0200087B0200087B0200087B
:100170007B0200087B0200087B02000800000000F0
:100180007B0200087B020008DFF810D000F032F993
:1001900000480047F9740008AFF3008070DD0020CC
:1001A0002C4B19680868B0E8F04F80F30988BFF35A
:1001B0006F8F4FF0000080F311887047000000003F
:1001C00008480068006880F308884FF0000080F35A
:1001D000148862B661B6BFF34F8FBFF36F8F00DF35
:1001E00000BF00BF08ED00E0DFF80C00016841F43B
:1001F00070010160704700BF88ED00E0EFF30980F7
:10020000BFF36F8F134B1A681EF0100F08BF20ED5D
:10021000108A20E9F04F106009B44FF0500080F3CD
:100220001188BFF34F8FBFF36F8F11F08DFA4FF02E
:10023000000080F3118809BC19680868B0E8F04F25
:100240001EF0100F08BFB0EC108A80F30988BFF3CE
:100250006F8F704760000020EFF30580704700004B
:100260000648804706480047FEE7FEE7FEE7FEE750
:10027000FEE7FEE7FEE7FEE7FEE7FEE7CD38000813
:10028000890100082DE9F05F0546002092469B4653
:1002900088460646814640241BE02846414647469C
:1002A000224600F097F853465A46C01A914110D39F
:1002B00011461846224600F07EF82D1A67EB010819
:1002C0004F4622460120002100F075F817EB000987
:1002D0004E41201EA4F10104DFDC484631462A4687
:1002E0004346BDE8F09F00000649074A08685043AE
:1002F00043F2390210440860400870470149086021
:1003000070470000980100206D4EC64110B5431A99
:10031000934209D28318881803E010F8011D03F8EE
:10032000011D521EF9D210BD40EA01039B0703D004
:1003300009E008C9121F08C0042AFAD203E011F824
:10034000013B00F8013B521EF9D210BDD2B201E0D0
:1003500000F8012B491EFBD270470022F6E710B5CA
:1003600013460A4604461946FFF7F0FF204610BD23
:1003700030B504460020034600E05B1C934203D2E4
:10038000E05CCD5C401BF8D030BD30B50B4601467B
:1003900000202022012409E021FA02F59D4205D324
:1003A00003FA02F5491B04FA02F52844151EA2F1CE
:1003B0000102F1DC30BD202A04DB203A00FA02F110
:1003C000002070479140C2F1200320FA03F3194343
:1003D00090407047202A04DB203A21FA02F00021E5
:1003E000704721FA02F3D040C2F120029140084345
:1003F00019467047064C074D06E0E06840F00103DF
:1004000094E8070098471034AC42F6D3FFF7C0FEDB
:10041000D02C0108F02C010870B58C1810F8015B85
:1004200015F0070301D110F8013B2A1106D110F88D
:10043000012B03E010F8016B01F8016B5B1EF9D191
:100440002B0705D40023521E0DD401F8013BFAE717
:1004500010F8013BCB1A921C03E013F8015B01F882
:10046000015B521EF9D5A142D8D3002070BD00BF58
:10047000FEE7704710B50146002226E002EB820439
:100480000B6903EBC4000023036043608360C36017
:10049000036243624FF0004303604FF48C434360B8
:1004A000436823F00043436001F1480343F822000E
:1004B000032A07D202EB82040B6903EBC40328333F
:1004C000C36001E00B69C360521C042AD6D3002428
:1004D000CC650C668C66CC668C650B6803F5805326
:1004E0000C69DC6010BD10B50146002222E002EB71
:1004F0008204CB6803EBC400002303604360836085
:10050000C36001F1180343F82200036843F4801329
:100510000360032A07D202EB8204CB6803EBC40317
:100520002833C36001E0CB68C360036843F4400331
:100530000360521C042ADAD300248C620B6803F592
:100540008053CC681C6110BD38B504460020009073
:10055000206800F58050806940F48011206800F523
:1005600080508161206800F58050806900900120F2
:1005700000F042FB0099206800F58050816138BD91
:1005800010B5024800F0D4FB10BD00004850002018
:1005900030B503461479557944EA0520084C0C44DB
:1005A0002064D4782406957844EA0544557844EAD2
:1005B0000524157844EA0500014C0C44606430BD04
:1005C0000080024010B5A4B0044601208DF83C0024
:1005D0008DF83D0000200D908DF84B0001208DF826
:1005E0004A0000208DF8480001208DF830000020DE
:1005F0008DF84C008DF83B0014908DF854001D9040
:100600008DF878001F908DF882008DF880004FF4EF
:1006100080401090C010119000208DF881000BA92F
:10062000204600F095F901208DF80C008DF80D00A2
:100630008DF81D008DF80E00002005908DF81C002F
:100640008DF81E00089001208DF824008DF804001C
:1006500000040290800106904012049001208DF861
:10066000250000200A9000906946204600F010F90D
:1006700024B010BD0020704710B501F06BF910BD1B
:1006800010B5024800F056FE002010BD4850002072
:1006900070B504460D46164633462A4621460448A0
:1006A00000F07AFD10B14FF0FF3070BD0020FCE784
:1006B0004850002070B504460D46164633462A467B
:1006C0002146044800F093FF10B14FF0FF3070BD99
:1006D0000020FCE7485000202DE9F04F80460C46F2
:1006E000164608F118031A69D3F810904FF0000C61
:1006F00053F82210A568E246086800F00040B0F107
:10070000004F04D003F1140050F8220010B1022071
:10071000BDE8F08F0CF1010C2868886048686FF321
:100720000C00D5F804B040EA0B004860207800F0D7
:10073000010038B1086820F44000D4F814B040EA51
:100740000B000860207800F0200038B1086820F025
:100750004060D4F810B040EA0B000860207800F048
:10076000040018B1086840F080000860086840F094
:100770008050086000BF00BF00BFBFF35F8F00BFA5
:1007800000BF00BF086840F0004008605DE00868F6
:1007900020F00050086026B1086840F080400860F2
:1007A00003E0086820F08040086000BF521C042A63
:1007B00000D3121F00BF53F82210086820F08050A9
:1007C0000860086800F00040B0F1004F04D003F169
:1007D000140050F82200E8B14A4653F822100027CE
:1007E00014E000BF00BF00BFBFF35F8F00BF00BFBA
:1007F00000BF086820F00040086000BF521C042AB7
:1008000000D3121F00BF53F822107F1C6745E8D3A6
:1008100002207DE70CF1010CAD682868886048680B
:100820006FF30C00D5F804B040EA0B0048600AF101
:10083000010A00BF00BF00BFBFF35F8F00BF00BF52
:1008400000BF086840F000400860A86800289ED1FA
:1008500026B1086840F08040086003E0086820F096
:1008600080400860086840F00050086003F1140000
:10087000D3F824B040F822B01A6172B60AF1010030
:10088000D3F828B05844986262B6002040E70000D0
:1008900070B505460C46286800F5805086692B48DF
:1008A0000640207B08B9012000E000208006617B23
:1008B00040EA4160617F09B9012100E0002140EA7E
:1008C0000150A17B40EA415061690843217F40EA21
:1008D000C110A17F40EA8110216A084394F82410D6
:1008E00040EA81000643286800F580508661286848
:1008F00000F580508669012000F07EF9286800F537
:10090000805086612179A06840EA4160A16908436E
:100910002169084394F8251040EAC110A16A40EA11
:1009200081002168084340F40001286800F58050E8
:100930000160286800F580500668012000F05CF92D
:10094000286800F58050066070BD0000233FDEF887
:1009500070B505460C46286806683A480640207C73
:1009600008B9012000E00020C005617C09B901211F
:1009700000E0002140EA8150A1680843E17F40EA9D
:10098000014061690843A17F09B9012100E000210C
:1009900040EA4130217F40EA0130A16908432179D2
:1009A00040EA812094F8201009B9012100E00021DB
:1009B00040EA4120E17B40EAC110616A084394F8B3
:1009C000281040EA01100643286806602868066877
:1009D000012000F011F928680660286886694FF642
:1009E00041700640A06C000494F84C1009B9012134
:1009F00000E0002140EAC110216D084394F8551031
:100A0000012900D100E0002140EAC10094F856100D
:100A1000012900D100E0002140EA810094F854103F
:100A2000012900D100E0002140EA41000643286886
:100A3000866128688669012000F0DEF828688661F2
:100A400070BD00000F8120FF2DE9F843044600200F
:100A500000904FF00108A66E04F1480050F82650AF
:100A6000E76E2FE0286A58B9684600F007FC009846
:100A700010B94FF0000803E0009828620098A860C1
:100A8000B8F1000F1ED0A06D10B91648686002E0E2
:100A90004FF48C40686000BF00BF00BFBFF35F8FA2
:100AA00000BF00BF00BF286840F00040286000BFC2
:100AB000761C042E00D3361F00BF04F1480050F806
:100AC00026507F1E17B1B8F1000FCBD1E06EB842AF
:100AD00006D00021206800F580508160A666E76698
:100AE000BDE8F8830046008010B5042000F024FE25
:100AF00010BD72B600BFFEE770B50446B3F5804F77
:100B000013D1D1E9000540EA05108D6840EA0520BF
:100B10008D6928438D8940EA054054F82250064EDD
:100B20003540284344F8220003E06FF0704044F859
:100B30002200002070BD00000000F0CF70B502461A
:100B4000086852F8200020F001000E6842F82600E4
:100B50008868082801D1402300E000234868184332
:100B60008E683043CE6830430E6930434E6930435F
:100B7000CE6930430E6A30434E6A30438E6A30434A
:100B8000CE6A30430E6B40EA060488690443C86BA2
:100B90000443074D45F4806545F4E025086852F8A4
:100BA0002000A84320430E6842F82600002070BDB4
:100BB0007FFB080010B50346D1E9000440EA0410A9
:100BC0008C6840EA04208C8940EA0444088A401E6C
:100BD00044EA0054087D801E44EA00608C6920438A
:100BE000541C53F8244004F040442043541C43F860
:100BF0002400002010BD000070B5044600F0AAFEDD
:100C000006462546681C10B104480078054400BF1C
:100C100000F0A0FE801BA842FAD370BD1C0000208B
:100C200010B50446204600F00BF800F08000802844
:100C300003D10248006807F059FF10BD2C000020C6
:100C40000146D1F88C007047024609B9012070476F
:100C500010680068C0F3001081F828001068006870
:100C600000F06000486210680068C0F3402080F027
:100C7000010081F8200010680068C0F30040C877C8
:100C800010680068C0F3403080F001008877106879
:100C90000068C0F3003008771068006800F4006056
:100CA00088611068006800F480404861106800683E
:100CB000C0F3805080F00100487410680068C0F3F1
:100CC000C05080F00100087410680068C0F3C010C4
:100CD000C8731068006800F46020886010680068BD
:100CE000C0F38020087110688069C0F3400081F86B
:100CF000540010688069C0F3C01080F0010081F8D2
:100D00004C001068806900F0300008651068806948
:100D1000000C886410688069C0F3800081F8560078
:100D200010688069C0F3C00081F8550000208EE78C
:100D300010B50446206800F58050406900F040007E
:100D400040280FD1206800F58050C06900F04000B5
:100D5000402807D14249206800F580504161204673
:100D600000F0B0FA206800F58050406900F0010002
:100D700078B1206800F58050C06900F0010040B1F2
:100D80004FF00111206800F580504161204600F0CD
:100D90001DFC206800F58050406900F40040B0F56B
:100DA000004F3DD1206800F58050C06900F400403C
:100DB000B0F5004F34D1D4F8880040F00800C4F8F2
:100DC0008800206800F58050406900F40050B0F5BC
:100DD000005F15D1206800F5805040692149084026
:100DE000C4F88C00206800F58050C06920F4C03140
:100DF000206800F58050C161E020C4F884000CE058
:100E0000206800F58050406948F280610840C4F8CD
:100E10008C00206800F5805041612046FFF700FFFC
:100E20002068806B00F0080008280BD12068C06A99
:100E300000F06000C4F89400204600F02BF9002078
:100E4000C4F894000848006800F4002030B14FF462
:100E5000002005490860204600F0C8FB10BD0000D6
:100E60004000010000207E00143C014038B50446DB
:100E70000CB9012038BDD4F8840028B92320C4F867
:100E80008400204600F05CF800BF002000902A4853
:100E9000006840F48040284908600846006800F473
:100EA0008040009000BF00BF2448006820F400008C
:100EB0002249086008460068A16808431F49086085
:100EC00008460068206800F58050006840F0010185
:100ED000206800F58050016000F03CFD05460DE003
:100EE00000F038FD401BB0F5FA7F07D90420C4F8A4
:100EF0008800E020C4F884000120BBE7206800F5EA
:100F00008050006800F001000028E9D12046FFF77A
:100F100059FB2046FFF7E7FA2046FFF7ABFA00211E
:100F200020466268FFF734FB0020C4F888001020D8
:100F3000C4F8840000209DE7443802400438014092
:100F400010B586B00446142101A8FFF706FA4C49F3
:100F5000206888427ED100BF00BF00200090494831
:100F6000006840F00070474908600846006800F0DB
:100F70000070009000BF00BF00BF00200090084636
:100F8000006840F0806008600846006800F08060FB
:100F9000009000BF00BF00BF00200090084600681E
:100FA00040F0006008600846006800F000600090B3
:100FB00000BF00BF00BF00BF0020009008460068CF
:100FC00040F0040008600846006800F0040000904B
:100FD00000BF00BF00BF002000900846006840F03E
:100FE000010008600846006800F00100009000BFA2
:100FF00000BF00BF002000900846006840F00200DB
:1010000008600846006800F00200009000BF00BFC2
:1010100032200190022002900020039003200490CF
:101020000B20059001A9184800F094FB8620019040
:101030000220029000200390032004900B200590D2
:1010400001A9124800F086FB4FF460500190022085
:10105000029000E011E000200390032004900B2098
:10106000059001A90A4800F075FB002205213D20EA
:1010700000F034FD3D2000F021FD06B010BD000061
:101080000080024030380240000802400000024068
:101090000004024070472DE9F05F04460F464FF010
:1010A0000008C34647B9D4F8880040F00100C4F8EE
:1010B00088000120BDE8F09FD4F88400232801D0E7
:1010C0000120F7E7E66D04F1480050F82650E06E85
:1010D000C0F1040942E0286800F4807018B1A969E1
:1010E000A167E9696167286800F4007008B9E06FDA
:1010F00040B3286800F4007010B1002121666166D9
:10110000D4F814A0286800F4807040B12868C0F3B7
:101110000D40A0F1040A296821674FF0010BA8686F
:1011200028621FFA8AF304F18001081F2A6A00F07E
:10113000D3F8206E401C2066606E00EB0A016166E9
:101140000020286200BF761C042E00D3361F00BF8B
:1011500004F1480050F8265008F10108286800F012
:10116000004020B9C84502D2BBF1000FB3D0E06EF9
:1011700000EB0801E166E06E10B12046FFF764FC69
:10118000E665BBF1010F05D1E06F38600021E16732
:1011900000208FE701208DE72DE9F04705460E4638
:1011A000174698462868046904F01C044FF47840F8
:1011B00000EAC62004434FF4F86000EA87100443B5
:1011C00024F0020444F001042868046100F0C2FB2A
:1011D00081460BE000F0BEFBA0EB0900B0F5803FBC
:1011E00002D30120BDE8F0872868046904F00100FB
:1011F0000028EFD12868406980B2C8F800000020BC
:10120000F0E72DE9F047064606F11804A76AE56AFB
:101210004FF001082AE04FF001097F1E04F114008D
:1012200050F8250020B9681C00F003054FF00009B4
:10123000B9F1000F1AD005EB8501F06850F83100C4
:1012400000F0004080B904F1140151F8250000F0CD
:10125000C7F9002104F1140040F82510681C00F0C3
:101260000305A762E56201E04FF0000817B1B8F18D
:10127000000FD0D10020BDE8F08700007CB5044607
:101280000D4806F0BDFE054685B105F12000206041
:101290000A4828614FF4C06120682B464122CDE9FD
:1012A00000010021084607F0DFFE04E001200449A8
:1012B0000870002020607CBD88290108E1970008A3
:1012C0002800002010B504460248006807F00EFC14
:1012D00010BD00002C000020F0B504460D4621464C
:1012E0002E460020A2F120000027076007814381DD
:1012F0000F680FB9086001E037683860306008682F
:1013000003E007891F44078100680028F9D1F0BD78
:1013100070B504460D460DB9012070BDD4F88400A7
:10132000102805D129462046FFF712FB0020F4E7DC
:101330000120F2E770B506463068056925F01C0506
:1013400000F002FD04461348844205D3124884424B
:1013500002D245F008051AE00F48844205D30F4831
:10136000844202D245F00C0511E00C48844203D3BC
:101370000B48844200D20AE00948844205D3094858
:10138000844202D245F0040501E045F010053068C2
:10139000056170BD002D3101C00E16020087930358
:1013A00000E1F50580D1F00870B50446D4F884005A
:1013B00010285FD12320C4F884000121A165206892
:1013C000C06B40F402702168C8632068D0F80C013B
:1013D000294908432168C1F80C012068D0F81001A0
:1013E00040F403102168C1F810010421E166204691
:1013F000FFF72AFB2068006840F0080021680860B9
:10140000206805680120FFF7F7FB20680560206869
:10141000006840F004002168086020680568012029
:10142000FFF7EAFB206805602046FFF78DF820688B
:1014300000F58050806940F40051206800F580502C
:101440008161206800F58050806940F002012068C9
:1014500000F580508161206800F58050C06907491F
:101460000843216801F58051C8612320C4F8840035
:10147000002070BD0120FCE760000200C1A0010057
:101480002DE9F0410446D4F88400232851D1C4F852
:101490008400206800F58050C06927490840216811
:1014A00001F58051C861206800F58050806920F402
:1014B0000051206800F580508161206800F580505F
:1014C000806920F00201206800F580508161206869
:1014D000006820F004002168086020680768012087
:1014E000FFF78AFB206807602046FFF72DF8206889
:1014F000006820F008002168086020680768012063
:10150000FFF77AFB20680760002508E004F1480037
:1015100050F82560706840F0004070606D1C042D2C
:10152000F4D30021A1651020C4F884000020BDE898
:10153000F0810120FBE700003E5FFEFF70B504462E
:101540000D463DB9D4F8880040F00100C4F8880089
:10155000012070BDD4F88400232835D1696BE16384
:10156000012229462046FFF7B7F838B1D4F88800A1
:1015700040F00200C4F888000120EAE700BF00BF85
:1015800000BFBFF34F8F00BF00BF00BF00BFA06A06
:10159000401CA062A06A042802D3A06A001FA062B7
:1015A00000BF206800F58050406900F0040048B199
:1015B0000421206800F5805041610021206800F579
:1015C000805041600020C4E70120C2E710B5044606
:1015D0000248006807F08AFA10BD000030000020C1
:1015E00010B50446204608F027F810BD70472DE9D5
:1015F000F04705460E46174698462868046904F0E9
:101600001C044FF4784000EAC62004434FF4F8600D
:1016100000EA8710044344F0020444F001041FFA76
:1016200088F0296848612868046100F093F98146D0
:101630000BE000F08FF9A0EB0900B0F5803F02D37A
:101640000120BDE8F0872868046904F00100002843
:10165000EFD100BFF5E7000000B587B0142102A864
:10166000FEF77BFE2A48006808B107B000BD0120E4
:101670002749086000BF002001902648006840F01C
:101680000100244908600846006800F0010001904C
:1016900000BF00BF41F23F000290022003900020F3
:1016A0000490032005900C20069002A91A4800F02F
:1016B00051F84FF4F0600290022003900020049053
:1016C000032005900C20069002A9144800F042F86F
:1016D0004CF2B300029002200390002004900320FB
:1016E00005900C20069002A90D4800F033F84FF445
:1016F00000700290022003900020049003200590C7
:101700000C20069002A9074800F024F800BFACE7BF
:101710000C00002038380240001402400010024043
:10172000000C02400018024010B50446042C01D100
:1017300002F0ACFB10BD000010B504460448006880
:10174000204020B1024804602046FFF7EDFF10BDA5
:10175000143C0140F8B502460B4600250024002049
:101760000021D6E0012606FA01F51E6806EA050406
:10177000AC4274D11E7906F00306012E04D01E7906
:1017800006F00306022E13D190684F000326BE40D8
:10179000B0434F00DE68BE40304390605068012681
:1017A0008E40B0431E79C6F300168E403043506021
:1017B0001E7906F00306032E09D0D0684F000326D9
:1017C000BE40B0434F009E68BE403043D0601E799B
:1017D00006F00306022E13D1CF0802F1200656F8B8
:1017E00027004E07F70E0F26BE40B0434F07FF0EEF
:1017F0001E69BE403043CF0802F1200646F827009C
:1018000010684F000326BE40B0431E7906F0030661
:101810004F00BE40304310605E6806F44036002E34
:1018200076D000BF002600963C4E366846F48046CF
:101830003A4F3E603E46366806F48046009600BF4A
:1018400000BF374E8F0856F827008E07370F0F2638
:10185000BE40B043334EB24202D1002624E057E0EE
:10186000314EB24201D101261EE0304EB24201D1CA
:10187000022619E02E4EB24201D1032614E02D4E6D
:10188000B24201D104260FE02B4EB24201D105260F
:101890000AE02A4EB24201D1062605E0284EB242A5
:1018A00001D1072600E008268F073F0FBE403043D6
:1018B0001B4E8F0846F82700224E3068A0435E6812
:1018C00006F4801606B120431E4E3060361D306887
:1018D000A0435E6806F4001606B12043194E361D7B
:1018E0003060184E361F3068A0435E6806F400363C
:1018F00006B12043134E361F3060361F3068A043B8
:101900005E6806F4803606B120430E4E083E306015
:10191000491C1029FFF426AFF8BD000044380240EE
:101920000838014000000240000402400008024064
:10193000000C024000100240001402400018024057
:10194000001C0240083C01400AB1816101E00B0427
:101950008361704701480068704700001400002050
:101960000348006803490978084401490860704742
:10197000140000201C00002010B50D48006840F441
:1019800000700B4908600846006840F480600860F9
:101990000846006840F480700860032000F0DCF81E
:1019A0000F2000F007F800F05FF8002010BD0000E5
:1019B000003C02402DE9F04188B004460027B846BB
:1019C00000BF002001902348006840F00400214936
:1019D00008600846006800F00400019000BF00BFE6
:1019E00002A903A800F08EF9069F1FB900F0B2F912
:1019F000054602E000F0AEF945001748B5FBF0F0EF
:101A0000A0F1010815481649086040F2E731144872
:101A1000C160C0F80480002101618160816100F033
:101A2000F9FE064696B90E4800F028FF06466EB944
:101A30001E2000F043F8102C07D2002221461E2061
:101A400000F04CF80748046000E00126304608B07A
:101A5000BDE8F0814038024040420F0000080040DD
:101A60003C0500201800002008B500BF00200090B1
:101A70001148006840F480400F490860084600683B
:101A800000F48040009000BF00BF00BF0020009025
:101A9000081F006840F08050091F08600846006871
:101AA00000F08050009000BF00BF00220F21901E68
:101AB00000F014F808BD0000443802400146084612
:101AC000002809DB00F01F0301229A4043099B0014
:101AD00003F1E023C3F8002100BF70472DE9F05F58
:101AE00080460D461646002702F06EF80746394636
:101AF0002A46334601F00700C0F1070ABAF1040F85
:101B000002D94FF0040A01E0C0F1070AD14600F102
:101B1000040ABAF1070F02D24FF0000A01E0A0F167
:101B2000030AD4464FF0010A0AFA09FAAAF1010A97
:101B30000AEA020A0AFA0CFA4FF0010B0BFA0CFB44
:101B4000ABF1010B0BEA030B4AEA0B0421464046BA
:101B500002F042F8BDE8F09F00BF00F00702064B1C
:101B600019684FF6FF031940044B0B4343EA022167
:101B7000014B196000BF70470CED00E00000FA0552
:101B800070B504460D460CB9012070BD5848006878
:101B900000F00700A84209D255490D7008460068B8
:101BA00000F00700A84201D00120EEE7207800F005
:101BB000020002281DD1207800F00400042805D17D
:101BC0004C48006840F4E0504A490860207800F032
:101BD0000800082805D14748006840F4604045499E
:101BE00008604448006820F0F000A16808434149BB
:101BF0000860207800F00100A8B36068012807D1D0
:101C00003C4808380068C0F34040B8B90120BCE740
:101C10006068022802D06068032807D13548083878
:101C20000068C0F3406048B90120AEE73148083889
:101C30000068C0F3400008B90120A6E72D480068FD
:101C400020F00300616808432A490860FFF782FE1C
:101C5000064609E0FFF77EFE801B41F2883188428C
:101C600002D9032091E707E02248006800F00C0049
:101C70006168B0EB810FEDD11D48006800F00700EE
:101C8000A84209D91A490D700846006800F00700FB
:101C9000A84201D0012078E7207800F00400042851
:101CA00007D11448006820F4E050E1680843114966
:101CB0000860207800F00800082808D10D48006866
:101CC00020F46040216940EAC1000A49086000F040
:101CD00051F808490968C1F30311074A515CC8402B
:101CE0000649086006480068FFF764FE00204CE7DC
:101CF000003C024008380240702901082000002002
:101D0000180000200F2202600D4A126802F0030240
:101D100042600B4A126802F0F0028260084A1268C0
:101D200002F4E052C260064A126802F46042D2082D
:101D30000261044A126802F007020A60704700005C
:101D400008380240003C024001480068704700002B
:101D50002000002000B5FFF7F7FF04490968C1F330
:101D60008221034A515CC84000BD0000083802408F
:101D7000802901082DE9F047002400250026A1460E
:101D80002548006800F00C0020B1042805D0082880
:101D90003AD105E0DFF8849039E0DFF8849036E04E
:101DA0001D48001F006800F03F041B48001F00682A
:101DB00000F4800078B11A481749091F0968C1F377
:101DC0008811A0FB01700146224600233846FEF729
:101DD00059FA05460EE011480F49091F0968C1F379
:101DE0008811A0FB01700146224600233846FEF709
:101DF00049FA05460848001F0068C0F30140401C2E
:101E00004600B5FBF6F902E0DFF8109000BF00BF16
:101E10004846BDE8F0870000083802400024F4007E
:101E200000C0A800F8B504460CB90120F8BD207820
:101E300000F00100002874D0F948006800F00C00A0
:101E400004280DD0F648006800F00C00082813D1D3
:101E5000F348001F006800F48000B0F5800F0BD13C
:101E6000EF4808380068C0F34040002859D0606847
:101E7000002856D10120D9E700BF6068B0F5803F47
:101E800008D1E7480838006840F48030E449083950
:101E900008601EE06068B0F5A02F0DD1E04808385A
:101EA000006840F48020DE49083908600846006870
:101EB00040F4803008600CE0D9480838006820F40D
:101EC0008030D749083908600846006820F480202F
:101ED000086000BF606890B1FFF73CFD054606E072
:101EE000FFF738FD401B642801D903209EE7CC484A
:101EF00008380068C0F340400028F1D011E0FFF737
:101F000029FD054606E0FFF725FD401B642801D9A1
:101F100003208BE7C24808380068C0F3404000281F
:101F2000F1D1207800F0020002285FD1BC4800689F
:101F300000F00C0058B1BA48006800F00C00082806
:101F40001CD1B748001F006800F48000B0B9B44845
:101F500008380068C0F3400020B1E068012801D0D3
:101F6000012063E7AE480838006820F0F8002169D6
:101F700040EAC100AA490839086037E0E06800B3C8
:101F80000120A8490860FFF7E5FC054606E0FFF7D9
:101F9000E1FC401B022801D9032047E7A04808388C
:101FA0000068C0F340000028F1D09D480838006860
:101FB00020F0F800216940EAC10099490839086019
:101FC00014E0002097490860FFF7C4FC054606E0CE
:101FD000FFF7C0FC401B022801D9032026E79048E8
:101FE00008380068C0F340000028F1D1207800F0E4
:101FF000080008282CD16069A8B101208A4908602E
:10200000FFF7A8FC054606E0FFF7A4FC401B0228EA
:1020100001D903200AE782486C300068C0F3400011
:102020000028F1D014E000207F490860FFF792FCFF
:10203000054606E0FFF78EFC401B022801D903206D
:10204000F4E677486C300068C0F340000028F1D116
:10205000207800F00400042870D100277048383040
:10206000006800F0805090B900BF002000906C48DC
:102070003830006840F080506949383108600846BF
:10208000006800F08050009000BF00BF0127674843
:10209000006800F48070B0B96448006840F4807053
:1020A00062490860FFF756FC054606E0FFF752FC60
:1020B000401B022801D90320B8E65C48006800F400
:1020C00080700028F2D000BFA068012808D15448D1
:1020D0006830006840F001005149683108601DE037
:1020E000A06805280DD14E486830006840F0040013
:1020F0004B49683108600846006840F001000860FC
:102100000CE047486830006820F00100444968311D
:1021100008600846006820F00400086000BFA0685E
:10212000A8B1FFF717FC054609E0FFF713FC401BB9
:1021300041F28831884202D9032077E626E0384808
:1021400068300068C0F340000028EED013E0FFF7CD
:1021500001FC054608E0FFF7FDFB401B41F288311A
:10216000884201D9032061E62D4868300068C0F339
:1021700040000028EFD1012F07D1294838300068EE
:1021800020F0805026493831086000BFA06900283F
:1021900045D02348006800F00C0008285DD0A069F5
:1021A000022845D100201F490866FFF7D3FB0546EA
:1021B00006E0FFF7CFFB401B022801D9032035E6DC
:1021C000174808380068C0F340600028F1D1D4E90E
:1021D00007010843616A40EA81110122A06AC2EB4B
:1021E000500041EA00412C20005D41EA00600C49AA
:1021F000091F086001200B490866FFF7ABFB054685
:1022000006E0FFF7A7FB401B022801D903200DE6DB
:10221000034808380068C0F340600028F1D049E066
:102220000838024000004742800E474200700040DC
:10223000002021490866FFF78DFB054606E0FFF701
:1022400089FB401B022801D90320EFE51B480068E9
:10225000C0F340600028F2D12CE0A069012800D131
:10226000E4E51648001D0668A069012820D006F4A0
:102270008001E06981421BD106F03F01206A814262
:1022800016D147F6C0703040616AB0EB811F0FD1A4
:1022900006F440310122A06AC2EB5000B1EB004FBE
:1022A00006D106F070612C20005DB1EB006F01D00B
:1022B0000120BBE50020B9E500004742003802409C
:1022C00010B504460CB9012010BD606A38B96068C9
:1022D000B0F5827F00D105E00021E16102E000213C
:1022E000216161610021A16294F8510028B90020A8
:1022F00084F85000204600F047F8022084F851008E
:102300002068006820F0400021680860A08800F480
:102310008270218901F404410843A18901F400611C
:102320000843217C01F002010843217D01F00101F5
:102330000843218B01F400710843217F01F038012B
:1023400008432021095D01F080010843218D01F43B
:1023500000510843216808600421A06901EA104087
:1023600094F8241001F010010843216848602068A7
:10237000C06920F400602168C86100206065012008
:1023800084F8510000209FE710B586B00446142160
:1023900001A8FDF7E2FF1B49206888422FD100BF4A
:1023A000002000901848006840F4805016490860EA
:1023B0000846006800F48050009000BF00BF00BFD6
:1023C0000020009010481438006840F002000E49C8
:1023D000143908600846006800F00200009000BF51
:1023E00000BF3820019002200290002003900320BB
:1023F00004900520059001A90448FFF7ABF906B049
:1024000010BD00000030014044380240000402408A
:102410002DE9FF5F0446884691461D460E9E012029
:1024200002900020019000BF94F85000012803D1D1
:10243000022004B0BDE8F09F012084F8500000BFE6
:10244000FFF788FA074694F851B060680390AA46EF
:10245000BBF1010F0BD00398B0F5827F04D1A068C7
:1024600010B9BBF1040F02D002200190DBE0B8F1FB
:10247000000F03D0B9F1000F00D015B90120019071
:10248000D1E094F85100042802D0052084F85100CE
:1024900000206065C4F83890E587A587C4F83080CF
:1024A000E586A586206460642068006800F040002E
:1024B000402805D02068006840F04000216808608E
:1024C000E068B0F5006F4AD1606810B1BAF1010F51
:1024D00009D1206B00882168C860206B801C2063B4
:1024E000E08E401EE08633E02068806800F0020045
:1024F000022810D1E08E70B1029801280BD1206B18
:1025000000882168C860206B801C2063E08E401E1C
:10251000E086002002902068806800F0010068B129
:10252000E08F58B12068C068A16B0880A06B801C48
:10253000A063E08F401EE08701200290FFF70AFAB7
:10254000C01BB04204D3701C10B1032001906AE09C
:10255000E08E0028C8D1E08F0028C5D14AE060682D
:1025600010B1BAF1010F09D1206B0078216808730E
:10257000206B401C2063E08E401EE08634E0206823
:10258000806800F00200022810D1E08E70B102983D
:1025900001280BD1206B007821680873206B401C48
:1025A0002063E08E401EE086002002902068806854
:1025B00000F0010068B1E08F58B12068C068A16BDD
:1025C0000870A06B401CA063E08F401EE0870120D4
:1025D0000290FFF7BFF9C01BB04201D3701C00B9D5
:1025E00016B9032001901EE0E08E0028C7D1E08FCD
:1025F0000028C4D13A463146204601F053F820B1B4
:1026000001200190202060650DE0A06850B900BF56
:10261000002000902068C0680090206880680090CA
:1026200000BF00BF00BF012084F8510000BF0020A0
:1026300084F8500000BF0198FBE670B504460E46D2
:1026400015460CB9012070BD94F8490028B9002046
:1026500084F84800204600F01FF804F108012068C3
:10266000FEF76CFA3146A2682068FEF7A3FA294605
:10267000236BD4E90102FEF73FFAA168206850F805
:10268000210040F00100A268216841F822000120E9
:1026900084F849000020D6E710B50446FEF7DCFFB9
:1026A00010BDF0B504460D4616462F46B44694F8C4
:1026B0004920012A01D0042A1FD100BF94F8480004
:1026C000012801D10220F0BD012084F8480000BF9C
:1026D000022084F84900194606E038788CF800009A
:1026E0000CF1010C7F1C491E0029F6D184F8492009
:1026F00000BF002084F8480001E00120E3E700204B
:10270000E1E7F0B504460D462E46174694F8490019
:1027100001281ED100BF94F84800012801D10220F1
:10272000F0BD012084F8480000BF022084F8490071
:10273000194604E0387830707F1C761C491E002949
:10274000F8D1012084F8490000BF002084F8480037
:1027500001E00120E4E70020E2E770477047000055
:1027600030B502460B4600BF92F83C00012801D16B
:10277000022030BD012082F83C0000BF022082F818
:102780003D00106844681068816824F0700418687F
:10279000044310684460184D1068A8421BD01068AC
:1027A000B0F1804F17D0154D1068A84213D0144DCA
:1027B0001068A8420FD0134D1068A8420BD0124DDC
:1027C0001068A84207D0114D1068A84203D0104DE0
:1027D0001068A84205D121F08001586801431068B3
:1027E0008160012082F83D0000BF002082F83C009B
:1027F00000BF00BFBDE70000000001400004004032
:1028000000080040000C004000040140004001406E
:102810000018004010B504460CB9012010BD94F812
:102820003D0028B9002084F83C00204600F025F83F
:10283000022084F83D00211D206801F059F8012094
:1028400084F8460000BF84F83E0001213F20015576
:10285000402001554120015500BF00BF012084F8F0
:10286000420043200155442001554520015500BF39
:10287000012084F83D000020D0E77047014691F820
:102880003D00012801D001207047022081F83D0061
:102890000868C06840F001000B68D8601A4B0868EF
:1028A00098421BD00868B0F1804F17D0174B0868CA
:1028B000984213D0164B086898420FD0154B086801
:1028C00098420BD0144B0868984207D0134B086805
:1028D000984203D0124B086898420CD1086880686F
:1028E00000F00702062A0CD00868006840F00100DA
:1028F0000B68186005E00868006840F001000B688C
:1029000018600020C0E70000000001400004004003
:1029100000080040000C004000040140004001405D
:1029200000180040704710B5044620680069C0F3E5
:102930004000D8B12068C068C0F34000B0B16FF06B
:10294000020021680861012020772068806900F07A
:10295000030018B12046FFF7E5FF05E0204600F030
:10296000DDF8204600F0A8F90020207720680069F3
:10297000C0F38000D8B12068C068C0F38000B0B157
:102980006FF00400216808610220207720688069C8
:1029900000F4407018B12046FFF7C4FF05E0204660
:1029A00000F0BCF8204600F087F90020207720686E
:1029B0000069C0F3C000D8B12068C068C0F3C0008F
:1029C000B0B16FF00800216808610420207720680A
:1029D000C06900F0030018B12046FFF7A3FF05E02F
:1029E000204600F09BF8204600F066F90020207792
:1029F00020680069C0F30010D8B12068C068C0F337
:102A00000010B0B16FF01000216808610820207735
:102A10002068C06900F4407018B12046FFF782FFBB
:102A200005E0204600F07AF8204600F045F9002045
:102A300020772068006900F0010058B12068C06864
:102A400000F0010030B16FF00100216808612046FC
:102A500000F0BAF920680069C0F3C01058B12068CE
:102A6000C068C0F3C01030B16FF080002168086109
:102A70002046FFF772FE20680069C0F3801058B14D
:102A80002068C068C0F3801030B16FF0400021684A
:102A90000861204600F0A4F920680069C0F34010E6
:102AA00058B12068C068C0F3401030B16FF020000A
:102AB000216808612046FFF751FE10BD10B586B0B1
:102AC0000446142101A8FDF748FC2068B0F1804FAE
:102AD0001DD100BF002000900E48006840F00100AA
:102AE0000C4908600846006800F00100009000BF33
:102AF00000BF0820019002200290002003900320D4
:102B000004900120059001A90348FEF723FE06B0BA
:102B100010BD0000303802400000024070472DE92F
:102B2000F04104460D461646002700BF94F83C00CD
:102B3000012802D10220BDE8F081012084F83C0088
:102B400000BF36B1042E1BD0082E31D00C2E5ED122
:102B500045E02946206800F049FF2068806940F080
:102B60000800216888612068806920F004002168DD
:102B7000886120688069296908432168886148E084
:102B80002946206800F06AFF2068806940F40060F0
:102B9000216888612068806920F4806021688861EC
:102BA00020688069296940EA01202168886130E055
:102BB0002946206800F090FF2068C06940F00800B6
:102BC0002168C8612068C06920F004002168C861DC
:102BD0002068C069296908432168C86119E029464D
:102BE000206800F0B5FF2068C06940F400602168EB
:102BF000C8612068C06920F480602168C8612068CD
:102C0000C069296940EA01202168C86101E0012703
:102C100000BF00BF00BF002084F83C0000BF384662
:102C200089E710B504460CB9012010BD94F83D00A9
:102C300028B9002084F83C00204600F025F8022046
:102C400084F83D00211D206800F052FE012084F828
:102C5000460000BF84F83E0001213F20015540207E
:102C600001554120015500BF00BF012084F84200FA
:102C700043200155442001554520015500BF012046
:102C800084F83D000020D0E708B50168B1F1804F1D
:102C90000FD100BF002100910649096841F00101F0
:102CA000044A11601146096801F00101009100BF5A
:102CB00000BF08BD403802407047000070B50446B0
:102CC0000D4615B994F83E000BE0042D02D13F20CB
:102CD000005D06E0082D02D14020005D01E04120AA
:102CE000005D012801D0012070BD1DB9022084F8CB
:102CF0003E000EE0042D03D102213F20015508E0E3
:102D0000082D03D102214020015502E0022141207B
:102D1000015501222946206800F056FE234920680B
:102D2000884203D022492068884201D1012000E076
:102D3000002028B12068406C40F4004021684864BD
:102D40001A49206888421BD02068B0F1804F17D004
:102D500018492068884213D01749206888420FD04C
:102D60001649206888420BD011492068884207D054
:102D700013492068884203D01249206888420CD148
:102D80002068806800F00706062E0CD020680068D6
:102D900040F001002168086005E02068006840F00C
:102DA00001002168086000209EE70000000001404B
:102DB000000401400004004000080040000C0040F6
:102DC000004001400018004010B504460349206847
:102DD000884201D1FEF7C4FD10BD0000000800408C
:102DE000704700BFFEE738B50446002000906A46F1
:102DF0000121636920689847002802DA6FF0040017
:102E000038BD6A460121636920689847002802DAC4
:102E10006FF00400F4E7009800F0040008B9012006
:102E2000EEE76A460021636920689847002802DAC5
:102E30006FF00400E4E7009800F48050B0F5805F84
:102E40001FD0009800F40050B0F5005F07D1009843
:102E500000F48070B0F5807F01D10220D0E70098A7
:102E600000F40050B0F5005F01D10320C8E70098DE
:102E700000F48070B0F5807F01D10420C0E7052008
:102E8000BEE76A461F21636920689847002802DA76
:102E90006FF00400B4E7009800F4805008B90620F1
:102EA000AEE7009800F01C00182801D10220A7E727
:102EB000009800F01C00082801D10320A0E700982A
:102EC00000F01C00142801D1042099E7052097E7A1
:102ED000F8B5044600270020009000250026606811
:102EE000002855D1A06808B1A06880472020206044
:102EF000002513E06A461221284663699847002896
:102F000002DA6FF0040608E0009800F01F00A84203
:102F100002D12560002603E000BF6D1C1F2DE9D9FA
:102F200000BF20681F2801D96FF0020656BB4FF47E
:102F300000420021236920689847002826DB6A4662
:102F4000002163692068984700281CDBA06980473E
:102F5000074612E0A0698047C01BB0F5FA7F09D888
:102F60006A460021636920689847002805DA6FF0F7
:102F7000040607E06FF0010604E0009800F400404A
:102F80000028E7D104E06FF0040601E06FF00306CB
:102F90005EB9A0698047074600BFA0698047C01B93
:102FA000B0F5FA6FF9D9012060603046F8BD0246ED
:102FB0002AB1C86818B1886808B1086910B94FF01B
:102FC000FF307047086890604B68D360CB685361EE
:102FD0008B6813610B6993610020F2E700B595B02F
:102FE0001C2212490EA8FDF791F900210EA805F048
:102FF000D9FD0F4908601C220C491C3107A8FDF7B8
:1030000085F9002107A805F0CDFD0A4908601C22BA
:10301000064938316846FDF779F90021684605F020
:10302000C1FD0549086015B000BD00001C2901085C
:1030300000000020040000200800002000B587B038
:103040001C216846FDF789F94FF020402F490860A0
:103050002F4848600020886000212C48C160016131
:1030600041618161C161016241624FF480518162BD
:103070000021C16201634163816341640A200090C1
:103080000F2001900A2002900F200390102004903E
:103090001120059000200690002269461B48FFF78A
:1030A000CCFA08B1FDF725FD4FF020401949086022
:1030B000174848600220886000211648C1600161FD
:1030C00041618161C161016241624FF4805181625D
:1030D0000021C16201634163816341640F2000905C
:1030E00001900A2002900F200390102004901120DC
:1030F000059000200690002269460648FFF79DFAD9
:1031000008B1FDF7F6FC07B000BD0000FC0300208D
:10311000040100A04C04002000B587B0142102A8CF
:10312000FDF71BF900BF002001908D48006840F0BA
:1031300010008B4908600846006800F010000190FC
:1031400000BF00BF00BF002001900846006840F0AB
:10315000200008600846006800F02000019000BFD1
:1031600000BF00BF002001900846006840F08000CA
:1031700008600846006800F08000019000BF00BFB2
:1031800000BF002001900846006840F0040008607D
:103190000846006800F00400019000BF00BF00BFB7
:1031A000002001900846006840F0010008600846D1
:1031B000006800F00100019000BF00BF00BF0020C8
:1031C00001900846006840F0020008600846006868
:1031D00000F00200019000BF00BF00BF002001907E
:1031E0000846006840F0400008600846006800F0AB
:1031F0004000019000BF00BF00BF002001900846C2
:10320000006840F0080008600846006800F0080008
:10321000019000BF00BF012242F63F015148FEF776
:1032200093FB01224FF4A0714F48FEF78DFB012262
:1032300048F610214D48FEF787FB012240F2C131CC
:103240004B48FEF781FB00224FF480414648FEF7D1
:103250007BFB01224FF655414648FEF775FB0122E4
:1032600041F248514448FEF76FFB0122D102434826
:10327000FEF76AFB42F63F000290012003900490A3
:103280000320059002A93748FEF764FA4FF4A070B6
:1032900002900120039004900320059002A9324877
:1032A000FEF758FA48F6102002900120039004908F
:1032B0000320059002A92D48FEF74CFA40F2C130D8
:1032C00002900120039004900320059002A9284851
:1032D000FEF740FA4FF48040029001200390022054
:1032E00004900320059002A91F48FEF733FA4FF619
:1032F000554002900120039004900320059002A9FC
:103300001C48FEF727FA41F2485002900120039032
:1033100004900320059002A91748FEF71BFA4FF40A
:10332000006002900120039004900320059002A900
:103330001248FEF70FFA042002904FF40410039095
:103340000120049002A90C48FEF704FA002205218E
:103350000820FEF7C3FB0820FEF7B0FB07B000BD56
:1033600030380240001002400014024000000240C9
:103370000004024000180240000C02400008024015
:1033800000B58BB0C0208B490870A8204870012080
:103390008870C820C870FF208749087048708870FE
:1033A0000020C870C02085490870A82048700120FE
:1033B0008870DE20C870002108460DF063FA7D4851
:1033C000007800067B49497840EA014079498978CC
:1033D00040EA01207749C978084302067548007819
:1033E00000067449497840EA01407249897840EA08
:1033F00001207049C978084300F47F4042EA002266
:103400006C48007800066B49497840EA01416948F8
:10341000807841EA00206749C978084300F47F00BA
:1034200042EA10226348007801066248407841EA87
:1034300000416048807841EA00205E49C97808432D
:1034400042EA10605E4908605B48007800065A490D
:10345000497840EA01405849897840EA01205649B4
:10346000C978084302065448007800065249497852
:1034700040EA01405049897840EA01204E49C97824
:10348000084300F47F4042EA00224B4800780006DF
:103490004949497840EA01414748807841EA00209B
:1034A0004549C978084300F47F0042EA10224248A7
:1034B000007801064048407841EA00413E48807863
:1034C00041EA00203C49C978084342EA10603D497E
:1034D00008603A48007800063849497840EA0140D7
:1034E0003649897840EA01203449C9780843020600
:1034F0003248007800063149497840EA01402F49B6
:10350000897840EA01202D49C978084300F47F40BA
:1035100042EA00222948007800062849497840EA12
:1035200001412648807841EA00202449C9780843AF
:1035300000F47F0042EA10222048007801061F486C
:10354000407841EA00411D48807841EA00201B494B
:10355000C978084342EA10601B4908601B481C49AF
:103560000022194BCDE900210290164A144919484E
:1035700004F092FD174805F001F8164890F82D0068
:10358000C0F3800018B1134805F038F902E0114883
:1035900004F0FAFF10490F4805F05CF81C220F49AF
:1035A00004A8FCF7B3FE0B4904A805F0FBFA0BB026
:1035B00000BD000054000020580000205C000020E6
:1035C000480000204C000020500000207D0A010827
:1035D000C557000850510020E9550008B0290108DE
:1035E00010B50E480E4908604FF482704860002103
:1035F0000B488160C160016141614FF400718161DC
:103600003821C16100210162416281620A21C162E7
:10361000FEF756FE08B1FDF76CFA10BD0030014010
:103620009C04002000B589B00020079008901C2160
:103630006846FCF792FE4FF0804017490860002072
:1036400048600021144881607721C1600021016138
:103650008161FFF7E6FA08B1FDF74BFA0020079009
:10366000089007A90C48FFF77BF808B1FDF741FA6D
:10367000602000903C2001900020029004900C22D9
:1036800069460548FFF74BFA08B1FDF732FA0248E0
:10369000FFF714FA09B000BDF404002000BFFEE7F4
:1036A00000BFFEE77CB504460D4616461648006886
:1036B0001821B0FBF1F01549B0FBF1F04FF47A712D
:1036C000484301906068B0F5827F0DD12B460022FF
:1036D00080212046009600F01BF898B1606D40F004
:1036E0002000606503207CBD00BF019800B908E0A0
:1036F0000198401E019020688068C0F3C010002827
:10370000F3D100BF0020EEE72000002040420F0070
:103710002DE9F84F04460D4690461E46DDF82890E8
:10372000FEF718F9A0EB0900371AFEF713F98246E5
:103730002C480068C0F3CB307843009045E0701C03
:10374000002842D0FEF706F9A0EB0A00B84200D2EA
:10375000A7BB2068406820F0E000216848606068EE
:10376000B0F5827F0DD1A068B0F5004F03D0A068FE
:10377000B0F5806F05D12068006820F04000216816
:103780000860A06AB0F5005F0DD100BF2068006836
:1037900020F40050216808602068006840F4005060
:1037A0002168086000BF012084F8510000BF00209C
:1037B00084F8500000BF0320BDE8F88FFFE70098B1
:1037C00000B900270098401E0090206880682840BB
:1037D000A84201D1012000E000204045AFD10020E7
:1037E000EAE700002000002010B500BF502080F361
:1037F0001188BFF34F8FBFF36F8F00BF0EF05CFED9
:1038000018B14FF080500449086000BF002080F3D9
:10381000118800BF10BD000004ED00E000B593B0BA
:10382000302107A8FCF799FD142102A8FCF795FDAB
:1038300000BF002001902348006840F080502149DB
:1038400008600846006800F08050019000BF00BF8B
:1038500000BF002001901C48006840F480401A49D5
:1038600008600846006800F48040019000BF00BF77
:10387000012007900004089002200D9041050E9150
:1038800006210F91782110910221119104211291AA
:1038900007A8FEF7C7FA08B1FDF72BF90F20029031
:1038A00002200390002004904FF4A0500590069051
:1038B000032102A8FEF764F908B1FDF71AF913B065
:1038C00000BD00004038024000700040034800681E
:1038D00040F47000014908607047000088ED00E086
:1038E00010B50248FFF71FF810BD00003C0500208E
:1038F00010B50268294B98420ED0B0F1804F0BD022
:10390000274B984208D0274B984205D0264B984227
:1039100002D0264B984203D122F070024B681A4322
:103920001E4B984220D0B0F1804F1DD01C4B9842C6
:103930001AD01C4B984217D01B4B984214D01B4BEB
:10394000984211D01A4B98420ED01A4B98420BD085
:10395000194B984208D0194B984205D0184B984201
:1039600002D0184B984203D122F44072CB681A431C
:1039700022F080034C6943EA040202608B68C36250
:103980000B688362054B984202D0084B984201D1E4
:103990000B6903630123436110BD00000000014077
:1039A0000004004000080040000C004000040140FA
:1039B0000040014000440140004801400018004020
:1039C000001C00400020004030B501F01F0501241C
:1039D00004FA05F3046A9C430462046A01F01F05BB
:1039E00002FA05F52C43046230BD000030B5056ACB
:1039F00025F001050562026A4368846924F07004B9
:103A000024F003040D682C4322F002028D682A433F
:103A1000104DA84200D103E00F4DA84206D100BFCF
:103A200022F00802CD682A4322F00402094DA84280
:103A300002D0094DA84207D123F4807323F4007308
:103A40004D692B438D692B43436084614D68456309
:103A5000026230BD000001400004014030B5056A3B
:103A600025F010050562026A4368846924F4E04485
:103A700024F440740D6844EA052422F020028D6885
:103A800042EA0512124DA84200D103E0114DA842AE
:103A900007D100BF22F08002CD6842EA051222F071
:103AA00040020B4DA84202D00A4DA84209D123F48E
:103AB000806323F400634D6943EA85038D6943EA1B
:103AC0008503436084614D688563026230BD0000F8
:103AD000000001400004014030B5056A25F48075FE
:103AE0000562026A4368C46924F0700424F0030488
:103AF0000D682C4322F400728D6842EA0522124DB3
:103B0000A84200D103E0114DA84207D100BF22F422
:103B10000062CD6842EA052222F480620A4DA84282
:103B200002D00A4DA84209D123F4805323F4005354
:103B30004D6943EA05138D6943EA05134360C46187
:103B40004D68C563026230BD0000014000040140C1
:103B500030B5056A25F480550562036A4468C26978
:103B600022F4E04222F440720D6842EA052223F476
:103B700000538D6843EA0533084DA84202D0084D32
:103B8000A84204D124F480444D6944EA8514446079
:103B9000C2614D680564036230BD00000000014051
:103BA0000004014000BFFEE70FB4054B10B503A9A8
:103BB000044A029800F034F810BC5DF814FB0000D1
:103BC0009D5800089C01002002480068C0F30220B4
:103BD000704700000CED00E010B5002804DB0A0778
:103BE000130E054A135406E00A07140E034A00F0A8
:103BF0000F031B1FD45410BD00E400E018ED00E0DB
:103C000002E008C8121F08C1002AFAD170477047A5
:103C1000002001E001C1121F002AFBD17047000003
:103C20002DE9FF4F8BB09A460F460546002606E069
:103C300025280BD052460D9990476D1C761C28788C
:103C40000028F5D10FB03046BDE8F08F0024A04623
:103C50000122604900E0044315F8013F203B02FACD
:103C600003F00842F7D128782E2817D115F8010F54
:103C700044F004042A280ED06FF02F022878A0F117
:103C8000300109290AD808EB880102EB410100EB59
:103C900001086D1CF2E757F8048B6D1C2878692821
:103CA0003ED006DC0028CDD063280BD0642804D198
:103CB00036E0732810D075284BD052460D999047A6
:103CC000761C85E017F8040B8DF8000000208DF8B5
:103CD0000100E946012003E057F8049B4FF0FF3054
:103CE00061074FF0000401D40AE0641C44450DDA7A
:103CF0008442FADB19F804100029F6D106E0641CAE
:103D00008442FCDB19F804100029F8D1264404E0B1
:103D100019F8010B52460D999047641EF8D257E0EE
:103D200001CF4FF00A0B002802DA40422D2102E0B9
:103D3000210504D52B218DF82410012103E0E10792
:103D400005D02021F7E70DF1200908910CE00021B2
:103D5000F9E701CF4FF00A0BF9E75946FCF715FBDD
:103D600001F1300209F8012D0028F6D1ADEB090070
:103D700000F1200B600701D44FF00108D84502DDA7
:103D8000A8EB0B0000E000208046002406E009A814
:103D90005246005D0D999047641C761C0898844239
:103DA000F5DB04E0302052460D999047761CB8F1BF
:103DB0000001A8F10108F5DC05E019F8010B5246F5
:103DC0000D999047761CBBF10001ABF1010BF4DCBF
:103DD0006D1C34E70928010070B504460025082C45
:103DE00000DA03E00125A4F10800C4B20448005D34
:103DF00040F002010122284600F0CEF870BD00001C
:103E0000342B010810B500F031F9FA20FCF7F4FE6C
:103E1000002409E04FF49661204600F02BF820467C
:103E200000F006F8601CC4B2102CF3DB10BD0000DB
:103E300070B504460025082C00DA03E00125A4F142
:103E40000800C4B20A48005D40F0010101230722C6
:103E5000284600F0B1F92046FFF7BEFF0448005D98
:103E600040F0040101230822284600F0A5F970BDA6
:103E7000342B010870B504460D46204600F07CF94D
:103E80002946204600F032F970BD00002DE9F041CE
:103E9000002701224F21384600F07EF805460DB973
:103EA000BDE8F08100246CE03848005D284000281F
:103EB00065D03748005D40F002010122384600F02D
:103EC0006BF800F00F06042E2BD006DC002E4BD032
:103ED000012E07D0022E50D105E0062E3BD00C2E2D
:103EE0004BD104E04AE0204601F0FEFC46E004EB42
:103EF0000420284A8118204600F070F804EB0421C1
:103F0000244A114481F8000104EB042013461844AC
:103F100090F8002104EB0420C118204600F0C2F8FC
:103F20002CE004EB04201B4A8118204600F056F8D0
:103F300004EB0421174A114481F8000104EB04202A
:103F40001346184490F8002104EB0420C1182046C1
:103F500000F0A8F812E00E48005D40F005010122D3
:103F6000384600F019F809E00948005D40F0060104
:103F70000122384600F010F800E000BF00BF601CCE
:103F8000C4B2082C90DB00BF8AE700003C2B01087C
:103F9000342B010860C80020F8B504460D461646CB
:103FA0000020009044B905F1C04733466A463946BF
:103FB0000848FEF776FB0AE0012C08D105F1C84756
:103FC00033466A4639460448FEF76BFB00BF9DF84E
:103FD0000000F8BDFC0300204C0400202DE9F04750
:103FE00004460E46002537464FF47A78A946082C39
:103FF00000DA04E04FF00109A4F10800C4B207E0C0
:10400000A8F101001FFA80F8B8F1000F00D10BE011
:104010001548005D40F0050101224846FFF7BCFF4E
:1040200000F001000028EBD000BF0CE00E48015D5D
:1040300001224846FFF7B0FF38707F1C681CC5B2EC
:10404000702D00D10BE00848005D40F00501012211
:104050004846FFF7A1FF00F001000028E6D100BFAD
:104060002846BDE8F0870000342B010810B5002475
:1040700013E00B48005D40F0010101238022002085
:1040800000F09AF80648005D40F00101012380220B
:10409000184600F091F8601CC4B2082CE9DB10BD92
:1040A000342B01082DE9F04104460E461746204600
:1040B00001F09AFC4FF00008082C00DA04E04FF001
:1040C0000108A4F10800C4B2002508E0725D0648AA
:1040D000015D0123404600F06FF8681CC5B2BD4287
:1040E000F4DBBDE8F0810000342B01082DE9F0413C
:1040F00004460F460025A846082C00DA04E04FF0DD
:104100000108A4F10800C4B21A48005D40F00301A0
:1041100001224046FFF740FF054645F0800515485F
:10412000005D40F0030101232A46404600F044F8B8
:104130004FF4E130B0FBF7F086B2F2B20D48015D0A
:104140000123404600F038F832120A48005D40F082
:1041500001010123404600F02FF805F07F050548D6
:10416000005D40F0030101232A46404600F024F898
:10417000BDE8F081342B010870B504460025082CF9
:1041800000DA03E00125A4F10800C4B20948005D8B
:1041900040F0030101230B22284600F00DF80548EA
:1041A000005D40F002010123C122284600F004F81E
:1041B00070BD0000342B01082DE9FF4104460D4677
:1041C0001E4644B905F1C047334602AA394608489D
:1041D000FEF797FA0AE0012C08D105F1C8473346EB
:1041E00002AA39460348FEF78CFA00BFBDE8FF81FA
:1041F000FC0300204C04002010B50446102C69D2AA
:10420000DFE804F0080E141A20262C32383E444A07
:1042100050565C62012240213048FDF795FB5AE080
:10422000012280212D48FDF78FFB54E0012211026D
:104230002A48FDF789FB4EE0012251022748FDF78D
:1042400083FB48E0012211462548FDF77DFB42E053
:10425000012202212248FDF777FB3CE001220421E4
:104260001F48FDF771FB36E0012208211C48FDF7CD
:104270006BFB30E0012210211948FDF765FB2AE0B5
:10428000012240211748FDF75FFB24E00122910243
:104290001548FDF759FB1EE00122D1021248FDF737
:1042A00053FB18E0012211030F48FDF74DFB12E00C
:1042B000012251030C48FDF747FB0CE0012291035A
:1042C0000948FDF741FB06E00122D1030648FDF74E
:1042D0003BFB00E000BF00BF10BD00000004024037
:1042E00000100240000C02400018024010B50446C5
:1042F000102C72D2DFE804F0080E141B22282E3492
:104300003A40464D545B6269002240213448FDF733
:104310001BFB63E0002280213148FDF715FB5DE0C7
:1043200000224FF480712E48FDF70EFB56E000226C
:104330004FF400712A48FDF707FB4FE000220121EE
:104340002848FDF701FB49E0002202212548FDF73E
:10435000FBFA43E0002204212248FDF7F5FA3DE094
:10436000002208211F48FDF7EFFA37E00022102154
:104370001C48FDF7E9FA31E0002240211A48FDF718
:10438000E3FA2BE000224FF480611848FDF7DCFAD5
:1043900024E000224FF400611448FDF7D5FA1DE037
:1043A00000224FF480511148FDF7CEFA16E00022AA
:1043B0004FF400510D48FDF7C7FA0FE000224FF40B
:1043C00080410A48FDF7C0FA08E000224FF400419E
:1043D0000648FDF7B9FA01E0FFE700BF00BF10BDD6
:1043E0000004024000100240000C0240001802408D
:1043F00010B500240DE0E0B24FF6FF72062100F088
:104400003DF8E0B240F20E72052100F037F8601C72
:10441000C4B2102CEFDB10BD30B52DED028B81B096
:104420000546B0EE408A9FED130A28EE000AF3EE2F
:10443000080A80EE201ABCEEC10A10EE104A0020D5
:10444000009004208DF80000200A8DF80100E0B2F1
:104450008DF802002846FFF749FF03226946064807
:1044600006F0A4F82846FFF7C7FE01B0BDEC028BAA
:1044700030BD000000FF7F479C040020F8B50646D1
:104480000D461446002000908DF8005020128DF843
:104490000100E0B28DF802003046FFF727FF03224B
:1044A0006946034806F082F83046FFF7A5FEF8BDDE
:1044B0009C0400202DE9F04104460D4600BF05F0A4
:1044C0000300002808D000BF0BA34FF4B67216A15A
:1044D0001DA0FFF769FB00BF00BF2E4606F0CCF819
:1044E0000746A06800683060A0680660384606F09D
:1044F000CFF8BDE8F08100002E2E2F4D6964646C6A
:104500006577617265732F54686972645F50617278
:1045100074792F4C7749502F7372632F636F7265D4
:104520002F6D656D702E63006D656D705F667265D1
:10453000653A206D656D2070726F7065726C7920C0
:10454000616C69676E656400417373657274696F4D
:104550006E2022257322206661696C656420617477
:10456000206C696E6520256420696E2025730A0021
:1045700070B5054606F080F80646A8680468002C69
:1045800016D02068A968086000BF04F00300002866
:1045900008D000BF09A34FF48C7214A11CA0FFF730
:1045A00003FB00BF00BF304606F072F8204670BD26
:1045B000304606F06DF80020F9E700002E2E2F4D52
:1045C0006964646C6577617265732F54686972649D
:1045D0005F50617274792F4C7749502F7372632F3B
:1045E000636F72652F6D656D702E63006D656D7004
:1045F0005F6D616C6C6F633A206D656D70207072D9
:104600006F7065726C7920616C69676E656400001B
:10461000417373657274696F6E2022257322206660
:1046200061696C6564206174206C696E6520256425
:1046300020696E2025730A0070B50546002411E03C
:1046400004EB4400094901EBC000067D4EB104EBC8
:10465000440001EBC0008068A84202D1204600F06F
:1046600087F9641C0A2CEBDB70BD000070C70020CA
:104670002DE9FF5F0646894617464FF00A0AD346E2
:10468000D04600240A200390002002900190009060
:1046900000BF73E004EB4400764901EBC000057DE8
:1046A000B8F10A0F02D10DB9A04665E0002D63D024
:1046B00000BF012D0AD0022D08DA00BF6EA340F220
:1046C00023127BA18AA0FFF76FFA00BF00BFAEB133
:1046D00004EB4401674A02EBC10130684968884233
:1046E0000CD13FB104EB4400114601EBC0008068DF
:1046F000B84203D1204604B0BDE8F09F012D28D177
:1047000004EB44005B4951F8300080B104EB4400F5
:1047100001EBC000418A029881422DDB039404EB37
:104720004400544901EBC000408A029024E004EBAD
:104730004400504901EBC000418A019881421BDBD3
:10474000A24604EB44004B4901EBC000408A0190B3
:1047500012E0022D10DB04EB4400464901EBC000DF
:10476000418A0098814207DBA34604EB440041499B
:1047700001EBC000408A0090601C04B20A2C89DB67
:1047800009F0020028B9B8F10A0F05D109F00100BB
:1047900010B94FF0FF30AEE7B8F10A0F01DA444626
:1047A00031E0BBF10A0F11DA5C4600BF04EB4400B4
:1047B000304951F8300040B100BF2FA340F26D12D4
:1047C00055A14BA0FFF7F0F900BF0CE0BAF10A0FBA
:1047D00001DA544607E003980A2801DA039C02E054
:1047E0004FF0FF3087E700BF0A2C08DB00BF22A391
:1047F00040F27F124EA13EA0FFF7D6F900BF00BFE6
:10480000204600F0B5F800BF0A2C08DB00BF1AA351
:1048100040F2831246A136A0FFF7C6F900BF00BFE1
:1048200000BF04EB4400134901EBC000007D40B120
:1048300000BF11A34FF4C27242A12DA0FFF7B4F93B
:1048400000BF00BF36B104EB44010A4A02EBC101CC
:1048500030684860002004EB4401064A02EBC101C5
:10486000488204EB4400114601EBC00087602046FB
:1048700041E7000070C700202E2E2F4D6964646C44
:104880006577617265732F54686972645F506172F5
:1048900074792F4C7749502F7372632F636F726551
:1048A0002F697076342F6574686172702E63000012
:1048B0007374617465203D3D204554484152505FFA
:1048C00053544154455F50454E44494E47207C7CEB
:1048D000207374617465203E3D2045544841525018
:1048E0005F53544154455F535441424C45000000CE
:1048F000417373657274696F6E202225732220667E
:1049000061696C6564206174206C696E6520256442
:1049100020696E2025730A006172705F7461626C99
:10492000655B695D2E71203D3D204E554C4C00006D
:1049300069203C204152505F5441424C455F5349ED
:104940005A4500006172705F7461626C655B695DFD
:104950002E7374617465203D3D204554484152508A
:104960005F53544154455F454D5054590000000079
:1049700010B5044604EB44000C4951F8300060B116
:1049800004EB4401094A52F8310004F055FE0020BE
:1049900004EB4401054A42F83100002004EB4401D5
:1049A000024A02EBC101087510BD000070C700206B
:1049B000F0B587B007460D4600BF002D0AD100BFF5
:1049C0002EA340F28A223BA13EA0FFF7EDF800BFE4
:1049D00007B0F0BD00BF7C682088B0F5807F08D1AB
:1049E0002079062805D16079042802D1608808283A
:1049F00003D0384604F020FEEAE7D4F80E00069013
:104A0000A0690590686808B9002607E005986968FC
:104A1000884201D1012000E0002006460EB10120AD
:104A200000E00220034604F1080206A9284600F02F
:104A3000CBFCE088B0F5807F03D0B0F5007F15D1C6
:104A400013E086B1022206AB04F10800291DCDE96E
:104A50000232CDE9001005F1260302462231284634
:104A600000F05CFB00E000BF01E000E000BF00BF21
:104A7000384604F0E1FD00BFAAE700002E2E2F4DBE
:104A80006964646C6577617265732F5468697264D8
:104A90005F50617274792F4C7749502F7372632F76
:104AA000636F72652F697076342F657468617270F8
:104AB0002E6300006E6574696620213D204E554CC2
:104AC0004C000000417373657274696F6E2022257B
:104AD0007322206661696C6564206174206C696E64
:104AE0006520256420696E2025730A002DE9FE43A8
:104AF00004460F461546A94600BF002C08D100BF4A
:104B00005DA340F21E326AA16DA0FFF74DF800BF11
:104B100000BF00BF47B900BF57A340F21F3272A1C8
:104B200067A0FFF741F800BF00BF00BF002D08D10C
:104B300000BF51A34FF448726EA161A0FFF734F893
:104B400000BF00BF2146286801F0B9F910B1DFF8B5
:104B5000B48186E0287800F0F000E02816D101202A
:104B60008DF8040000208DF805005E208DF8060009
:104B7000687800F07F008DF80700A8788DF80800AD
:104B8000E8788DF809000DF1040869E02868A1684B
:104B90000840D4E90112114088420ED0288880B222
:104BA0004FF6A961884208D0E06810B104F10C0901
:104BB00003E06FF00300BDE8FE835348007800EB8C
:104BC0004000524901EBC000007D02281BDB4E482B
:104BD000007800EB400001EBC0008068A04212D1D9
:104BE0004949097801EB4101484A02EBC101D9F872
:104BF00000004968884206D1434802783946204679
:104C000000F086F8D7E7002622E006EB46003F4991
:104C100001EBC000007D022818DB06EB460001EB2B
:104C2000C0008068A04211D106EB4601374A02EB72
:104C3000C101D9F800004968884207D1324806709E
:104C400032463946204600F063F8B4E7701CC6B21D
:104C50000A2EDADB3A464946204600F00DF9AAE76B
:104C600000BF4FF40060434604F12602394600902D
:104C7000204600F025FD9EE72E2E2F4D6964646CC2
:104C80006577617265732F54686972645F506172F1
:104C900074792F4C7749502F7372632F636F72654D
:104CA0002F697076342F6574686172702E6300000E
:104CB0006E6574696620213D204E554C4C00000005
:104CC000417373657274696F6E20222573222066AA
:104CD00061696C6564206174206C696E652025646F
:104CE00020696E2025730A007120213D204E554C0D
:104CF0004C00000069706164647220213D204E55B3
:104D00004C4C0000CC2901088401002070C7002011
:104D1000F8B505460E46144600BF04EB4400314981
:104D200001EBC000007D022808DA00BF2EA340F28C
:104D3000EE223BA146A0FEF737FF00BF00BF04EB09
:104D40004400284901EBC000007D022839D104EB62
:104D5000440001EBC000408AB0F58E7F11DD04EB0A
:104D600044000A4602EBC000011D284600F09CFAF0
:104D700038BB032004EB44011A4A02EBC101087559
:104D80001FE004EB4400174901EBC000408AB0F576
:104D9000877F16DB04EB44000B4603EBC00000F1F9
:104DA0000C0204EB440003EBC000011D284600F098
:104DB00087FA30B9032004EB44010A4A02EBC1012F
:104DC00008754FF40060009004EB4400054901EBC6
:104DD000C00000F10C0305F126023146284600F020
:104DE0006FFCF8BD70C700202E2E2F4D6964646CD7
:104DF0006577617265732F54686972645F50617280
:104E000074792F4C7749502F7372632F636F7265DB
:104E10002F697076342F6574686172702E6300009C
:104E20006172705F7461626C655B6172705F69640E
:104E3000785D2E7374617465203E3D204554484171
:104E400052505F53544154455F535441424C4500C6
:104E5000417373657274696F6E2022257322206618
:104E600061696C6564206174206C696E65202564DD
:104E700020696E2025730A002DE9FE4F81460F46FA
:104E8000164609F1260A4FF0FF30029000200190EB
:104E90004946386801F013F838B9387800F0F00066
:104EA000E02802D00FB1386818B96FF00F00BDE8E4
:104EB000FE8F4A4601213846FFF7DAFB8046B8F1FB
:104EC000000F02DA4FFA88F0F1E700BFB8F17F0F68
:104ED00008D300BF5FA340F2C1326CA16FA0FEF700
:104EE00063FE00BF00BF08F0FF0404EB44007549F7
:104EF00001EBC000007D70B90120019004EB44017A
:104F0000704A02EBC101087504EB4400114601EB45
:104F1000C000C0F8089000BF04EB4400694901EBF1
:104F2000C000007D01280FD004EB440001EBC0005D
:104F3000007D022808DA00BF46A340F2CD3262A10C
:104F400056A0FEF731FE00BF00BF019800B93EB980
:104F50003946484600F0A8F902900EB90298A6E733
:104F600000BF46B900BF3BA340F2E13260A14BA0B5
:104F7000FEF71AFE00BF00BF04EB4400514901EBED
:104F8000C000007D022811DB5C4804704FF4006013
:104F9000009004EB440001EBC00000F10C0352460A
:104FA0003146484600F08CFB029050E004EB440090
:104FB000444901EBC000007D012848D14FF0000BAF
:104FC000354618E000BF6889298988420AD12868D7
:104FD00040B100BF1FA340F2F13249A12FA0FEF75C
:104FE000E3FD00BF00BF287B00F0400010B14FF090
:104FF000010B02E02D68002DE4D100BFBBF1000FD2
:1050000007D032464FF420710E2004F009F905460E
:1050100003E03546284604F01FFDA5B104EB44002B
:10502000284951F8300030B104EB4401254A52F8C8
:10503000310004F001FB04EB4400224941F83050F8
:105040000020029002E04FF0FF30029000BF029873
:105050002DE700002E2E2F4D6964646C6577617218
:1050600065732F54686972645F50617274792F4C54
:105070007749502F7372632F636F72652F69707653
:10508000342F6574686172702E63000074797065E6
:10509000206F766572666C6F7700000041737365F0
:1050A0007274696F6E2022257322206661696C65B7
:1050B00064206174206C696E6520256420696E200F
:1050C00025730A0070C700206172705F7461626CA2
:1050D000655B695D2E7374617465203D3D205045AC
:1050E0004E44494E47206F7220535441424C450074
:1050F0007120213D204E554C4C00000084010020C1
:105100006E6F207061636B65742071756575657372
:1051100020616C6C6F776564210000002DE9FC5FF5
:1051200006460F4690469946DDE90CAB00200190FB
:1051300000BF002E08D100BF31A340F257423EA16C
:1051400041A0FEF731FD00BF00BF4FF420721C21CB
:105150000E2003F0DBFD05461DB94FF0FF30BDE822
:10516000FC9F00BF68891C2808DA00BF24A340F216
:1051700062423FA134A0FEF717FD00BF00BF6C687C
:105180000F9802F062F9E08000BF96F82C00062824
:1051900008D000BF1AA340F2694242492AA0FEF794
:1051A00003FD00BF00BFD9F80000A060B9F80400FB
:1051B000A081DBF80000C4F81200BBF80400E08214
:1051C000DAF80000C4F80E000E980068A0614FF4F1
:1051D000807020800820608006202071042060718B
:1051E00040F6060043463A4629460090304600F015
:1051F00067FA284604F020FA00250198AFE700007E
:105200002E2E2F4D6964646C6577617265732F541F
:10521000686972645F50617274792F4C7749502FBE
:105220007372632F636F72652F697076342F6574A4
:10523000686172702E6300006E6574696620213D9E
:10524000204E554C4C000000417373657274696FB9
:105250006E2022257322206661696C65642061746A
:10526000206C696E6520256420696E2025730A0014
:10527000636865636B207468617420666972737417
:1052800020706275662063616E20686F6C642073A5
:105290007472756374206574686172705F6864729B
:1052A000000000008C2C010870B504460D46034A2E
:1052B0002946204600F004F870BD0000CC29010802
:1052C0007FB504460D4616460121074A201D04F10C
:1052D00026038DE825000391324619462046FFF744
:1052E0001DFF04B070BD0000D229010870B5002474
:1052F00064E004EB4400334901EBC000057D002D60
:105300005BD004EB440001EBC000408A401C04EB7E
:1053100044012C4A02EBC101488204EB44001146CF
:1053200001EBC000408AB0F5967F0DDA04EB440033
:1053300001EBC000007D01280AD104EB440001EB21
:10534000C000408A052803DB2046FFF711FB34E04C
:1053500004EB44001B4901EBC000007D032807D18A
:10536000042004EB4401174A02EBC101087524E054
:1053700004EB4400134901EBC000007D042807D171
:10538000022004EB44010F4A02EBC101087514E04E
:1053900004EB44000B4901EBC000007D01280CD157
:1053A00004EB44020B4603EBC202111D04EB440262
:1053B00003EBC2029068FFF777FF641C0A2C98DBAE
:1053C00070BD000070C700202DE9F84305460E4669
:1053D0001746984600BF95F82C00062808D000BF55
:1053E0002EA340F2A9123BA143A0FEF7DDFB00BFB4
:1053F00000BF5EB1306848B12946306800F05FFDFB
:1054000020B9307800F0F000E02803D16FF00F00F1
:10541000BDE8F8832A4641463046FFF729F904469D
:10542000002C01DA60B2F3E7022004EB44013C4AAD
:1054300002EBC101087504EB4400114601EBC0000A
:10544000856004EB440001EBC0003968C160B98895
:105450000182002004EB440102EBC101488204EB0D
:105460004400114651F83000B0B104EB440051F84B
:105470003090002004EB440142F831004FF400600A
:105480003B4605F1260249460090284600F018F9EF
:10549000484604F0D1F800BF0020B9E72E2E2F4D6A
:1054A0006964646C6577617265732F5468697264AE
:1054B0005F50617274792F4C7749502F7372632F4C
:1054C000636F72652F697076342F657468617270CE
:1054D0002E6300006E657469662D3E6877616464B2
:1054E000725F6C656E203D3D204554485F485741D2
:1054F0004444525F4C454E00417373657274696F4A
:105500006E2022257322206661696C6564206174B7
:10551000206C696E6520256420696E2025730A0061
:1055200070C700202DE9F04104460E464FF00E08EA
:1055300060890E2800DC4FE0E07B18B996F8300057
:10554000401CE0736568AF89287800F00100B0B1B5
:105550002878012809D1687888B9A8785E280ED102
:10556000607B40F01000607309E006221D49284668
:10557000FAF7FEFE18B9607B40F008006073082F50
:1055800003D0B7F5C16F22D110E096F82D0000F0DE
:10559000080000B920E04146204604F0B1FA00B10D
:1055A0001AE03146204600F017FE11E096F82D0073
:1055B00000F0080000B90FE04146204604F0A0FAD0
:1055C00000B109E031462046FFF7F2F900E003E0C0
:1055D00000BF0020BDE8F081204604F02DF8002037
:1055E000F8E70000CC290108704700009AB0064691
:1055F000642101A8FAF7B1FE00240027A046A146C5
:10560000354600BF2C48FDF7EEFB044695F82D000B
:10561000C0F3800058B1012C09DC2848FBF730FFAB
:10562000284602F0B1FF284603F018F83FE095F84D
:105630002D00C0F38000002839D1012C37DD022C69
:1056400006D0032C0AD0042C0ED0052C17D111E063
:105650004FF400694FF48048012711E04FF0000932
:105660004FF4804801270BE04FF400694FF0000829
:10567000012705E04FF00009C846012700E000BF00
:1056800000BFA7B101A90D48FBF7DEFACDF81C90C9
:10569000CDF8188001A90948FBF73AFE0748FBF747
:1056A00083FE284603F0AAF8284603F03DF864205C
:1056B00003F004F9A6E70000305100204850002014
:1056C0002DE9F04705460E4617469846DDF820902E
:1056D000484601F0BAFE82460E21304603F098FAA1
:1056E00000B122E07468A4F80CA0D8F80000206093
:1056F000B8F80400A0803868C4F80600B888608153
:1057000000BF95F82C00062808D000BF08A34FF46E
:10571000997215A121A0FEF747FA00BF00BF3146DC
:105720002846AA699047BDE8F0876FF00100FAE7C4
:105730002E2E2F4D6964646C6577617265732F54EA
:10574000686972645F50617274792F4C7749502F89
:105750007372632F6E657469662F65746865726E07
:1057600065742E63000000006E657469662D3E68E6
:1057700077616464725F6C656E206D75737420620E
:1057800065203620666F722065746865726E657478
:105790005F6F75747075742100000000417373654C
:1057A0007274696F6E2022257322206661696C65B0
:1057B00064206174206C696E6520256420696E2008
:1057C00025730A0010B5044600BF44B900BF0CA3FE
:1057D00040F2DF1211A115A0FEF7E6F900BF00BFED
:1057E000732084F82E0074212F2001551948606120
:1057F0001948A061204601F09BFC002010BD00006C
:105800002E2E2F4C5749502F5461726765742F65A7
:10581000746865726E657469662E63006E6574697E
:105820006620213D204E554C4C00000041737365AD
:105830007274696F6E2022257322206661696C651F
:1058400064206174206C696E6520256420696E2077
:1058500025730A00ED4A000821730008064600245B
:10586000354600BF4FF0FF310B48006803F066F982
:105870000028F7D100BF284601F040FD04463CB1A6
:10588000294620462A69904710B1204603F0D4FEED
:10589000002CF0D1E6E700002C00002038B50446CB
:1058A0008DF8000069460320ABBE204638BD0000DD
:1058B00010B50024002210210A48FCF745F80A2000
:1058C000FBF79AF9012210210648FCF73DF800BFCA
:1058D00004E0204600F008F8601CC4B2102CF8DB8D
:1058E00010BD00000000024010B50446102C69D223
:1058F000DFE804F0080E141A20262C32383E444A01
:1059000050565C62012210213048FCF71DF85AE025
:10591000012204212D48FCF717F854E0012211035D
:105920002B48FCF711F84EE0012291022848FCF7C1
:105930000BF848E0012211022548FCF705F842E087
:10594000012251032348FBF7FFFF3CE00122D10273
:105950002048FBF7F9FF36E0012211461B48FBF710
:10596000F3FF30E0012211461B48FBF7EDFF2AE070
:10597000012211021948FBF7E7FF24E00122402130
:105980001648FBF7E1FF1EE00122D1031448FBF7A4
:10599000DBFF18E00122D1021248FBF7D5FF12E02D
:1059A0000122D1020E48FBF7CFFF0CE00122510289
:1059B0000B48FBF7C9FF06E0012240210348FBF733
:1059C000C3FF00E000BF00BF10BD00000018024090
:1059D000000C02400010024000040240001402408B
:1059E000000002400008024010B50446102C74D29A
:1059F000DFE804F0080E141B222930373D434A50DB
:105A0000575E656C002210213548FBF79DFF65E06D
:105A1000002204213248FBF797FF5FE000224FF499
:105A200080513048FBF790FF58E000224FF480612E
:105A30002C48FBF789FF51E000224FF48071294880
:105A4000FBF782FF4AE000224FF400512648FBF7A3
:105A50007BFF43E000224FF400612348FBF774FF13
:105A60003CE0002201211E48FBF76EFF36E00022D9
:105A700001211E48FBF768FF30E000224FF48071DF
:105A80001B48FBF761FF29E0002240211848FBF783
:105A90005BFF23E000224FF400411648FBF754FF60
:105AA0001CE000224FF400611348FBF74DFF15E0A6
:105AB00000224FF400610F48FBF746FF0EE0002282
:105AC0004FF400710B48FBF73FFF07E00022402135
:105AD0000348FBF739FF01E0FFE700BF00BF10BD3F
:105AE00000180240000C0240001002400004024076
:105AF00000140240000002400008024070B5054654
:105B00000C4622460321284600F03AF970BD0000F9
:105B10002DE9FF5F05468A46654880680390039833
:105B200000780007860E142E00DAB7E06889042892
:105B300000D2B3E06868047814B1082C70D100E09A
:105B4000A6E0DFF86C9109F114095948007D00F0D6
:105B5000F000E02800D1A5E0554A1168506900F036
:105B6000AEF900B19EE02889082800D296E006F13F
:105B70000E01284603F04CF8002840D02889304414
:105B80001FFA80FB2889584500DD8BE04FF4207216
:105B900059460E2003F0BAF8074607B982E0798922
:105BA00006F10800814203D2384603F045FD79E052
:105BB000324678680399FAF7A9FB3146384603F074
:105BC0009FFF00280DD000BF00BF3AA3B62247A117
:105BD00054A0FDF7E9FF00BF00BF384603F02CFDDD
:105BE00060E02946384603F073FB18B1384603F0ED
:105BF00023FD57E0284603F01FFD3D4611E006F166
:105C00000E01284603F07CFF58B100BF00BF29A356
:105C1000C7224EA143A0FDF7C7FF00BF00BF41E070
:105C200024E0D5F804803146284602F0F1FFE0B9BF
:105C30006F68D9F80000F8601D48006938610020DD
:105C400088F80000A8F80200FF2038720020788150
:105C500001200021FF230A46CDE9010A00914946AF
:105C6000284600F0A1FB834600BF11E0032C0ED0B4
:105C70000B2C0CD00C2C0AD0042C08D0052C06D0F0
:105C80000D2C04D00E2C02D0112C00D000BF00BF70
:105C900000BF284603F0D0FCBDE8FF9F284603F074
:105CA000CBFCF9E7284603F0C7FC00BFF4E700008F
:105CB000689000202E2E2F4D6964646C65776172A8
:105CC00065732F54686972645F50617274792F4CE8
:105CD0007749502F7372632F636F72652F697076E7
:105CE000342F69636D702E630000000069636D706E
:105CF0005F696E7075743A206D6F76696E67207299
:105D00002D3E7061796C6F616420746F2069636DE2
:105D10007020686561646572206661696C65640AFB
:105D200000000000417373657274696F6E20222554
:105D30007322206661696C6564206174206C696EF1
:105D40006520256420696E2025730A0069636D70E3
:105D50005F696E7075743A20726573746F72696EE4
:105D600067206F726967696E616C20702D3E70618B
:105D7000796C6F6164206661696C65640A0000007B
:105D80002DE9FF470746884691464FF420722421AB
:105D9000222002F0BBFF05460DB9BDE8FF8700BF1A
:105DA0006889242808D200BF19A34FF4B47226A131
:105DB00030A0FDF7F9FE00BF00BFD7F804A06C6863
:105DC00084F8008084F801900020A080E080796849
:105DD0006A6802F108001C22FAF798FADAF80C0057
:105DE000039003A800F048FD06465EB100206080E5
:105DF00001200021FF2303AACDE9010600912846D6
:105E000000F0D2FA284603F017FC00BFC5E70000F7
:105E10002E2E2F4D6964646C6577617265732F5403
:105E2000686972645F50617274792F4C7749502FA2
:105E30007372632F636F72652F697076342F696395
:105E40006D702E6300000000636865636B207468EA
:105E50006174206669727374207062756620636174
:105E60006E20686F6C642069636D70206D6573735C
:105E700061676500417373657274696F6E202225D6
:105E80007322206661696C6564206174206C696EA0
:105E90006520256420696E2025730A0070B50546CB
:105EA0000C4622460B212846FFF76AFF70BD00BF53
:105EB000EFF3058008B1012070470020FCE718B51A
:105EC00002460092D04300B10AB9012018BD91F8F2
:105ED0002D0000F0020008B90020F7E74868904262
:105EE00001D10020F2E700988B681840D1E9013415
:105EF0002340984208D1886822EA00008C68E34376
:105F0000984201D10120E1E70020DFE72DE9F74FBA
:105F10008CB004460F464FF00008B98CA1F1140074
:105F2000C11700EB5171C1F3CF0A142005906068CE
:105F30000990DDF8249099F8000000F00F0014217A
:105F4000B1EB800F04D06FF005000FB0BDE8F08F0B
:105F500000BF608914280BDA00BF72A34FF43F72B0
:105F60007FA186A0FDF720FE00BF6FF00500ECE7E3
:105F700000BFB9F8060001F068FA04900498C0F375
:105F80000C000790049800F4005003902089143806
:105F90001FFA80FBBDE04FF6FF7000EACA005845CB
:105FA00001DD584603E04FF6FF7000EACA00089092
:105FB0004FF4207214210E2002F0A8FE054605B908
:105FC000ADE000BF6889142808DA00BF55A34FF47C
:105FD000497274A169A0FDF7E7FD00BF00BF14225C
:105FE00068680999FAF792F9D5F8049008980A9028
:105FF00054E061890598081A80B2029000BF618957
:106000000598814208DA00BF46A340F22D326DA107
:106010005AA0FDF7C9FD00BF00BF02990A98884247
:1060200001DA0A9800E002988046B8F1000F03D127
:1060300000200590246831E000F068FC06461EB997
:10604000284603F0F9FA6AE0616805980844334687
:1060500041224146CDE90008002003F005F80B90ED
:106060000B9830B9304600F057FC284603F0E4FAAC
:1060700055E0204603F0F0FC746156483061284634
:106080000B9903F01BF80A98A0EB080080B20A9065
:106090000A9810B100200590246800BF0A980028D3
:1060A000A7D10598404480B20590B88C1438584563
:1060B00001DB012000E0002006900798C0F30C00EF
:1060C0000490069808B1039818B1049840F4005061
:1060D0000490049801F0B9F9A9F806000899143160
:1060E00088B201F0B2F9A9F802000020A9F80A006C
:1060F0007B69294638460E9A9847284603F09CFA51
:106100000898ABEB00001FFA80FB0798504480B260
:106110000790BBF1000F7FF43EAF002015E74FF072
:10612000FF3012E72E2E2F4D6964646C6577617223
:1061300065732F54686972645F50617274792F4C73
:106140007749502F7372632F636F72652F69707672
:10615000342F6970345F667261672E63000000003F
:106160006970345F6672616728293A2070627566CB
:1061700020746F6F2073686F7274000041737365D1
:106180007274696F6E2022257322206661696C65C6
:1061900064206174206C696E6520256420696E201E
:1061A00025730A0074686973206E656564732061E5
:1061B000207062756620696E206F6E65207069655B
:1061C00063652100702D3E6C656E203E3D20706F32
:1061D00066660000697000082DE9F04707460E4624
:1061E0007D6828780421B1EB201F05D0384603F0E4
:1061F00023FA0020BDE8F087287800074FEA90686E
:10620000688801F022F981463989494503DD49460C
:10621000384603F06DFB7889404505DB38894845F1
:1062200002DBB8F1140F04DA384603F005FA002057
:10623000E0E728694D494861E86808610846007D43
:1062400000F0F000E0280AD196F82D0000F00100DF
:1062500018B1706808B134461CE000241AE03046DA
:1062600000F088F808B1344614E000243F48007D6F
:106270007F280FD03E48046809E0B44200D105E011
:10628000204600F077F800B103E000BF2468002C3E
:10629000F3D100BF354908693146FFF710FE28B930
:1062A0003248007C00F0F000E02804D1384603F0CA
:1062B000C3F900209EE724B9384603F0BDF9002059
:1062C00098E7E8884FF63F71084038B1384600F04B
:1062D00055F907460FB900208CE77D682348046014
:1062E0004660856028780007800E204988814146F5
:1062F000384603F005FC687A01280DD0062806D040
:1063000011280ED1314638460AF05CFD22E03146B4
:10631000384605F0ABFB1DE031463846FFF7F8FB89
:1063200018E0124948692146FFF7C9FD70B90F48C6
:10633000007D00F0F000E02808D00FFA88F1384620
:1063400003F08BFA02213846FFF7D8FB384603F0FA
:1063500073F900BF00BF00200449086048608860EE
:1063600088810861486100BF44E700006890002010
:106370001C01002010B5044694F82D0000F0010027
:1063800070B1606860B1074840696168884205D0B3
:10639000044948692146FFF792FD08B1012010BD6C
:1063A0000020FCE7689000202DE9FE4F07460C46D0
:1063B00015469846DDE90C9A0E9EA34625B10CB110
:1063C000206808B906F1040B43462A465946384668
:1063D000CDE9009A029600F003F8BDE8FE8F0000B8
:1063E0002DE9F84F05460F4690469A46DDF828B04D
:1063F0000C9E00BFA87B012808D000BF37A34FF434
:10640000557243A145A0FDF7CFFB00BF00BFB8F117
:10641000000F46D04FF014091421284602F0F8FB73
:1064200018B16FF00100BDE8F88F6C6800BF688993
:10643000142808D200BF29A34FF4627241A137A0EB
:10644000FDF7B2FB00BF00BF84F808A00B98607294
:10645000D8F80000206148464FEAE97109EB9171D4
:10646000C1F3870141F04001217084F801B028890F
:1064700000F0EBFF60800020E0803E48008800F0E4
:10648000E4FFA0803B480088401C3A4908801FB9BF
:1064900039480068E06001E03868E0600020608111
:1064A00009E06889142802DA6FF00100BBE76C6824
:1064B00020690090E846B08C48B12889B18C8842A8
:1064C00005DD424631462846FFF720FDABE7424650
:1064D0002946304673699847A5E700002E2E2F4DB8
:1064E0006964646C6577617265732F54686972645E
:1064F0005F50617274792F4C7749502F7372632FFC
:10650000636F72652F697076342F6970342E630063
:10651000702D3E726566203D3D20310041737365EC
:106520007274696F6E2022257322206661696C6522
:1065300064206174206C696E6520256420696E207A
:1065400025730A00636865636B2074686174206654
:106550006972737420706275662063616E20686F63
:106560006C64207374727563742069705F68647200
:106570000000000086010020142B01082DE9F14FD6
:1065800084B004984568287800F00F001421B1EB1E
:10659000800F00D011E1E88800F057FFC0F30C0035
:1065A0004FF6FF7101EAC00A688800F04EFF074607
:1065B00028780007810E02910299B94200DDFCE0C3
:1065C0000298381A87B2049802F020FE06467D48E9
:1065D000018888190A280ADD3146284600F0E6FCC1
:1065E00020B17848008830440A2800DDE5E076488C
:1065F000046811E06069E968884209D1A0692969E5
:10660000884205D1A089A988884201D1012000E0F3
:10661000002000B102E02468002CEBD100BF34B9A7
:106620003146284600F0A8FB044694B9C5E0E88846
:1066300000F00BFFC0F30C0058B9E08900F005FF33
:10664000C0F30C0028B11422294604F10800F9F720
:106650005DFEE888012121EA50100190019850B1B7
:106660000AEB070188B2504503DB4FF6EB71884215
:1066700000DD80E000BF2046019A049900F098F9FF
:1066800083460BF1010000B975E04E4800883044A4
:106690004C490880019840B10AEB070188B2A083F9
:1066A000A17F41F00101A17700BFBBF1010F60D1D3
:1066B000A08B143080B2009060684068D0F80090E1
:1066C00060684568142204F108012846F9F71EFEA7
:1066D000009800F0BAFE68800020E8806881606859
:1066E00004900DE0D9F8040003901421484603F00B
:1066F00007FA4946049802F0E1FC0398D0F80090AC
:10670000B9F1000FEED130480068844202D14FF059
:1067100000080EE02C48D0F8008006E0D8F8000011
:10672000A04200D104E0D8F80080B8F1000FF5D104
:1067300000BF4146204600F0BDFA049802F066FD15
:10674000064600BF1F480088B04208DA00BF1FA3FA
:1067500040F29B222CA133A0FDF726FA00BF00BF18
:1067600018480088801B17490880049805B0BDE8C8
:10677000F08F0020FAE700BF44B900BF13A34FF425
:106780002A7232A127A0FDF70FFA00BF00BF606890
:1067900090B900BF0C480068844208D000BF0BA32A
:1067A00040F2AB222CA11FA0FDF7FEF900BF00BFF5
:1067B0000021204600F07EFA00BF049802F03CFF62
:1067C0000020D3E78C010020880100202E2E2F4DC1
:1067D0006964646C6577617265732F54686972646B
:1067E0005F50617274792F4C7749502F7372632F09
:1067F000636F72652F697076342F6970345F6672CB
:1068000061672E630000000069705F7265617373D9
:106810005F70627566636F756E74203E3D20636CB9
:10682000656E0000417373657274696F6E20222576
:106830007322206661696C6564206174206C696EE6
:106840006520256420696E2025730A006970722016
:10685000213D204E554C4C006E6F7420666972735A
:1068600074616C74686F756768206A7573742065ED
:106870006E7175657565640010B502462148016842
:1068800021E091F82D0000F00100D8B191F82D0021
:10689000C0F38000B0B14868A0B110688B681840A0
:1068A000D1E901342340984201D1084610BD91F846
:1068B0002D0000F0020028B91068CB68984201D181
:1068C0000846F3E709680029DBD10F480068A0B14A
:1068D0000D48006890F82D0000F0010068B10A48EA
:1068E000006890F82D00C0F3800030B106480068C1
:1068F000406810B110787F2801D10020D6E7024807
:106900000068D3E71C0100202001002010B50520FD
:1069100001F01EFB10BD000010B5044600BF002CA6
:1069200008D100BF06A34FF4317214A116A0FDF7E1
:106930003BF900BF00BF2146052001F03BFA10BD26
:106940002E2E2F4D6964646C6577617265732F54C8
:10695000686972645F50617274792F4C7749502F67
:106960007372632F636F72652F697076342F69704D
:10697000345F667261672E63000000007020213D65
:10698000204E554C4C000000417373657274696F62
:106990006E2022257322206661696C656420617413
:1069A000206C696E6520256420696E2025730A00BD
:1069B0002DE9F74F84B00646884600250120019056
:1069C000D8F8040002900299488800F03EFD834602
:1069D000029800780007800E03900398584503DD65
:1069E000681E07B0BDE8F08F0398ABEB00001FFAFC
:1069F00080FB0299C88800F028FDC0F30C004FF618
:106A0000FF7101EAC00A00BF00BFD8F804400020AF
:106A10002060A4F804A00AEB0B00E080E088504559
:106A200002DA4FF0FF30DCE7D6F804903EE0D9F808
:106A30000470A088B988884220DAC4F800909DB11B
:106A4000A088E988884203DBE088B988884202DDB3
:106A50004FF0FF30C5E7C5F80080E888A18888427C
:106A60000BD00020019008E0E088B988884202DD60
:106A70004FF0FF30B5E7C6F804801AE0A088B98867
:106A8000884202D14FF0FF30ABE7A088F9888842F6
:106A900002DA4FF0FF30A4E72DB1E888B9888842C8
:106AA00001D000200190D7F800903D46B9F1000FC9
:106AB000BDD100BFB9F1000F28D1002D17D000BF04
:106AC000E888A188884208DD00BF3EA34FF4DB724E
:106AD0004BA153A0FDF768F800BF00BFC5F80080C8
:106AE000E888A188884211D0002001900EE000BF04
:106AF000706840B100BF33A34FF4DF7252A148A0C9
:106B0000FDF752F800BF00BFC6F80480069820B910
:106B1000B07F00F00100002851D00198002848D033
:106B2000706818B170684068808810B100200190CA
:106B30003FE02546D4F800900BE0D9F80440E888FF
:106B4000A188884202D00020019005E02546D4F8B3
:106B50000090B9F1000FF0D100BF0198002828D0B3
:106B600000BF706840B900BF16A340F2DF1244A115
:106B70002BA0FDF719F800BF00BF00BF7068406888
:106B8000A04208D100BF0FA34FF4F0723CA124A093
:106B9000FDF70AF800BF00BF00BF206840B100BF8A
:106BA00008A34FF4F1723AA11DA0FCF7FDFF00BF4E
:106BB00000BF019808B1012013E7002011E7002071
:106BC0000FE700002E2E2F4D6964646C65776172AB
:106BD00065732F54686972645F50617274792F4CC9
:106BE0007749502F7372632F636F72652F697076C8
:106BF000342F6970345F667261672E630000000095
:106C0000636865636B20667261676D656E7473207F
:106C1000646F6E2774206F7665726C61700000007F
:106C2000417373657274696F6E202225732220662A
:106C300061696C6564206174206C696E65202564EF
:106C400020696E2025730A006E6F20707265766968
:106C50006F757320667261676D656E742C20746841
:106C60006973206D75737420626520746865206691
:106C70006972737420667261676D656E74210000BD
:106C800073616E69747920636865636B000000004E
:106C900076616C69646174655F6461746167726177
:106CA0006D3A6E6578745F70627566213D4E554C25
:106CB0004C00000070B504460D460E480068A04226
:106CC00003D10C49206808600EE000BF002D08D1F8
:106CD00000BF09A340F2451216A11DA0FCF764FFF6
:106CE00000BF00BF206828602146042001F062F840
:106CF00070BD0000880100202E2E2F4D6964646C49
:106D00006577617265732F54686972645F50617250
:106D100074792F4C7749502F7372632F636F7265AC
:106D20002F697076342F6970345F667261672E63E5
:106D30000000000073616E69747920636865636B9D
:106D4000206C696E6B6564206C69737400000000D0
:106D5000417373657274696F6E20222573222066F9
:106D600061696C6564206174206C696E65202564BE
:106D700020696E2025730A0070B505460E46042072
:106D800001F0E6F8044664B93146284600F00EF9F1
:106D9000B04203DB042001F0DBF804460CB900200C
:106DA00070BD20212046F9F7D8FA0F20E077064879
:106DB00000682060044804601422294604F1080099
:106DC000F9F7A4FA2046EBE7880100202DE9F04707
:106DD00004468846002500BFA04507D100BF40A358
:106DE000AB224EA150A0FCF7DFFE00BF00BFB8F100
:106DF000000F0DD000BFD8F80000A04207D000BFA0
:106E000037A3AD2252A148A0FCF7CEFE00BF00BFC1
:106E10006068D0F80490B9F80400002824D16768AD
:106E2000D9F800006060142204F108017868F9F7CD
:106E30006DFA01213846FFF731F8384602F0E6F9DD
:106E4000064600BFA819B0F5803F07DB00BF24A3AA
:106E5000BC2244A134A0FCF7A7FE00BF00BFA819C4
:106E600085B2384602F0E8FB67681CE0D7F804906A
:106E7000BA46D9F80070504602F0C8F9064600BF7D
:106E8000A819B0F5803F07DB00BF15A3CC2235A1C0
:106E900025A0FCF789FE00BF00BFA81985B25046A7
:106EA00002F0CAFB00BF002FE0D141462046FFF7A9
:106EB00001FF00BF33480088A84207DA00BF08A3DB
:106EC000D22231A118A0FCF76FFE00BF00BF2D48F1
:106ED0000088401B2B4908802846BDE8F087000049
:106EE0002E2E2F4D6964646C6577617265732F5423
:106EF000686972645F50617274792F4C7749502FC2
:106F00007372632F636F72652F697076342F6970A7
:106F1000345F667261672E630000000070726576F0
:106F200020213D2069707200417373657274696F2E
:106F30006E2022257322206661696C65642061746D
:106F4000206C696E6520256420696E2025730A0017
:106F5000707265762D3E6E657874203D3D206970B7
:106F60007200000070627566735F6672656564200A
:106F70002B20636C656E203C3D203078666666662B
:106F8000000000008C01002069705F7265617373FE
:106F90005F70627566636F756E74203E3D2070622F
:106FA0007566735F66726565640000002DE9F84FD1
:106FB00005468946002700BF0026B2460020009003
:106FC00083461B48046821E06069E968884207D16C
:106FD000A0692969884203D1A089A988884201D083
:106FE000012000E0002068B10BF1010B1EB926461C
:106FF000CDF800A006E0E07FF17F884202DC264663
:10700000CDF800A0206800B1A2462468002CDBD196
:107010002EB130460099FFF7D9FE804647444F45D0
:1070200002DABBF1010FC7DC3846BDE8F88F00007B
:107030008801002070B500250A4804680FE0E07F51
:10704000002805DDE07F401EE0772546246806E045
:107050002646246829463046FFF7B8FE00BF002CBC
:10706000EDD170BD8801002070B505462C4600BFEB
:10707000002C08D100BF0FA340F2CE221CA11FA0FC
:10708000FCF792FD00BF00BF00BFAC4208D000BFBC
:1070900008A340F2CF2223A118A0FCF785FD00BF72
:1070A00000BF606910B1606902F0C6FA2046FFF7C0
:1070B00033FC70BD2E2E2F4D6964646C6577617250
:1070C00065732F54686972645F50617274792F4CD4
:1070D0007749502F7372632F636F72652F697076D3
:1070E000342F6970345F667261672E6300000000A0
:1070F00070637220213D204E554C4C0041737365E6
:107100007274696F6E2022257322206661696C6536
:1071100064206174206C696E6520256420696E208E
:1071200025730A00706372203D3D2070000000004E
:107130002DE9F041A2B004460027B846002664219C
:1071400009A8F9F70AF962486249086000208DF839
:107150001C0080208DF81D00E1208DF81E0000200D
:107160008DF81F008DF8200088208DF8210007A8D9
:1071700048604FF40001574881605749C160574942
:1071800001614FF4C0614161F9F770FE0746382193
:107190005348F9F7E2F82120514908604FF44000C4
:1071A0004861002008614F4800F0BCFE062084F8CA
:1071B0002C0048484068007884F82600454840681C
:1071C000417827200155434840688178282001559F
:1071D00040484068C178292001553E4840680179FF
:1071E0002A2001553B48406841792B20015540F247
:1071F000DC50A08494F82D0040F00A0084F82D00A3
:107200000322002101200AF0BFFB37490860032256
:10721000002101200AF0B8FB344908601C223449DF
:107220006846F9F773F82146684601F0BBFC31491E
:107230003148FBF7BCFE3048FBF74AFE002F41D136
:107240002D48FBF7D0FD0646012E06DC204601F056
:1072500005FA204601F098F936E0022E06D0032EFA
:1072600009D0042E0BD0052E11D10DE04FF400658E
:107270004FF4804810E000254FF480480CE04FF4B4
:1072800000654FF0000807E00025A84604E04FF431
:1072900000654FF4804800BF00BF09A90D48F9F709
:1072A000D3FC0F95CDF8388009A90A48FAF730F8D1
:1072B0000848FAF779F8204601F0A0FA204601F0D4
:1072C00033FA01E0F9F715FC22B0BDE8F0810000C7
:1072D0000080024048500020A84F0020084F0020A6
:1072E000F8500020882901082C00002030000020E0
:1072F00094290108340000203051002038B504469C
:10730000002000900448007818B969460348F9F74E
:10731000C2FE009838BD0000280000204850002020
:107320002DE9F0418CB080460D4600240026002750
:1073300030216846F9F711F830216846F9F70DF861
:107340002E4629E0042C04D36FF00B000CB0BDE8EE
:10735000F08104EB440170684DF82100708904EB62
:1073600044016A4602EB8101486054B104EB4400D9
:10737000694601EB8001601E00EB400002EB8000DB
:107380008160306830B9002004EB44016A4602EBAA
:1073900081018860641C3668002ED3D128890D498C
:1073A0004860C1F808D008464563284602F054FBFF
:1073B00008490948FAF7C2F800BF4FF0FF31074803
:1073C000006801F0BBFB0028F7D10348F9F719FF6B
:1073D0003846BBE7F850002048500020300000201D
:1073E0002DE9F041044625466868804703F0DCF942
:1073F00006460D49286809684718B81BB0F1004FC8
:1074000001D3012000E0002030B12968881922460C
:10741000064903F051FA04E022460449384603F0D5
:107420004BFABDE8F081000074010020E173000810
:107430000146080601F47F4240EA022001F47F027F
:1074400040EA122040EA1160704701460806000C2D
:1074500040EA11207047000008B50020009000BFEE
:107460006846804208D000BF0CA340F25112174971
:1074700017A0FCF799FB00BF00BF00BF00BF03F0DF
:107480003BF900F063F900F03DFD00F0D5FF09F095
:107490008DFC04F0DFFA03F0AFFA08BD2E2E2F4D5D
:1074A0006964646C6577617265732F54686972648E
:1074B0005F50617274792F4C7749502F7372632F2C
:1074C000636F72652F696E69742E6300782B0108F3
:1074D000417373657274696F6E2022257322206672
:1074E00061696C6564206174206C696E6520256437
:1074F00020696E2025730A00FAF73EFAFCF78EF930
:10750000FBF70AFEFCF78EF8FCF76AF8FBF796FD2E
:10751000FEF7CEF90C210448FBF7D0FBFBF75EFD2C
:1075200001F0D8F900BFFEE7F40400200146002076
:10753000842901D0CA1C10447047000070B505466C
:1075400005B970BD05F00300002813D000BF00BFCF
:107550003DA340F2732248A150A0FCF725FB00BFD9
:1075600000BF00BF03F088F80646304603F090F8ED
:1075700000BFE6E7A5F1080452480068844205D33D
:1075800005F10C0050490968884213D900BF00BFBB
:107590002DA340F27F224DA140A0FCF705FB00BFC8
:1075A00000BF00BF03F068F80646304603F070F8ED
:1075B00000BFC6E74C4803F0D9F82079002816D15F
:1075C00000BF00BF20A34FF4237248A133A0FCF7F3
:1075D000EBFA00BF00BF444803F0E0F800BF03F03F
:1075E0004BF80646304603F053F800BFA9E72046A3
:1075F00000F026F9002816D100BF00BF12A340F208
:10760000952244A125A0FCF7CFFA00BF00BF364861
:1076100003F0C4F800BF03F02FF80646304603F02D
:1076200037F800BF8DE7002020714748006884428A
:1076300001D245480460204602F0DCFA2A4803F0F3
:10764000ADF800BF7DE700002E2E2F4D6964646CFD
:107650006577617265732F54686972645F506172F7
:1076600074792F4C7749502F7372632F636F726553
:107670002F6D656D2E6300006D656D5F66726565CB
:107680003A2073616E69747920636865636B206169
:107690006C69676E6D656E74000000004173736500
:1076A0007274696F6E2022257322206661696C6591
:1076B00064206174206C696E6520256420696E20E9
:1076C00025730A00D8000020DC0000206D656D5F86
:1076D000667265653A20696C6C6567616C206D65E2
:1076E0006D6F727900000000E00000206D656D5F35
:1076F000667265653A20696C6C6567616C206D65C2
:107700006D6F72793A20646F75626C652066726580
:10771000650000006D656D5F667265653A20696C95
:107720006C6567616C206D656D6F72793A206E6F64
:107730006E2D6C696E6B65643A20646F75626C6562
:107740002066726565000000E400002010B500BFEF
:1077500000BF194820F00300184908600846046873
:107760004FF4C86020800020608020714FF4C86012
:1077700002F048FE124908600120096808714FF4C0
:10778000C8600F49096808800D49096848800B489E
:1077900000680C4908600C4802F0F0FF00280AD08D
:1077A00000BF00BF09A340F21F2214A11AA0FCF7DA
:1077B000FBF900BF00BF10BD83900020D80000205F
:1077C000DC000020E4000020E00000202E2E2F4DE1
:1077D0006964646C6577617265732F54686972645B
:1077E0005F50617274792F4C7749502F7372632FF9
:1077F000636F72652F6D656D2E6300006661696C45
:10780000656420746F20637265617465206D656DB9
:107810005F6D757465780000417373657274696F8C
:107820006E2022257322206661696C656420617474
:10783000206C696E6520256420696E2025730A001E
:107840002DE9F0410446204600F084F905462088E1
:1078500002F0D8FD0646608802F0D4FD0746208875
:10786000B0F5C86F10D86088B0F5C86F0CD86088C4
:10787000A84202D03888A84206D10648006886424D
:1078800005D07088A84202D00020BDE8F081012018
:10789000FBE70000DC0000202DE9F0478146B9F14C
:1078A000000F02D10020BDE8F08709F1030020F0AD
:1078B000030085B20C2D00D20C25B5F5C86F01D898
:1078C0004D4501DA0020EEE75C4802F04FFF5C48CE
:1078D000006800F03FF90646A6E0304602F092FD4F
:1078E0000446207900287CD1218806F10800081A76
:1078F000A84276D3218806F10800091A05F1140080
:10790000814229D306F1080028441FFA80F800BFFD
:10791000B8F5C86F08D100BF4AA340F2873255A11D
:1079200059A0FCF741F900BF00BF404602F06AFDD4
:10793000074600213971218839807E80A4F80080B3
:10794000012020713888B0F5C86F07D0388802F060
:1079500059FDA0F8028001E001202071384800683C
:10796000844227D13648D0F800A004E0BAF80000DD
:1079700002F048FD82469AF8040018B14C480068AD
:107980008245F3D12E48C0F800A000BF00684849E6
:10799000096888420CD02A480068007940B100BFCD
:1079A00028A340F2B53243A137A0FCF7FDF800BF91
:1079B00000BF00BF214802F0F1FE00BF04F1080043
:1079C00028443B490968884208D900BF1DA340F2FA
:1079D000B9323FA12CA0FCF7E7F800BF00BF00BF01
:1079E00000E01DE004F0030040B100BF15A340F229
:1079F000BB3243A124A0FCF7D7F800BF00BF00BFF3
:107A000004F0030040B100BF0EA340F2BD3248A114
:107A10001DA0FCF7C9F800BF00BF04F1080042E751
:107A2000304602F0EFFC0688C5F5C860B0423FF66C
:107A300054AF024802F0B2FE002034E7E00000201C
:107A4000E40000202E2E2F4D6964646C657761720E
:107A500065732F54686972645F50617274792F4C3A
:107A60007749502F7372632F636F72652F6D656D49
:107A70002E630000696E76616C6964206E657874AF
:107A80002070747200000000417373657274696F36
:107A90006E2022257322206661696C656420617402
:107AA000206C696E6520256420696E2025730A00AC
:107AB000DC0000206D656D5F6D616C6C6F633A205A
:107AC000216C667265652D3E75736564000000006B
:107AD0006D656D5F6D616C6C6F633A20616C6C6F8E
:107AE0006361746564206D656D6F7279206E6F746B
:107AF0002061626F76652072616D5F656E642E0035
:107B00006D656D5F6D616C6C6F633A20616C6C6F5D
:107B10006361746564206D656D6F72792070726F3A
:107B20007065726C7920616C69676E65642E000007
:107B30006D656D5F6D616C6C6F633A2073616E692A
:107B4000747920636865636B20616C69676E6D652D
:107B50006E740000014602480088081A80B270471F
:107B6000D80000202DE9F84F81468B460BF1030029
:107B700020F0030085B20C2D00D20C25B5F5C86F9E
:107B800001D85D4502DA0020BDE8F88F00BF5C48EF
:107B90000068814503D35B480068814508D300BF76
:107BA00059A340F2D12264A169A0FBF7FDFF00BFF9
:107BB00000BF53480068814503D35248006881459F
:107BC00009D300BF02F058FD0090009802F060FD5C
:107BD00000BF4846D8E7A9F108063046FFF7BAFFCC
:107BE00007463188C81B08381FFA80FA00BF554580
:107BF00008DD00BF44A34FF439725FA154A0FBF726
:107C0000D3FF00BF00BF554501DD0020BCE755454F
:107C100001D14846B8E7604802F0A8FD308802F07C
:107C2000F1FB04462079002833D100BF3088B0F53D
:107C3000C86F08D100BF34A340F2F52257A144A079
:107C4000FBF7B2FF00BF00BF2088009007F10800DB
:107C500028441FFA80F856480068A04204D14046E4
:107C600002F0D0FB52490860404602F0CBFB0446CC
:107C700000202071009820806780A6F8008020886E
:107C8000B0F5C86F04D0208802F0BCFBA0F80280D9
:107C900031E005F1140050452DD807F108002844C3
:107CA0001FFA80F800BF3088B0F5C86F08D100BF58
:107CB00015A340F2163239A125A0FBF775FF00BFCE
:107CC00000BF404602F09EFB0446394800688442EB
:107CD00001D23748046000202071308820806780FE
:107CE000A6F800802088B0F5C86F04D0208802F084
:107CF00089FBA0F80280284802F050FD484643E77F
:107D0000D8000020DC0000202E2E2F4D6964646C0A
:107D10006577617265732F54686972645F50617230
:107D200074792F4C7749502F7372632F636F72658C
:107D30002F6D656D2E6300006D656D5F7472696DEA
:107D40003A206C6567616C206D656D6F727900001B
:107D5000417373657274696F6E20222573222066E9
:107D600061696C6564206174206C696E65202564AE
:107D700020696E2025730A006D656D5F7472696DF0
:107D80002063616E206F6E6C7920736872696E6B10
:107D9000206D656D6F727900E0000020696E76617C
:107DA0006C6964206E657874207074720000000045
:107DB000E400002070B504460D4600BF0D2C09DB21
:107DC00000BF0AA34FF4D57214A11BA0FBF7ECFE71
:107DD00000BF70BD00BF05B9FBE7214951F8240081
:107DE0002946FCF767FB00BFF3E700002E2E2F4D5E
:107DF0006964646C6577617265732F546869726435
:107E00005F50617274792F4C7749502F7372632FD2
:107E1000636F72652F6D656D702E63006D656D709B
:107E20005F667265653A2074797065203C204D4527
:107E30004D505F4D41580000417373657274696F16
:107E40006E2022257322206661696C65642061744E
:107E5000206C696E6520256420696E2025730A00F8
:107E6000742A010870B504460D4600BF002C08D1E5
:107E700000BF09A340F2951213A118A0FBF794FECE
:107E800000BF00BF04B105B970BD29462046FCF70C
:107E900011FB00BFF8E700002E2E2F4D6964646CC3
:107EA0006577617265732F54686972645F5061729F
:107EB00074792F4C7749502F7372632F636F7265FB
:107EC0002F6D656D702E6300696E76616C6964203C
:107ED000706F6F6C2064657363000000417373659D
:107EE0007274696F6E2022257322206661696C6549
:107EF00064206174206C696E6520256420696E20A1
:107F000025730A0010B5002406E0054951F8240045
:107F100000F008F8601C84B20D2CF6D310BD0000F0
:107F2000742A010810B50023846823604368DB1CB1
:107F300023F00301002207E083681B680B6083685D
:107F4000196003881944521C43889342F4DC10BD25
:107F500070B5044600BF0D2C0ADB00BF09A340F238
:107F6000571214A11BA0FBF71FFE00BF002070BD1D
:107F700000BF224951F82400FCF7FAFA05462846CA
:107F8000F5E700002E2E2F4D6964646C65776172F1
:107F900065732F54686972645F50617274792F4CF5
:107FA0007749502F7372632F636F72652F6D656D04
:107FB000702E63006D656D705F6D616C6C6F633A00
:107FC0002074797065203C204D454D505F4D4158DF
:107FD00000000000417373657274696F6E20222582
:107FE0007322206661696C6564206174206C696E1F
:107FF0006520256420696E2025730A00742A010813
:1080000010B5044600BF002C08D100BF07A34FF4F1
:108010009E7212A116A0FBF7C7FD00BF00BF0CB9EE
:10802000002010BD2046FCF7A3FAFAE72E2E2F4DB4
:108030006964646C6577617265732F5468697264F2
:108040005F50617274792F4C7749502F7372632F90
:10805000636F72652F6D656D702E6300696E76615A
:108060006C696420706F6F6C20646573630000003E
:10807000417373657274696F6E20222573222066C6
:1080800061696C6564206174206C696E652025648B
:1080900020696E2025730A002DE9F05F04460E4624
:1080A00017469846DDE90AB900BF002C0BD100BF86
:1080B00049A340F2271255A15BA0FBF775FD00BF55
:1080C0000020BDE8F09F00BF00BFB9F1000F0AD14A
:1080D00000BF41A34FF494725DA153A0FBF764FD70
:1080E00000BF0020EDE700BF06B9624E07B9614F3F
:1080F000B8F1000F01D1DFF87C8100206060A06042
:10810000E0605D4860610020A08484F82D00E0619B
:10811000C4F820B05948007884F830000C982061E9
:1081200043463A463146204600F0F8F92046C84713
:1081300008B10020C5E700BF94F83000FF2802D145
:10814000002084F830004FF0000A4D48056829E00F
:1081500000BFA54208D100BF1FA340F28B1249A166
:1081600031A0FBF721FD00BF00BF0AF1010A00BFEB
:10817000BAF1FF0F08DD00BF17A340F28D1246A130
:1081800029A0FBF711FD00BF00BF95F8300094F85F
:108190003010884205D194F83000401C84F830003B
:1081A00002E02D68002DD3D100BF002DC4D194F87A
:1081B0003000FE2803D100203049087004E094F814
:1081C0003000401C2D4908702D48006820602C4864
:1081D0000460204675E700002E2E2F4D6964646C04
:1081E0006577617265732F54686972645F5061725C
:1081F00074792F4C7749502F7372632F636F7265B8
:108200002F6E657469662E63000000006E657469E8
:10821000665F6164643A20696E76616C6964206EA1
:108220006574696600000000417373657274696F5C
:108230006E2022257322206661696C65642061745A
:10824000206C696E6520256420696E2025730A0004
:108250006E657469665F6164643A204E6F20696E72
:1082600069742066756E6374696F6E2067697665E0
:108270006E000000142B0108158500082401002061
:108280001C0100206E6574696620616C7265616412
:108290007920616464656400746F6F206D616E792C
:1082A000206E65746966732C206D61782E2073755D
:1082B00070706F72746564206E756D62657220698E
:1082C000732032353500000070B504460D4629464E
:1082D000204604F0D7FA2946204608F035FF70BD45
:1082E00010B503460868DC68A04201D1012000E017
:1082F000002030B909B9002000E00868D8600120EA
:1083000010BD0020FCE70000F8B505460C461646F7
:1083100000BF002C08D100BF18A340F2CB1224A14B
:1083200027A0FBF741FC00BF00BF00BF46B900BF5C
:1083300012A34FF4E6721EA121A0FBF735FC00BF8B
:1083400000BF20686968884201D1012000E0002058
:1083500090B9206800906868306069463046FFF741
:10836000B3FF0CB9002000E02068686001212846B6
:1083700000F064F80120F8BD0020FCE72E2E2F4D00
:108380006964646C6577617265732F54686972649F
:108390005F50617274792F4C7749502F7372632F3D
:1083A000636F72652F6E657469662E63000000004E
:1083B000696E76616C696420706F696E74657200B5
:1083C000417373657274696F6E2022257322206673
:1083D00061696C6564206174206C696E6520256438
:1083E00020696E2025730A0010B5034608689C6852
:1083F000A04201D1012000E0002030B909B90020DD
:1084000000E008689860012010BD0020FCE7000033
:1084100002466AB10748016808E091F83000401C44
:10842000C0B2904201D10846704709680029F4D1D2
:108430000020F9E71C0100207047000070B50446D9
:108440000D4600BF002C08D100BF12A340F26D32D0
:108450001DA126A0FBF7A8FB00BF00BF94F82D00CC
:1084600000F0040020B194F82D0000F0010000B9E4
:1084700070BD05F0010050B1606840B194F82D0066
:1084800000F0080018B1211D2046FCF70DFF00BFC9
:10849000EEE700002E2E2F4D6964646C65776172E3
:1084A00065732F54686972645F50617274792F4CE0
:1084B0007749502F7372632F636F72652F6E6574E7
:1084C00069662E63000000006E657469665F6973FB
:1084D0007375655F7265706F7274733A20696E763A
:1084E000616C6964206E6574696600004173736530
:1084F0007274696F6E2022257322206661696C6533
:1085000064206174206C696E6520256420696E208A
:1085100025730A0003466FF00B0070472DE9F84FF2
:1085200080460C4615461E464FF00009CA4604B95F
:10853000114C05B9104D06B90F4E0CB1206808B9A1
:10854000012000E00020074627B16A462146404648
:10855000FFF7DAFE4A4629464046FFF745FF5246F6
:1085600031464046FFF7BCFE27B96A4621464046E1
:10857000FFF7CAFEBDE8F88F142B01080149086017
:10858000704700002001002010B5044600BF002CF9
:1085900009D100BF10A340F29B321CA123A0FBF71E
:1085A00003FB00BF10BD00BF94F82D0000F00100D8
:1085B00078B100BF94F82D0000F0FE0084F82D0083
:1085C00000BF94F82D0000F0080010B12046FCF721
:1085D00033F800BFE6E700002E2E2F4D6964646C6F
:1085E0006577617265732F54686972645F50617258
:1085F00074792F4C7749502F7372632F636F7265B4
:108600002F6E657469662E63000000006E657469E4
:10861000665F7365745F646F776E3A20696E76612A
:108620006C6964206E65746966000000417373654F
:108630007274696F6E2022257322206661696C65F1
:1086400064206174206C696E6520256420696E2049
:1086500025730A0000B1C1617047000010B50446DF
:1086600000BF002C09D100BF0FA340F206421BA19E
:1086700023A0FBF799FA00BF10BD00BF94F82D00AE
:1086800000F0040070B100BF94F82D0000F0FB0072
:1086900084F82D0000BF00BFE06910B12046E169F9
:1086A000884700BF00BFE7E72E2E2F4D6964646C3A
:1086B0006577617265732F54686972645F50617287
:1086C00074792F4C7749502F7372632F636F7265E3
:1086D0002F6E657469662E63000000006E65746914
:1086E000665F7365745F6C696E6B5F646F776E3A1B
:1086F00020696E76616C6964206E6574696600003D
:10870000417373657274696F6E202225732220662F
:1087100061696C6564206174206C696E65202564F4
:1087200020696E2025730A0010B5044600BF002C96
:1087300009D100BF11A34FF478721DA125A0FBF74A
:1087400033FA00BF10BD00BF94F82D0000F0040004
:1087500090B900BF94F82D0040F0040084F82D007B
:1087600000BF03212046FFF769FE00BFE06910B19A
:108770002046E169884700BF00BFE3E72E2E2F4D5A
:108780006964646C6577617265732F54686972649B
:108790005F50617274792F4C7749502F7372632F39
:1087A000636F72652F6E657469662E63000000004A
:1087B0006E657469665F7365745F6C696E6B5F7517
:1087C000703A20696E76616C6964206E65746966C2
:1087D00000000000417373657274696F6E2022257A
:1087E0007322206661696C6564206174206C696E17
:1087F0006520256420696E2025730A0010B50446A3
:1088000000BF002C09D100BF0EA34FF454721AA16F
:1088100020A0FBF7C9F900BF10BD00BF94F82D00E0
:1088200000F0010058B900BF94F82D0040F001009D
:1088300084F82D0000BF03212046FFF7FFFD00BF95
:10884000EAE700002E2E2F4D6964646C6577617233
:1088500065732F54686972645F50617274792F4C2C
:108860007749502F7372632F636F72652F6E657433
:1088700069662E63000000006E657469665F73654B
:10888000745F75703A20696E76616C6964206E65FC
:1088900074696600417373657274696F6E20222576
:1088A0007322206661696C6564206174206C696E56
:1088B0006520256420696E2025730A0070B5044682
:1088C00025460DB1294600E00121084608F094FD37
:1088D000002070BD10B508F0D7FE002010BD10B507
:1088E000FDF7E5FA10B109F0DDFD10BD09F0D4FD8A
:1088F000FBE7F8B504460D46A06840B1E06830B12A
:108900000020009094E80F0009F06BF8F8BD0022F9
:10891000D4E9000109F038F8F8E700002DE9FF413B
:1089200007460D4614460295002001903DB980206F
:1089300000909DE8070087E80700BDE8FF81002060
:1089400003900026601C08B9761E03E014B1264689
:1089500006B90126FDF7ABFAB0B103AA01A9284672
:1089600009F072FB012802D11020009001E00020E4
:1089700000900398B8B14FF080500E490860BFF3E3
:108980004F8FBFF36F8F0EE0324601A9284609F0E2
:10899000A7FA012802D11020009004E00EB90020AF
:1089A00000E0402000909DE8070087E8070000BF36
:1089B000C3E7000004ED00E077B581B00646144639
:1089C00000200090254605B90125FDF770FAA8B1F1
:1089D00000236A4602A9304609F094F9012802D022
:1089E000FF2004B070BD009890B14FF0805009494D
:1089F0000860BFF34F8FBFF36F8F09E000232A4653
:108A000002A9304609F0AAF8012801D0FF20E8E7C2
:108A10000020E6E704ED00E010B50446606820B1F0
:108A20000120616808F09BFF10BD012008F086FF5F
:108A3000FAE7000038B50446002500200090FDF755
:108A400036FA90B16946204609F0DAF9012801D0DA
:108A5000FF2038BD009888B14FF080500849086069
:108A6000BFF34F8FBFF36F8F08E000231A461946FC
:108A7000204609F073F8012800D0FF252846E8E7D2
:108A800004ED00E0F8B506460C46002000900EB953
:108A90008020F8BD0025601C08B96D1E03E014B1EC
:108AA000254605B90125FDF702FA98B16A4600216D
:108AB000304609F0C9FA012801D0FF20E9E7009803
:108AC00080B14FF0805008490860BFF34F8FBFF36B
:108AD0006F8F07E02946304609F01CFB012801D0C2
:108AE000FF20D6E70020D4E704ED00E038B50446C7
:108AF000002500200090FDF7DAF990B16946204684
:108B000009F07EF9012801D0FF2038BD009888B116
:108B10004FF0805008490860BFF34F8FBFF36F8F4D
:108B200008E000231A461946204609F017F80128E4
:108B300000D0FF252846E8E704ED00E0F8B506463A
:108B40000C46002000900EB98020F8BD0025601C66
:108B500008B96D1E03E014B1254605B90125FDF7DE
:108B6000A6F998B16A460021304609F06DFA01284D
:108B700001D0FF20E9E7009880B14FF0805008490C
:108B80000860BFF34F8FBFF36F8F07E02946304671
:108B900009F0C0FA012801D0FF20D6E70020D4E771
:108BA00004ED00E07FB504460D46606998B1A06908
:108BB00088B1B4F90800FEF7B9FC0646D4E90510FF
:108BC000CDE9006102902B462269D4E9001009F03A
:108BD000F5FB039013E0B4F90800FEF7A7FC064686
:108BE00003A8CDE90060238A9AB22B46D4E900108D
:108BF00009F0B2FB012802D0002004B070BD039838
:108C0000FBE710B50446204608F024FC002010BD08
:108C100070B504460D4600222946204600F002F8B1
:108C200070BD00002DE9F04704460D46904600BF98
:108C300044B900BF1CA340F2DF1227A129A0FAF714
:108C4000B3FF00BF00BF14B1B5F5803F02D30120D0
:108C5000BDE8F0870DB90020FAE7AEB220893044B4
:108C600080B2B04201DA0120F2E794F80C9009F0EA
:108C7000800038B16068471B04F11000874209D2B8
:108C80000120E5E7B8F1000F02D06068471B01E062
:108C90000120DDE7676060893044608120893044CD
:108CA00020810020D4E700002E2E2F4D6964646CD3
:108CB0006577617265732F54686972645F50617281
:108CC00074792F4C7749502F7372632F636F7265DD
:108CD0002F706275662E63007020213D204E554C2A
:108CE0004C000000417373657274696F6E20222519
:108CF0007322206661696C6564206174206C696E02
:108D00006520256420696E2025730A002DE9FE4F39
:108D100082460E4690465746B8F1010F0AD0B8F188
:108D2000410F06D0B8F5C17F0BD0B8F5207F7DD1BB
:108D30006AE000BF42463146002000F037F90446A1
:108D4000AEE0002400200290B14600BF0C20FFF7E7
:108D5000FFF8054645B900F0A9FD14B1204600F022
:108D60006BFC0020BDE8FE8FF81C20F00300C0F56E
:108D7000147080B2484501DD484605E0F81C20F03B
:108D80000300C0F5147080B283460020CDE9008056
:108D900005F110003844C01C20F003015B464A4630
:108DA000284600F074FD00BF287900F00300002879
:108DB00008D000BF3CA34FF4807247A152A0FAF73D
:108DC000F3FE00BF00BF00BFF81C20F00300C0F599
:108DD0001470002808D100BF33A34FF4817254A14E
:108DE00049A0FAF7E1FE00BF00BF0CB92C4601E034
:108DF000029805600295A9EB0B001FFA80F9002785
:108E0000B9F1000FA2DC4BE0F81C20F00301F01CCC
:108E100020F00300084485B205F110001FFA80F924
:108E2000F01C20F00300A84206D800E02BE0F01C64
:108E300020F00300484501D9002093E74846FEF79B
:108E40002BFD04460CB900208CE70020CDE9008002
:108E500004F110003844C01C20F0030133463246B0
:108E6000204600F014FD00BF207900F0030040B15F
:108E700000BF0DA34FF491723AA123A0FAF794FE1C
:108E800000BF00BF0CE000BF00BF07A340F22712E5
:108E90003FA11DA0FAF788FE00BF00BF002061E7D8
:108EA00000BF20465EE700002E2E2F4D6964646CE3
:108EB0006577617265732F54686972645F5061727F
:108EC00074792F4C7749502F7372632F636F7265DB
:108ED0002F706275662E6300706275665F616C6CE0
:108EE0006F633A207062756620712D3E7061796CF7
:108EF0006F61642070726F7065726C7920616C694B
:108F0000676E656400000000417373657274696F79
:108F10006E2022257322206661696C65642061746D
:108F2000206C696E6520256420696E2025730A0017
:108F3000504255465F504F4F4C5F42554653495A39
:108F400045206D757374206265206269676765727C
:108F5000207468616E204D454D5F414C49474E4D30
:108F6000454E5400706275665F616C6C6F633A20A9
:108F7000706275662D3E7061796C6F6164207072ED
:108F80006F7065726C7920616C69676E6564000052
:108F9000706275665F616C6C6F633A206572726FA8
:108FA0006E656F7573207479706500002DE9FC4162
:108FB00007460D46144600BF412C0AD0012C08D0AC
:108FC00000BF0EA34FF4A57218A11DA0FAF7ECFD87
:108FD00000BF00BF0B20FEF7BBFF064616B90020FE
:108FE000BDE8FC8100202B462A463946CDE90040E9
:108FF000304600F04CFC3046F2E700002E2E2F4D9C
:109000006964646C6577617265732F546869726412
:109010005F50617274792F4C7749502F7372632FB0
:10902000636F72652F706275662E6300696E76617C
:109030006C696420706275665F7479706500000009
:10904000417373657274696F6E20222573222066E6
:1090500061696C6564206174206C696E65202564AB
:1090600020696E2025730A002DE9FC5F05460C4639
:1090700017469846DDE90C9BAA460AF1030020F04A
:1090800003002044584502D90020BDE8FC9FB9F1F7
:10909000000F06D00AF1030020F0030000EB0906E0
:1090A00000E000260220234622463146CDE900702A
:1090B000404600F0ECFB4046E7E7000070B506468E
:1090C0000D4600BF0EB1002D09D100BF1BA340F219
:1090D000593226A133A0FAF767FD00BF70BD00BF6B
:1090E000344604E0208929890844208124682068C6
:1090F0000028F7D100BF20896189884208D000BFCD
:109100000EA340F2623231A126A0FAF74DFD00BF56
:1091100000BF00BF206840B100BF08A340F2633227
:1091200036A120A0FAF740FD00BF00BF20892989A1
:1091300008442081256000BFD0E700002E2E2F4D6F
:109140006964646C6577617265732F5468697264D1
:109150005F50617274792F4C7749502F7372632F6F
:10916000636F72652F706275662E63002868202118
:109170003D204E554C4C2920262620287420213D88
:10918000204E554C4C29202870726F6772616D6DAE
:1091900065722076696F6C6174657320415049294E
:1091A00000000000417373657274696F6E202225A0
:1091B0007322206661696C6564206174206C696E3D
:1091C0006520256420696E2025730A00702D3E7489
:1091D0006F745F6C656E203D3D20702D3E6C656E3A
:1091E00020286F66206C6173742070627566206938
:1091F0006E20636861696E2900000000702D3E6E6C
:10920000657874203D3D204E554C4C0001460020B1
:1092100002E0421C90B209680029FAD170470000B0
:109220002DE9F04180460E461446218932464046DB
:10923000FFF76CFD074617B90020BDE8F081214615
:10924000384600F045F8054600BF45B100BF05A30C
:1092500040F224520FA114A0FAF7A6FC00BF00BFF1
:109260003846EAE72E2E2F4D6964646C657761728B
:1092700065732F54686972645F50617274792F4C02
:109280007749502F7372632F636F72652F70627509
:10929000662E6300706275665F636F707920666129
:1092A000696C656400000000417373657274696FD6
:1092B0006E2022257322206661696C6564206174CA
:1092C000206C696E6520256420696E2025730A0074
:1092D0002DE9F04105460C460026002700BF25B1C8
:1092E0001CB12889218988420CDA00BF44A340F2CE
:1092F000C9324FA15AA0FAF757FC00BF6FF00F0018
:10930000BDE8F08100BF00BF6889801B6189C91B6F
:10931000884203D36089A0EB070802E06889A0EBCC
:1093200006086268D1196A6890194246F6F7EEFF9E
:109330004644474400BF6889B04208D200BF30A30A
:1093400040F2D93250A146A0FAF72EFC00BF00BF70
:1093500000BF6089B84208D200BF29A340F2DA32C8
:109360004FA13FA0FAF720FC00BF00BF6089B842C0
:1093700001D8002724686889B04211D100262D68E1
:1093800000BF65B95CB100BF1DA34FF479724BA15A
:1093900033A0FAF709FC00BF6FF00F00B0E700BF81
:1093A000002C13D06089218988420FD100BF20682A
:1093B00058B100BF12A340F2E93244A128A0FAF745
:1093C000F3FB00BF6FF005009AE700BF002D13D03C
:1093D0006889298988420FD100BF286858B100BF29
:1093E00007A340F2EE3239A11DA0FAF7DDFB00BF62
:1093F0006FF0050084E700BF002C85D100207FE7D7
:109400002E2E2F4D6964646C6577617265732F54DD
:10941000686972645F50617274792F4C7749502F7C
:109420007372632F636F72652F706275662E6300AF
:10943000706275665F636F70793A207461726765F8
:1094400074206E6F742062696720656E6F7567683F
:1094500020746F20686F6C6420736F757263650091
:10946000417373657274696F6E20222573222066C2
:1094700061696C6564206174206C696E6520256487
:1094800020696E2025730A006F66667365745F74C9
:109490006F203C3D20705F746F2D3E6C656E000048
:1094A0006F66667365745F66726F6D203C3D2070F9
:1094B0005F66726F6D2D3E6C656E0000705F746F3D
:1094C00020213D204E554C4C000000007062756616
:1094D0005F636F7079282920646F6573206E6F74E5
:1094E00020616C6C6F77207061636B65742071759F
:1094F00065756573210000002DE9F05F804689469F
:1095000016461D464FF0000AD34600BFB8F1000FC3
:109510000BD100BF21A340F20A422CA133A0FAF7DD
:1095200043FB00BF0020BDE8F09F00BF00BFB9F1C2
:10953000000F0AD100BF19A340F20B4235A12BA0A6
:10954000FAF732FB00BF0020EDE700BF444620E001
:1095500035B16089A84203DC6089281A85B217E01A
:109560006089401B87B2B74200DD374662685119F7
:1095700009EB0A003A46F6F7C9FE0BEB07001FFAA3
:1095800080FB0AEB07001FFA80FAF01B86B2002569
:1095900024680EB1002CDBD15846C4E72E2E2F4D87
:1095A0006964646C6577617265732F54686972646D
:1095B0005F50617274792F4C7749502F7372632F0B
:1095C000636F72652F706275662E630070627566D8
:1095D0005F636F70795F7061727469616C3A206962
:1095E0006E76616C69642062756600004173736514
:1095F0007274696F6E2022257322206661696C6522
:1096000064206174206C696E6520256420696E2079
:1096100025730A00706275665F636F70795F7061B1
:10962000727469616C3A20696E76616C6964206459
:1096300061746170747200002DE9F0470446002CDB
:109640000ED100BF44B900BF38A34FF4377243A115
:1096500045A0FAF7A9FA00BF00BF0020BDE8F087D7
:1096600000265EE001F008F8824600BFA07B0028DB
:1096700008DC00BF2DA340F2F12245A13AA0FAF781
:1096800093FA00BF00BFA07B401E00F0FF0884F8E3
:109690000E80504600F0FCFFB8F1000F3FD1276864
:1096A000207B00F00F05607B00F00200002814D042
:1096B000A14600BFD9F81000002808D100BF1BA3A5
:1096C00040F2FF2238A128A0FAF76EFA00BF00BFCF
:1096D0002046D9F8101088471DE0022D04D12146FC
:1096E0000C20FEF767FB16E0012D04D121460B206C
:1096F000FEF760FB0FE01DB92046FDF71FFF0AE0F3
:1097000000BF00BF09A340F20F3230A116A0FAF744
:109710004BFA00BF00BF701CC6B23C4600E00024FC
:1097200000BF002C9ED1304698E700002E2E2F4D12
:109730006964646C6577617265732F5468697264DB
:109740005F50617274792F4C7749502F7372632F79
:10975000636F72652F706275662E63007020213D05
:10976000204E554C4C000000417373657274696F54
:109770006E2022257322206661696C656420617405
:10978000206C696E6520256420696E2025730A00AF
:10979000706275665F667265653A20702D3E72650F
:1097A00066203E203000000070632D3E63757374A8
:1097B0006F6D5F667265655F66756E6374696F6E07
:1097C00020213D204E554C4C00000000696E766112
:1097D0006C696420706275662074797065000000A1
:1097E00070B50446254629460748FEF73BFB074867
:1097F0000078012806D10020044908700448006858
:10980000FFF774F970BD00008829010828000020C6
:109810002C00002070B500BF00F02EFF0546002090
:1098200009490870284600F033FF00BF0748046864
:1098300006E0606F18B1204602F0C4F870BDE4681D
:10984000002CF6D100BFF9E72501002038010020E7
:1098500010B50446FFF7DEFF10BD70B504460D4697
:1098600001222946204600F001F870BD70B505467A
:109870000C461646002C04DA6142284600F040F9F6
:1098800070BD324621462846FFF7CCF9F8E770B59F
:10989000DDE90445002606604160028143810473CE
:1098A0004573012686730026C67370BD70B500F03F
:1098B000E3FE05460C48047801200B490870284651
:1098C00000F0E6FE7CB900BF0021084807F00CFA62
:1098D00040B100F0D1FE054600200349087028463B
:1098E00000F0D6FE00BF70BD250100205198000891
:1098F0002DE9F04106460F4600BF002E08D100BFFB
:109900002CA34FF4CC7237A13CA0FAF74DF900BF5D
:1099100000BF3089B84201DCBDE8F0813089C01B4E
:109920001FFA80F83D46344613E06089281A85B254
:109930002089A0EB08002081246800BF44B900BF43
:109940001CA340F2AF1237A12CA0FAF72DF900BFEB
:1099500000BF6089A842E8DB207B00F00F000028F0
:109960001BD16089A84218D0607B00F0020000285B
:1099700013D1A088001B284481B22046FEF7F2F8DC
:10998000044600BF44B900BF0AA340F2BD122BA198
:109990001AA0FAF709F900BF00BF6581608920812C
:1099A000206810B12068FFF747FE0020206000BF4C
:1099B000B2E700002E2E2F4D6964646C65776172EA
:1099C00065732F54686972645F50617274792F4CAB
:1099D0007749502F7372632F636F72652F706275B2
:1099E000662E6300706275665F7265616C6C6F6392
:1099F0003A207020213D204E554C4C004173736538
:109A00007274696F6E2022257322206661696C650D
:109A100064206174206C696E6520256420696E2065
:109A200025730A00706275665F7265616C6C6F63A6
:109A30003A207120213D204E554C4C006D656D5FE4
:109A40007472696D2072657475726E656420712020
:109A50003D3D204E554C4C0070B50446002C18D0AE
:109A600000BF00F009FE0546A07B401CA0732846FD
:109A700000F00EFE00BF00BFA07B002808DC00BF86
:109A800004A340F242320FA113A0FAF78DF800BFF1
:109A900000BF70BD2E2E2F4D6964646C65776172B6
:109AA00065732F54686972645F50617274792F4CCA
:109AB0007749502F7372632F636F72652F706275D1
:109AC000662E63007062756620726566206F76652B
:109AD00072666C6F77000000417373657274696F12
:109AE0006E2022257322206661696C656420617492
:109AF000206C696E6520256420696E2025730A003C
:109B00002DE9F04104460D4600BF44B900BF18A33B
:109B100040F24B2222A125A0FAF746F800BF00BF71
:109B200014B1B5F5803F02D30120BDE8F0810DB935
:109B30000020FAE7AEB200BF6089B0420ADA00BF87
:109B40000BA340F2552223A118A0FAF72DF800BF6D
:109B50000120EAE700BF67686068284460606089A8
:109B6000801B60812089801B20810020DDE70000B0
:109B70002E2E2F4D6964646C6577617265732F5466
:109B8000686972645F50617274792F4C7749502F05
:109B90007372632F636F72652F706275662E630038
:109BA0007020213D204E554C4C00000041737365E0
:109BB0007274696F6E2022257322206661696C655C
:109BC00064206174206C696E6520256420696E20B4
:109BD00025730A00696E6372656D656E745F6D61F1
:109BE000676E6974756465203C3D20702D3E6C6520
:109BF0006E0000002DE9F041044600BF3B480068BC
:109C0000844208D200BF3AA340F2DF1244A14AA026
:109C1000F9F7CAFF00BF00BF00BF51480068844287
:109C200008D300BF32A34FF4F0724EA142A0F9F75F
:109C3000BBFF00BF00BF00BF2079002808D000BFD5
:109C40002BA340F2E1124EA13BA0F9F7ADFF00BFFC
:109C500000BF00BF2088B0F5C86F08D900BF24A39B
:109C60004FF4F2724DA134A0F9F79EFF00BF00BF80
:109C7000208800F0C7FB0546AC4219D02879B8B956
:109C800037480068854213D04F480068A84201D188
:109C90004D480460288820802888B0F5C86F07D018
:109CA0002046FDF757FF0746288800F0ABFB4780AA
:109CB000608800F0A7FB0646A64215D0307998B917
:109CC00041480068A04201D13F48066020883080AA
:109CD0002088B0F5C86F07D03046FDF73BFF074638
:109CE000208800F08FFB4780BDE8F081D80000207D
:109CF0002E2E2F4D6964646C6577617265732F54E5
:109D0000686972645F50617274792F4C7749502F83
:109D10007372632F636F72652F6D656D2E63000024
:109D2000706C75675F686F6C65733A206D656D2048
:109D30003E3D2072616D0000417373657274696FFE
:109D40006E2022257322206661696C65642061742F
:109D5000206C696E6520256420696E2025730A00D9
:109D6000DC000020706C75675F686F6C65733A206B
:109D70006D656D203C2072616D5F656E6400000052
:109D8000706C75675F686F6C65733A206D656D2DDB
:109D90003E75736564203D3D20300000706C756732
:109DA0005F686F6C65733A206D656D2D3E6E6578EA
:109DB00074203C3D204D454D5F53495A455F414C11
:109DC00049474E4544000000E40000202DE9F041E1
:109DD00005460E461C4807681C480068001D07F031
:109DE000CBF950B91948006890F82C100120884030
:109DF00017490968814316480160681C38B936B1B3
:109E000012480168091D134807F000FA1AE07C198E
:109E10000E4800684460BC4207D20C480168091D26
:109E20000D48006807F0D8F90CE008480168091DE2
:109E30000A48006807F0D0F909480068844201D256
:109E400007480460BDE8F081740000206000002035
:109E50007800002054540020680000206400002096
:109E60009000002010B5044607F0DCF92348006894
:109E7000401C224908602248006840B9204804601C
:109E80000846006801280DD100F0BEF90AE01D481F
:109E9000006838B91A480068C06AE16A884201D887
:109EA0001748046018480068401C1749086094F877
:109EB0002C1001208840154909680843134908609F
:109EC000E16A01EB8101124A02EB8100211D07F0DA
:109ED0009DF907F0D1F90B48006868B1084800689F
:109EE000C06AE16A884207D24FF080500949086091
:109EF000BFF34F8FBFF36F8F10BD000070000020C5
:109F0000600000207C0000208C00002078000020F1
:109F10008451002004ED00E010B516E007F082F94E
:109F20000C48C068C468201D07F026F90A4800687C
:109F3000401E0949086009480068401E074908603A
:109F400007F09AF9204600F05FF8044800680028FE
:109F5000E4D110BD40540020700000206C000020AF
:109F600070B504460D46206C70B1216CE068014468
:109F7000E160D4E90210884201D32168E1602846FB
:109F8000226CE168F6F7C2F970BD2DE9F041044694
:109F90000F4615464FF00008A66B206C48B92068A4
:109FA00000282CD1A06808F02BFB80460020A06080
:109FB00025E07DB93946226C6068F6F7A7F9216C77
:109FC000606808446060D4E90101884217D32068C2
:109FD000606014E03946226CE068F6F797F9216C6E
:109FE000E068411AE1602168E068884203D2216C90
:109FF000A068411AE160022D01D106B1761E701CE5
:10A00000A0634046BDE8F08110B5044694F85900BD
:10A0100030B9206B07F04EF9204607F04BF91AE0F3
:10A0200094F85900012803D1204607F043F912E0C3
:10A0300094F85900022801D1012000E0002050B915
:10A0400000BF502080F31188BFF34F8FBFF36F8F95
:10A0500000BF00BFFEE710BD01464A6A22B10A6B8D
:10A060001268C2F1200000E00020704730B54FF4C4
:10A070007053174800F007042CB1C01D20F00700F2
:10A08000134C041B1B1B0246124C22600024114D72
:10A090006C60D018083820F007000F4C20600024B6
:10A0A0000D4D2D686C600C4D2D682C601146441AC6
:10A0B0004C60094C24680C60084D4C682C60084DBD
:10A0C0004C682C604FF00044064D2C6030BD000001
:10A0D000685400209C000020A4000020AC00002058
:10A0E000A8000020B800002000BFFFF715FF0648B9
:10A0F00000680128F9D94FF0805004490860BFF387
:10A100004F8FBFF36F8FF0E78451002004ED00E024
:10A1100010B5044654B10020A06020600021E16029
:10A1200000231A461946204607F018FD10BD2DE9F8
:10A13000F04106460D4617469846069C0DB9246028
:10A1400000E02760E66325640121204607F0BAFCA1
:10A15000BDE8F0812DE9FF5F81460E469246DDE9BC
:10A160000E7B109CAAF10100216B01EB800828F006
:10A17000070808F0070008B9012000E0002050B9E6
:10A1800000BF502080F31188BFF34F8FBFF36F8F54
:10A1900000BF00BFFEE786B1002507E0715D04F156
:10A1A00034004155705D00B902E06D1C182DF5D3E7
:10A1B00000BF00214B20015502E0002084F834004C
:10A1C000202F00D31F27E762E76400202065201DB1
:10A1D00006F0FFFF04F1180006F0FBFF2461C7F151
:10A1E0002000A06164620020606584F85800494640
:10A1F0004046039A00F0C4F92060BBF1000F01D083
:10A20000CBF80040BDE8FF9F10B5002407E004EB49
:10A2100084010F4A02EB810006F0CEFF641C202C63
:10A22000F5D30C4806F0C8FF0B4806F0C5FF0B48F5
:10A2300006F0C2FF0A4806F0BFFF0A4806F0BCFF5E
:10A2400004480949086004480849086010BD000036
:10A250008451002004540020185400202C54002065
:10A260004054002054540020640000206800002066
:10A2700010B50146164800E0006803688B42FBD326
:10A280000246436813448B4204D143684C6823441C
:10A29000436001460A464B6813440468A34211D147
:10A2A0000C4C03682468A34208D04B6804686468B7
:10A2B00023444B6003681B680B6005E0054B1B687B
:10A2C0000B6001E003680B60884200D0016010BDA4
:10A2D0009C000020A400002070B5054606F0A2FFF7
:10A2E000A86B08B9012400E0002406F0C5FF204651
:10A2F00070BD70B5054606F095FFA86BE96B884206
:10A3000001D1012400E0002406F0B6FF204670BD14
:10A310000A490968096809B9012100E0002121B151
:10A320004FF0FF31064A116006E004490968C96828
:10A33000C868034A4168116070470000640000204B
:10A34000900000200E480068401C08B9012000E081
:10A35000002050B900BF502080F31188BFF34F8F09
:10A36000BFF36F8F00BF00BFFEE700BF502080F338
:10A370001188BFF34F8FBFF36F8F00BF00BFFEE7A1
:10A38000BC00002070B5044606F04CFF94F945501F
:10A3900010E0606A08B9012000E0002038B904F13B
:10A3A000240008F0EDF918B107F0DAF800E003E056
:10A3B000681E45B2002DECDC00BFFF2084F845008C
:10A3C00006F05AFF06F02EFF94F9445010E0206981
:10A3D00008B9012000E0002048B904F1100008F09D
:10A3E000CFF908B107F0BCF8681E45B200E001E003
:10A3F000002DECDC00BFFF2084F8440006F03CFF99
:10A4000070BD000001460248006808447047000023
:10A41000D80000202DE9F04104464FF0000807F075
:10A420008BF94948006808B9FFF720FE47480068E3
:10A430002040002870D1D4B1083404F00700B0B136
:10A4400004F00700C0F10800044404F0070008B954
:10A45000012000E0002050B900BF502080F3118897
:10A46000BFF34F8FBFF36F8F00BF00BFFEE7002C1D
:10A4700052D03748006884424ED8364E3046056880
:10A4800001E02E462D686868A04202D228680028A4
:10A49000F7D12D48006885423ED0306800F10808A9
:10A4A000286830606868001B102819D92F1907F038
:10A4B000070008B9012000E0002050B900BF50207B
:10A4C00080F31188BFF34F8FBFF36F8F00BF00BFC2
:10A4D000FEE76868001B78606C603846FFF7C8FECE
:10A4E0001B4968680968081A194908600846006825
:10A4F00019490968884203D215480068164908605E
:10A500001249686809680843686000202860134899
:10A510000068401C1149086008F07EF908F0070047
:10A5200008B9012000E0002050B900BF502080F39E
:10A530001188BFF34F8FBFF36F8F00BF00BFFEE7DF
:10A540004046BDE8F0810000A4000020B8000020D3
:10A55000A80000209C000020AC000020B0000020DB
:10A560000648006830B10549096801F15000096DDD
:10A57000491C01600148006870470000600000202D
:10A58000001F4FF080730360001F21F00103036080
:10A59000001F054B036014380260001F6FF00203B8
:10A5A000036020387047000045A30008F8B5064650
:10A5B0000C4615464FF47A702B46084A2146009007
:10A5C0003046F7F725FF10B14FF0FF30F8BD2A46AF
:10A5D00002492046F5F79AFE0020F7E770D80020E0
:10A5E000F9F710FC00BFFEE7F9F702FF00BF0024F7
:10A5F00006E0B2EE080A2046F9F70EFF601CC4B26E
:10A60000102CF6DB642006F0F7FEF0E7F8F7B8FE52
:10A6100000BF0020FEF7F5FAFBE7F0B587B004466F
:10A620000D461646FEF75BF90746AEB1324601A865
:10A630002168FEF773F901A807C804AB07C30498A3
:10A64000102806D105982860FEF749F9C01B07B00D
:10A65000F0BD4FF0FF30FAE74FF0FF3201A821685C
:10A66000FEF75CF901A807C804AB07C3059828608A
:10A67000FEF735F9C01BEAE710B54FF0FF3103488C
:10A680000068FEF7FFF9012010BD000094010020D2
:10A6900010B5044602480068FEF7CCF910BD000072
:10A6A000940100202DE9F04100F07EF8074600BF3C
:10A6B0000F4804680CB9BDE8F0816068381AB0F141
:10A6C000004F01D3012000E0002000B1F3E708496A
:10A6D00020680860A568E668064960680860214649
:10A6E0000A20FDF767FB0DB13046A847E0E7000000
:10A6F000700100207401002010B50348FEF78CF9AA
:10A700000249086010BD00001C2B010894010020C4
:10A710007FB504460D46094B0FCB8DE80F00009521
:10A7200000216846FEF7E5F82060206818B94FF070
:10A73000FF3004B070BD0020FBE70000242B0108AF
:10A7400070B505460E46002231462868FEF734F9FA
:10A7500008B9002401E04FF0FF34204670BD0146E7
:10A76000086808B9002070470120FCE710B50446CE
:10A770004FF0FF312068FEF785F910BD1CB5044687
:10A780000020009001906846FEF746F9206020689E
:10A7900010B94FF0FF301CBD0020FCE710B5044697
:10A7A0002068FEF747F910BD10B5F7F7D3F810BDD4
:10A7B0002DE9F04188B004460D4616461F46DDF8E7
:10A7C00038801C2101A8F5F7C8FD019402950FFA05
:10A7D00088F0ADF80C000597314601A8FEF7E2F9C4
:10A7E00008B0BDE8F08100002DE9F04104460E46B6
:10A7F000174600BFB4F1804F08D300BF09A340F251
:10A80000291215A122A0F9F7CFF900BF00BFFFF769
:10A81000CBFF05193A463146284600F04DF8BDE811
:10A82000F08100002E2E2F4D6964646C6577617293
:10A8300065732F54686972645F50617274792F4C2C
:10A840007749502F7372632F636F72652F74696D30
:10A85000656F7574732E630054696D656F75742030
:10A8600074696D6520746F6F206C6F6E672C206D3E
:10A870006178206973204C5749505F55494E5433D5
:10A88000325F4D41582F34206D73656373000000B3
:10A89000417373657274696F6E202225732220667E
:10A8A00061696C6564206174206C696E6520256443
:10A8B00020696E2025730A002DE9F04106460F46F7
:10A8C00090460A20FDF744FB0446002C0CD100BF43
:10A8D00007D100BF20A3BE222CA13CA0F9F764F948
:10A8E00000BF00BFBDE8F08100202060A760C4F871
:10A8F0000C8066603F48006810B93E480460F1E78C
:10A900003C49606809684968401AB0F1004F01D3BA
:10A91000012000E0002028B136480068206035485A
:10A92000046017E03348056811E0286850B160689A
:10A9300029684968401AB0F1004F01D3012000E0B6
:10A94000002018B1286820602C6002E02D68002DDE
:10A95000EBD100BF00BFC5E72E2E2F4D6964646C9C
:10A960006577617265732F54686972645F506172B4
:10A9700074792F4C7749502F7372632F636F726510
:10A980002F74696D656F7574732E63007379735FCF
:10A9900074696D656F75743A2074696D656F75744F
:10A9A00020213D204E554C4C2C20706F6F6C204D5B
:10A9B000454D505F5359535F54494D454F555420B1
:10A9C000697320656D7074790000000041737365D0
:10A9D0007274696F6E2022257322206661696C652E
:10A9E00064206174206C696E6520256420696E2086
:10A9F00025730A007001002010B5012408E0064903
:10AA000001EBC40251F834000449FFF7EDFE641C69
:10AA1000032CF4D310BD0000F82A0108E1730008EC
:10AA200070B51548006810B94FF0FF3070BDFFF7E2
:10AA3000BBFE0446104800684068001BB0F1004FA0
:10AA400001D3012000E0002008B10020EEE70A4811
:10AA500000684068051B00BFB5F1004F08D300BF78
:10AA600006A34FF4DC7212A116A0F9F79DF800BFFF
:10AA700000BF2846DAE70000700100202E2E2F4D7F
:10AA80006964646C6577617265732F546869726478
:10AA90005F50617274792F4C7749502F7372632F16
:10AAA000636F72652F74696D656F7574732E6300C3
:10AAB000696E76616C696420736C65657074696D2C
:10AAC00065000000417373657274696F6E20222502
:10AAD0007322206661696C6564206174206C696E04
:10AAE0006520256420696E2025730A002DE9FF5F2B
:10AAF00004460E4600BF002C0AD100BF42A340F21C
:10AB00003D224DA153A0F9F74FF800BFBDE8FF9FCC
:10AB100000BF00BF207D012808D100BF3AA34FF439
:10AB2000107256A14BA0F9F73FF800BF00BF207D7F
:10AB30000A2807D121465E4802F068FE204600F050
:10AB4000FBFD5FE04FF0000AD346276DD4F8248068
:10AB5000D4F89050D4F81090207DE8B9E08A38B34A
:10AB600000BF54480068A04205D152480068C06840
:10AB7000504908600DE04F49086806E0C168A142ED
:10AB800002D1E168C16002E0C0680028F6D100BFD0
:10AB900000BF0020E0600BE0B246B4F816B000BF82
:10ABA0002146454802F032FE01204449087000BFAA
:10ABB000206F10B1206F04F028FEE06E10B1E06E3F
:10ABC00004F023FE606F10B1606F04F01EFEBAF156
:10ABD000000F0AD0208B211D23464246CDE9001BE1
:10ABE00002903946204604F015FD207D0390204652
:10ABF00000F0A2FD00BF1DB16FF00C014846A84750
:10AC000000BF00BF00BF81E72E2E2F4D6964646C2A
:10AC10006577617265732F54686972645F50617201
:10AC200074792F4C7749502F7372632F636F72655D
:10AC30002F7463702E6300007463705F6162616ED5
:10AC4000646F6E3A20696E76616C6964207063622D
:10AC500000000000417373657274696F6E202225D5
:10AC60007322206661696C6564206174206C696E72
:10AC70006520256420696E2025730A00646F6E27A5
:10AC8000742063616C6C207463705F61626F7274B6
:10AC90002F7463705F6162616E646F6E20666F72A5
:10ACA000206C697374656E2D706362730000000020
:10ACB0003C0100203001002038010020400100202C
:10ACC00010B5044601212046FFF710FF10BD00001B
:10ACD00070B505460120FDF73BF904461CBB00F0AA
:10ACE0009FFE01F04DFC0120FDF732F90446CCB97E
:10ACF000092001F0DDFB0120FDF72AF9044684B9A3
:10AD0000082001F0D5FB0120FDF722F904463CB9EB
:10AD1000284601F099FB0120FDF71AF9044600BF0F
:10AD200000BF00BF00BF44B39C212046F5F715FBD0
:10AD30000C3465724FF48660A4F858004000E0833C
:10AD4000A083FF2004F8010C4FF40670E084062075
:10AD5000A0866086C01FA0840120A08708480068E4
:10AD6000606108480078A0744FF48660E087064868
:10AD7000A0670648C4F888000C3C204670BD00005F
:10AD80002C01002042010020D9EE000800DD6D00FA
:10AD900010B5044600BF002C0BD100BF0CA34FF42C
:10ADA000F47217A11CA0F8F7FFFE00BF6FF00F00B0
:10ADB00010BD00BF207D012805D000BF608B40F092
:10ADC0001000608300BF0121204600F039F8EFE752
:10ADD0002E2E2F4D6964646C6577617265732F54F4
:10ADE000686972645F50617274792F4C7749502F93
:10ADF0007372632F636F72652F7463702E6300002C
:10AE00007463705F636C6F73653A20696E76616C12
:10AE10006964207063620000417373657274696FC6
:10AE20006E2022257322206661696C65642061743E
:10AE3000206C696E6520256420696E2025730A00E8
:10AE40003EB504460D4600BF002C08D100BF55A3F7
:10AE50004FF4AF725FA167A0F8F7A6FE00BF00BF76
:10AE6000002D56D0207D042802D0207D072850D107
:10AE7000A06F18B9208DB0F5066F4AD000BFA07E34
:10AE800000F0100040B900BF46A34FF4B27263A1B6
:10AE900058A0F8F789FE00BF00BF208BE18A221D71
:10AEA000CDE90021029023462046626A216D04F01C
:10AEB000B1FB204602F03CFC00BF00BF5E480068CA
:10AEC000A04205D15C480068C0685B4908600DE09D
:10AED0005949086806E0C168A14202D1E168C16031
:10AEE00002E0C0680028F6D100BF00BF0020E0608B
:10AEF00000BF01205149087000BF51480068A042BE
:10AF000002D105F071FB02E0204600F015FC0020A4
:10AF10003EBD207D20B1012824D002283AD12CE06A
:10AF2000E08AD8B100BF47480068A04205D1454833
:10AF30000068C068434908600DE04249086806E0BF
:10AF4000C168A14202D1E168C16002E0C068002886
:10AF5000F6D100BF00BF0020E06000BF204600F037
:10AF6000EBFB1BE0204601F029FB2146364802F0AE
:10AF70004DFC204600F0D8FC10E000BF21462E48D2
:10AF800002F044FC01202D49087000BF204600F06B
:10AF9000D3FB03E0204600F059F8B9E700BF0020DA
:10AFA000B6E700002E2E2F4D6964646C65776172E0
:10AFB00065732F54686972645F50617274792F4CA5
:10AFC0007749502F7372632F636F72652F746370AC
:10AFD0002E6300007463705F636C6F73655F7368EA
:10AFE0007574646F776E3A20696E76616C6964205F
:10AFF00070636200417373657274696F6E202225FD
:10B000007322206661696C6564206174206C696ECE
:10B010006520256420696E2025730A007063622D07
:10B020003E666C61677320262054465F5258434C3D
:10B030004F5345440000000038010020400100202B
:10B040006C010020300100203401002070B505465D
:10B0500000BF45B900BF1EA34FF4CE7228A12BA09C
:10B06000F8F7A2FD00BF00BF287D032804D0042804
:10B070000AD0072818D10FE0284604F073FC0446D4
:10B080000CB90520287511E0284604F06BFC044635
:10B090000CB90520287509E0284604F063FC044635
:10B0A0000CB90920287501E0002070BD00BF1CB953
:10B0B000284601F063FD09E0601C38B900BF688BC9
:10B0C00040F00800688300BF0020EEE72046ECE770
:10B0D0002E2E2F4D6964646C6577617265732F54F1
:10B0E000686972645F50617274792F4C7749502F90
:10B0F0007372632F636F72652F7463702E63000029
:10B1000070636220213D204E554C4C0041737365A5
:10B110007274696F6E2022257322206661696C65E6
:10B1200064206174206C696E6520256420696E203E
:10B1300025730A002DE9F05F80460D4691469A4638
:10B140000A9F00BFB8F1000F07D100BF40A3A322A0
:10B150004CA154A0F8F728FD00BF00BF00BF002D90
:10B1600007D100BF3AA3A42258A14EA0F8F71CFDB6
:10B1700000BF00BF07F0010008B1042000E000207C
:10B1800007F0020109B1002100E00021084407F0A6
:10B19000080109B1002100E00021084407F0100176
:10B1A00009B1002100E0002146180320FCF7D0FE81
:10B1B000041E05D12846FEF73FFA0020BDE8F09FA7
:10B1C000A77200202060656000BF2889B04207DABE
:10B1D00000BF1FA3B02246A132A0F8F7E5FC00BFD4
:10B1E00000BF2889801B208114212846FDF710FD0F
:10B1F00020B1204604F0FCFA0020DFE760684068D8
:10B20000E060B8F81600FCF720F9E1680880B8F8AB
:10B210001800FCF71AF9E16848805046FCF708F975
:10B22000E1684860B346F11706EB91718910491D3A
:10B230004FF6FF7202EA013141EA0900FCF705F915
:10B24000E16888810020E16848822046B6E7000076
:10B250002E2E2F4D6964646C6577617265732F546F
:10B26000686972645F50617274792F4C7749502F0E
:10B270007372632F636F72652F7463705F6F757481
:10B280002E6300007463705F6372656174655F7341
:10B2900065676D656E743A20696E76616C696420CD
:10B2A00070636200417373657274696F6E2022254A
:10B2B0007322206661696C6564206174206C696E1C
:10B2C0006520256420696E2025730A007463705F11
:10B2D0006372656174655F7365676D656E743A204E
:10B2E000696E76616C6964207062756600000000AA
:10B2F000702D3E746F745F6C656E203E3D206F70E4
:10B30000746C656E000000002DE9F04106460D46A4
:10B31000174600BF002F08D100BF10A340F6C5029A
:10B320001AA124A0F8F740FC00BF00BF15B93046B1
:10B33000BDE8F081AC8C74B12820844202DD211A72
:10B3400089B200E000218846464501DA314600E036
:10B3500041460E4600BF3046EAE700002E2E2F4D34
:10B360006964646C6577617265732F54686972648F
:10B370005F50617274792F4C7749502F7372632F2D
:10B38000636F72652F7463702E6300007463705F67
:10B390006566665F73656E645F6D73735F6E65741B
:10B3A00069663A20696E76616C6964206473745FC3
:10B3B00069700000417373657274696F6E20222595
:10B3C0007322206661696C6564206174206C696E0B
:10B3D0006520256420696E2025730A002DE9F84355
:10B3E00004460D460027B94600BF05F0030040B9EA
:10B3F00000BF60A340F211426B496CA0F8F7D4FB88
:10B4000000BF00BF00BF002C08D100BF59A340F20D
:10B41000134270A165A0F8F7C7FB00BF00BF05F09D
:10B42000020000B1012707F0010008B1042000E08C
:10B43000002007F0020109B1002100E000210844CA
:10B4400007F0080109B1002100E00021084407F0DD
:10B45000100109B1002100E0002100EB01094FF4C7
:10B46000207249463620FDF751FCB0F1000809D1A1
:10B4700000BF608B40F08000608300BF4FF0FF3062
:10B48000BDE8F88300BFB8F80A00484508DA00BFF5
:10B4900038A340F2394257A144A0F8F785FB00BF1A
:10B4A00000BF00972A4641462046E36DFFF742FE63
:10B4B000061E07D100BF608B40F08000608300BF94
:10B4C000701EDDE700BF307B00F0030040B100BF1D
:10B4D00028A340F2424256A134A0F8F765FB00BF12
:10B4E00000BF00BF308940B100BF22A340F24342F9
:10B4F00055A12EA0F8F758FB00BF00BFE06E08B9B9
:10B50000E66607E0E06E00E0006801680029FBD114
:10B51000066000BF0020A4F8680005F0020010B922
:10B5200005F0010010B1E06D401CE06505F0010080
:10B5300028B100BF608B40F02000608300BF7068BE
:10B54000FDF764FE34F8661F0844208034F866096D
:10B5500070B100BF206F50B9E06E40B900BF05A3C5
:10B5600040F2654243A111A0F8F71EFB00BF00BFE7
:10B57000002085E72E2E2F4D6964646C657761721B
:10B5800065732F54686972645F50617274792F4CCF
:10B590007749502F7372632F636F72652F746370D6
:10B5A0005F6F75742E630000342C0108417373655E
:10B5B0007274696F6E2022257322206661696C6542
:10B5C00064206174206C696E6520256420696E209A
:10B5D00025730A007463705F656E71756575655FCC
:10B5E000666C6167733A20696E76616C696420707D
:10B5F000636200007463705F656E71756575655F89
:10B60000666C6167733A20636865636B2074686178
:10B610007420666972737420706275662063616E4F
:10B6200020686F6C64206F70746C656E00000000A1
:10B630007365672D3E746370686472206E6F74204A
:10B64000616C69676E6564007463705F656E7175C7
:10B650006575655F666C6167733A20696E76616CCB
:10B660006964207365676D656E74206C656E6774C0
:10B67000680000007463705F656E71756575655F65
:10B68000666C6167733A20696E76616C69642071DB
:10B6900075657565206C656E6774680070B52348C4
:10B6A0000078401C2149087000BF2148046839E037
:10B6B000A07F1E490978884233D01C480078A077C3
:10B6C000A07E00F0010078B100BF608B40F0020066
:10B6D000608300BF204601F051FA00BF608B4FF637
:10B6E000FC710840608300BFA07E00F0080048B1F4
:10B6F00000BF608B4FF6F7710840608300BF2046A3
:10B70000FFF7A4FCE568A06F48B100200949087064
:10B71000204602F009FD0748007800B1C5E72C4635
:10B7200000E0E468002CC3D170BD0000420100209D
:10B73000380100204001002010B5044600BF207DE4
:10B74000012807D100BF06A3D42211A115A0F8F744
:10B750002BFA00BF00BF21460120FCF72BFB10BDD8
:10B760002E2E2F4D6964646C6577617265732F545A
:10B77000686972645F50617274792F4C7749502FF9
:10B780007372632F636F72652F7463702E63000092
:10B790007463705F667265653A204C495354454E38
:10B7A00000000000417373657274696F6E2022257A
:10B7B0007322206661696C6564206174206C696E17
:10B7C0006520256420696E2025730A002DE9F04765
:10B7D00005460C469146984635E026462468706832
:10B7E000FDF714FD074600BFB5F86600B84208DA59
:10B7F00000BF22A340F257422DA137A0F8F7D4F999
:10B8000000BF00BF35F8660FC01B288030893C4957
:10B81000098808443A490880304603F0E9FF35F8C2
:10B82000660900280FD000BF002C0BD1B8F1000F23
:10B8300008D100BF11A340F2614232A126A0F8F75F
:10B84000B3F900BF00BFB4B1E1684868FBF7F0FD91
:10B850008246E1688889FBF7F8FD00F0030008B133
:10B86000012000E000202189084450442D49096846
:10B87000401A0028B1DD2046BDE8F0872E2E2F4D5E
:10B880006964646C6577617265732F54686972646A
:10B890005F50617274792F4C7749502F7372632F08
:10B8A000636F72652F7463705F696E2E63000000B2
:10B8B0007063622D3E736E645F71756575656C654E
:10B8C0006E203E3D20706275665F636C656E286E0B
:10B8D0006578742D3E702900417373657274696FC9
:10B8E0006E2022257322206661696C656420617474
:10B8F000206C696E6520256420696E2025730A001E
:10B90000600100207463705F726563656976653AF3
:10B910002076616C6964207175657565206C656E53
:10B92000677468005C01002010B5044600BF207DEC
:10B93000012807D100BF06A3DF2211A117A0F8F745
:10B9400033F900BF00BF21460220FCF733FA10BDD7
:10B950002E2E2F4D6964646C6577617265732F5468
:10B96000686972645F50617274792F4C7749502F07
:10B970007372632F636F72652F7463702E630000A0
:10B980007463705F667265655F6C697374656E3A47
:10B9900020214C495354454E00000000417373650B
:10B9A0007274696F6E2022257322206661696C654E
:10B9B00064206174206C696E6520256420696E20A6
:10B9C00025730A0010B50446606F20B1606F03F064
:10B9D0001CFF0020606710BD0D4801880088401CD6
:10B9E0000B4A10800B48006818B10B480088814250
:10B9F00005DA0A48006800F11402505C70470648F6
:10BA00000078081AC2B203480068805CF6E70000BC
:10BA100054010020500100204E0100204801002068
:10BA200070B50B48046810E0E568A07E00F00800DF
:10BA300048B100BF608B4FF6F7710840608300BFCC
:10BA40002046FFF703FB2C4600BF002CECD170BD55
:10BA50003801002010B5F4F747FCC0F30D0000F5E5
:10BA600040400149088010BD280100202DE9FE4F0B
:10BA700005468B4600BF002D07D100BFE2A38322FD
:10BA8000EEA1F4A0F8F790F800BF00BFFB4968688A
:10BA900008606889142800DAC8E3F94A1168506917
:10BAA000FAF70DFA28B9F648007D00F0F000E0281A
:10BAB00000D1BBE3F14909688889FBF7C6FC001394
:10BAC0008700142F02DB2889B84200DAAEE3A7F121
:10BAD0001400EC4908800020EB4908606889B842EE
:10BAE00008DBE8480088E949088039462846FEF71F
:10BAF00007F84AE000BF286838B900BFC2A3C222D5
:10BB0000E3A1D4A0F8F750F800BF00BF14212846E5
:10BB1000FDF7F6FF6889DD490880DA480088098862
:10BB2000401A1FFA80FAD94801882846FDF7E8FF35
:10BB300028684089504500DA78E328684068D2498F
:10BB4000086051462868FDF7DBFF2889A0EB0A0052
:10BB5000288100BF688938B100BFABA3DF22D0A124
:10BB6000BCA0F8F721F800BF00BF00BF28892968F2
:10BB70000989884207D000BFA3A3E022CBA1B5A0CA
:10BB8000F8F712F800BF00BF00BFBC490968088879
:10BB9000FBF75BFCB94909680880B849096848881F
:10BBA000FBF753FCB54909684880B44909684868FF
:10BBB000FBF73EFCB14909684860C4490860AF49D9
:10BBC00009688868FBF734FCAC4909688860C0499B
:10BBD0000860AA490968C889FBF737FCA7490968C2
:10BBE000C881A64909688889FBF72FFC00F03F004F
:10BBF000B84908702889B8490880B648007800F02C
:10BC0000030040B108460088401C08802889098844
:10BC1000884200DD0AE34FF00009B048046873E091
:10BC200000BF207D38B900BF77A3FB22ACA189A05B
:10BC3000F7F7BAFF00BF00BF00BF207D0A2807D179
:10BC400000BF71A3FC22B0A182A0F7F7ADFF00BF37
:10BC500000BF00BF207D012807D100BF6AA3FD22DD
:10BC6000B4A17CA0F7F7A0FF00BF00BF207A50B1BD
:10BC7000217A8348406890F83000401CC0B281426D
:10BC800001D0A1463FE0208B7C49096809888842A1
:10BC900037D1E08A794909684988884231D17849A1
:10BCA0006068096988422CD17549206849698842D1
:10BCB00027D100BFE068A04208D100BF52A340F2E4
:10BCC0000D12A6A163A0F7F76FFF00BF00BFB9F187
:10BCD000000F07D0E068C9F80C0080480068E060F9
:10BCE0007E48046000BFE068A04208D100BF46A3C0
:10BCF00040F21512A4A157A0F7F756FF00BF00BFEE
:10BD000004E0A14600BFE468002C89D100BF002CEC
:10BD100078D1A848046839E000BF207D0A2808D0FF
:10BD200000BF39A340F21F12A3A14AA0F7F73CFFBE
:10BD300000BF00BF207A48B1217A5148406890F88E
:10BD40003000401CC0B2814200D01EE0208B4B4925
:10BD500009680988884217D1E08A484909684988F2
:10BD6000884211D146496068096988420CD144492A
:10BD700020684969884207D1204604F081FB2846A3
:10BD8000FDF75AFCBDE8FE8F00BFE468002CC3D16C
:10BD9000A146954806681FE0307A50B1317A38489C
:10BDA000406890F83000401CC0B2814201D0B146DA
:10BDB00011E0F08A314909684988884209D130493F
:10BDC00030684969884200D108E00EB1306800B996
:10BDD00004E0B14600BFF668002EDDD100BF8EB191
:10BDE000B9F1000F07D0F068C9F80C007E48006870
:10BDF000F0607D480660304600F04AFC2846FDF7BA
:10BE00001BFCBFE7F2E000002E2E2F4D6964646C2E
:10BE10006577617265732F54686972645F506172EF
:10BE200074792F4C7749502F7372632F636F72654B
:10BE30002F7463705F696E2E630000007463705F1F
:10BE4000696E7075743A20696E76616C69642070F1
:10BE500062756600417373657274696F6E20222586
:10BE60007322206661696C6564206174206C696E60
:10BE70006520256420696E2025730A004801002092
:10BE8000689000204C010020500100204E0100204D
:10BE9000702D3E6E65787420213D204E554C4C002F
:10BEA000702D3E6C656E203D3D203000702D3E743F
:10BEB0006F745F6C656E203D3D20702D3E6E657821
:10BEC000742D3E746F745F6C656E00005801002025
:10BED0005C01002064010020620100203801002084
:10BEE0007463705F696E7075743A2061637469760B
:10BEF00065207063622D3E737461746520213D205E
:10BF0000434C4F53454400007463705F696E707515
:10BF1000743A20616374697665207063622D3E73A4
:10BF20007461746520213D2054494D452D57414988
:10BF3000540000007463705F696E7075743A20611C
:10BF40006374697665207063622D3E7374617465F5
:10BF500020213D204C495354454E00007463705FCE
:10BF6000696E7075743A207063622D3E6E657874E8
:10BF700020213D2070636220286265666F72652013
:10BF800063616368652900007463705F696E707532
:10BF9000743A207063622D3E6E65787420213D20D6
:10BFA00070636220286166746572206361636865EE
:10BFB000290000003C0100207463705F696E707599
:10BFC000743A2054494D452D5741495420706362BD
:10BFD0002D3E7374617465203D3D2054494D452DBF
:10BFE000574149540000000034010020002C73D058
:10BFF00000209149086028890881084645608F48DB
:10C000000068C86000208E4908608E4908708E491B
:10C0100008808E48007800F0080018B1687B40F076
:10C0200001006873A06F80B1204602F07DF80D30EA
:10C0300028B1A06F48B186480088002805DD608DD2
:10C0400010B9204603F0EEFBBCE0824804602046B5
:10C0500001F0C8FC804608F10D00002816D0794890
:10C06000007800F0080090B100BFD4F8900028B12B
:10C070006FF00D01D4F890202069904700BF214651
:10C08000754801F0C3FB2046FFF756FB99E04FF0DF
:10C0900000086D480088002819DD6B48B0F800A042
:10C0A00000BFD4F8800038B152462146D4F8803021
:10C0B00020699847804601E04FF0000800BF08F172
:10C0C0000D0000B97EE000205F49088000BF2046D7
:10C0D00000F0D8F808B175E084E059480068A8B3CA
:10C0E00000BFA06F50B100BFAFF2E4234FF4F37272
:10C0F0005AA1AFF2A020F7F757FD00BF00BFA07E06
:10C1000000F0100038B14E480068FDF795FA20465F
:10C11000FEF7D6FD56E000BFD4F8840048B10023F6
:10C120004749D4F884C020690A682146E047804620
:10C1300007E00023424821460268184602F0CCFE80
:10C14000804600BF08F10D0008B93BE005E0B8F1FA
:10C15000000F02D03A480068A0673A48007800F023
:10C16000200018B3A06F30B1A06F407B40F02000DA
:10C17000A16F48731AE0208DB0F5066F02D0208DB4
:10C18000401C208500BFD4F8840040B100231A462B
:10C190002146D4F884C02069E047804601E04FF092
:10C1A000000800BF08F10D0000B90BE0002029498C
:10C1B0000860204600F066F800B103E0204600F079
:10C1C000DDFC00BF0020234908601D4908601A48B3
:10C1D000406840B318494868FDF72EFA0020164918
:10C1E000486020E0154909688889FBF72EF900F0BE
:10C1F0000400A8B9114800680088104909684988F6
:10C200001D4ACDE9002102901C48006810490988A8
:10C210004218194B1B1D1A480168002003F0FAF957
:10C220002846FDF709FA00BF00BFABE52846FDF739
:10C2300003FA00BFA6E5000060C700204801002007
:10C2400068010020650100206001002064010020D9
:10C25000620100206C010020380100207063622D13
:10C260003E726566757365645F64617461203D3D0F
:10C27000204E554C4C0000007890002058010020C2
:10C280005C01002010B5044600BF002C08D100BF9F
:10C2900013A340F25A221FA128A0F7F785FC00BF84
:10C2A00000BF3048007800F01000B8B1A07E00F068
:10C2B000100050B900BFD4F8900028B16FF00E0103
:10C2C000D4F890202069904700BF2146264801F00D
:10C2D0009DFA2046FFF730FA012010BD0020FCE750
:10C2E0002E2E2F4D6964646C6577617265732F54CF
:10C2F000686972645F50617274792F4C7749502F6E
:10C300007372632F636F72652F7463705F696E2E33
:10C31000630000007463705F696E7075745F6465BC
:10C320006C617965645F636C6F73653A20696E76E2
:10C33000616C696420706362000000004173736582
:10C340007274696F6E2022257322206661696C65A4
:10C3500064206174206C696E6520256420696E20FC
:10C3600025730A0065010020380100202DE9F04105
:10C370000446002600BF002C08D100BF14A340F6DD
:10C38000240220A126A0F7F70FFC00BF00BF216DFB
:10C39000481EFBF74DF880464346002231462046B2
:10C3A00000F09EFD05461DB94FF0FF30BDE8F0815D
:10C3B000334600222946204600F010FF231D224666
:10C3C0002946204600F08CFE07463846EEE700007E
:10C3D0002E2E2F4D6964646C6577617265732F54DE
:10C3E000686972645F50617274792F4C7749502F7D
:10C3F0007372632F636F72652F7463705F6F7574F0
:10C400002E6300007463705F6B656570616C6976A4
:10C41000653A20696E76616C696420706362000021
:10C42000417373657274696F6E20222573222066D2
:10C4300061696C6564206174206C696E6520256497
:10C4400020696E2025730A002DE9F04107467F2FF1
:10C4500001DD7F2000E0384606460EB9BDE8F081D8
:10C46000701EC6B24FF0000800250F48046813E0A4
:10C47000607DB04208DB607DB0420CD10B49206A80
:10C480000968081A404506D30849206A0968A1EBE3
:10C4900000082546667DE468002CE9D115B12846E0
:10C4A000FEF70EFC00BFD9E7380100202C01002068
:10C4B0002DE9F041054600BF082D0AD0092D08D00E
:10C4C00000BF13A340F2DD621DA121A0F7F76CFBB2
:10C4D00000BF00BF00270026274804680EE0207D2B
:10C4E000A8420AD12549206A0968081AB84204D32B
:10C4F0002249206A09680F1A2646E468002CEED10A
:10C500001EB100213046FEF7F1FABDE8F0810000CF
:10C510002E2E2F4D6964646C6577617265732F549C
:10C52000686972645F50617274792F4C7749502F3B
:10C530007372632F636F72652F7463702E630000D4
:10C54000696E76616C6964207374617465000000C3
:10C55000417373657274696F6E20222573222066A1
:10C5600061696C6564206174206C696E6520256466
:10C5700020696E2025730A00380100202C0100205C
:10C5800070B5002600250B4804680BE00A49206AB4
:10C590000968081AB04204D30749206A09680E1ACC
:10C5A0002546E468002CF1D115B12846FEF788FB3A
:10C5B00070BD00003C0100202C01002070B5044635
:10C5C00000BF44B900BF12A340F211121CA11FA06A
:10C5D000F7F7EAFA00BF00BF00BF207D012808D0AE
:10C5E00000BF0BA34FF4897222A118A0F7F7DCFA61
:10C5F00000BF00BF012507E0244951F82510086855
:10C60000214602F059FD6D1C042DF5D370BD0000CC
:10C610002E2E2F4D6964646C6577617265732F549B
:10C62000686972645F50617274792F4C7749502F3A
:10C630007372632F636F72652F7463702E630000D3
:10C6400070636220213D204E554C4C004173736550
:10C650007274696F6E2022257322206661696C6591
:10C6600064206174206C696E6520256420696E20E9
:10C6700025730A007063622D3E7374617465203DFA
:10C680003D204C495354454E00000000E82A010863
:10C690002DE9FE4305465448007800F0040008B137
:10C6A000BDE8FE8300BF002D08D100BF4FA340F2BC
:10C6B00081225BA162A0F7F777FA00BF00BF4A486A
:10C6C000007800F01000B0B1674800680088664943
:10C6D00009684988654ACDE90021029064480068EC
:10C6E000644909884218614B1B1D6348016828464C
:10C6F00002F090FF75E03C48007800F0020000284E
:10C700006FD0687DFEF7E4FA044674B900BFA869EB
:10C7100038B14FF0FF320021AB6928699847804655
:10C7200001E06FF00F0800BFBAE7504810384069C9
:10C7300020604E48103800696060E88AE0824A480C
:10C740000068008820830320207549480068401C49
:10C750006062606AE062204600F022F90646A66543
:10C7600026656664E66542480068401E6065286983
:10C770002061E567687A00F00C006072287A207208
:10C7800000BF00BF3D480068E0603C48046003F023
:10C790005BFE00BF01203A49087000BF204600F050
:10C7A0002FFF31480068C08924F8600F208860801E
:10C7B000603C201DFAF760F88046608E221D4146DD
:10C7C000FEF7A2FD608612212046FEF707FE07460F
:10C7D00027B100212046FEF789F961E7204600F0E5
:10C7E000CDF900BF5CE70000640100202E2E2F4D24
:10C7F0006964646C6577617265732F5468697264EB
:10C800005F50617274792F4C7749502F7372632F88
:10C81000636F72652F7463705F696E2E6300000032
:10C820007463705F6C697374656E5F696E70757444
:10C830003A20696E76616C69642070636200000062
:10C84000417373657274696F6E20222573222066AE
:10C8500061696C6564206174206C696E6520256473
:10C8600020696E2025730A0048010020789000207E
:10C8700058010020620100205C01002038010020E6
:10C880004001002070B506460D46D6B13068C0B1F3
:10C890000C480168304600F01BF80B480168304630
:10C8A00000F016F86DB1286858B10848046806E031
:10C8B00020683168884201D128682060E468002C33
:10C8C000F6D170BD38010020300100203401002075
:10C8D0002DE9F04105460E46344600BF002D08D133
:10C8E00000BF0CA34FF4106216A123A0F7F75CF968
:10C8F00000BF00BF0AE020682968884205D1E768C8
:10C900002046FEF7DDF93C4600E0E468002CF2D159
:10C91000BDE8F0812E2E2F4D6964646C65776172DD
:10C9200065732F54686972645F50617274792F4C1B
:10C930007749502F7372632F636F72652F74637022
:10C940002E6300007463705F6E657469665F697062
:10C950005F616464725F6368616E6765645F706382
:10C96000626C6973743A20696E76616C6964206FD9
:10C970006C645F6164647200417373657274696FA3
:10C980006E2022257322206661696C6564206174C3
:10C99000206C696E6520256420696E2025730A006D
:10C9A00010B5044600BF002C08D100BF09A340F613
:10C9B000AF0214A11AA0F7F7F7F800BF00BF224892
:10C9C00000682249096808441F4908600846006851
:10C9D00010BD00002E2E2F4D6964646C6577617266
:10C9E00065732F54686972645F50617274792F4C5B
:10C9F0007749502F7372632F636F72652F74637062
:10CA00002E6300007463705F6E6578745F69737382
:10CA10003A20696E76616C69642070636200000080
:10CA2000417373657274696F6E20222573222066CC
:10CA300061696C6564206174206C696E6520256491
:10CA400020696E2025730A00440100202C0100207B
:10CA500070B505460C4600BF002D08D100BF25A3C8
:10CA600040F21F4230A13AA0F7F79EF800BF00BF86
:10CA7000E9688889FAF7E9FC00F0010020B1204656
:10CA800002F0C3FE002433E013E0E1688889FAF77E
:10CA9000DCFC00F0010038B10120FAF7D6FCE968AF
:10CAA00089890843E968888126462468304602F06F
:10CAB0009FFE4CB1E06840682189084429892E4ACC
:10CAC00012681144081AE0D594B128892A490968E6
:10CAD0000844E1684968401A002809DDE068808858
:10CAE00025490988401A288129896868FCF700FFD0
:10CAF0002C6070BD2E2E2F4D6964646C6577617259
:10CB000065732F54686972645F50617274792F4C39
:10CB10007749502F7372632F636F72652F74637040
:10CB20005F696E2E630000007463705F6F6F735FE8
:10CB3000696E736572745F7365676D656E743A20B4
:10CB4000696E76616C69642063736567000000003C
:10CB5000417373657274696F6E202225732220669B
:10CB600061696C6564206174206C696E6520256460
:10CB700020696E2025730A00580100202DE9F84F26
:10CB8000044600BF002C08D100BFA7A340F2E14239
:10CB9000B2A1B8A0F7F708F800BF00BF00BF207D22
:10CBA000012808D100BFA0A340F2E342BBA1B1A07D
:10CBB000F6F7FAFF00BF00BFC2480068A04202D1EA
:10CBC0000020BDE8F88FB4F86000B4F8481088423F
:10CBD00002DAB4F8600001E0B4F848008146E56E7E
:10CBE00045B9A07E00F0020018B1204602F01AFEFE
:10CBF000E7E710E1221D2146204602F0FBFC074634
:10CC000017B96FF00300DCE70CB1206858B90FB119
:10CC1000381D00E00020014611B96FF00300D0E795
:10CC20000868206000BFE9684868FAF701FC616C99
:10CC3000401A29890844484519D9B4F86000484584
:10CC40000CD1206F50B994F8990038B9002004F83D
:10CC5000980F012060700020A070983CA07E00F02A
:10CC6000020018B1204602F0DDFDAAE7D3E0002063
:10CC700084F89900266F26B100E0366830680028F5
:10CC8000FBD1B5E000BFE9688889FAF7DEFB00F068
:10CC9000040040B100BF64A340F236528AA175A0DF
:10CCA000F6F782FF00BF00BF206FA0B1A07E00F0AA
:10CCB000440080B9E06E38B1E06E006858B9E06EAB
:10CCC0000089618E884206DAB4F8640018B1B4F8BD
:10CCD0006600092801DB012000E0002020B9A07EC9
:10CCE00000F0A00000B98FE0207D022807D01020BE
:10CCF000FAF7ABFBE96889890843E96888813A4615
:10CD00002146284600F0FCFA0090009838B100BF98
:10CD1000608B40F08000608300BF009851E7286876
:10CD2000E066207D022806D000BF608B4FF6FC71C4
:10CD30000840608300BFE9684868FAF779FB8046DD
:10CD4000E9688889FAF781FB00F0030008B1012047
:10CD500000E000202989084408EB000A206DB0EBB0
:10CD60000A0001D5C4F850A0E9688889FAF76DFB7C
:10CD700000F0030008B1012000E0002029890844E8
:10CD800088B300202860206F10B925672E462EE05A
:10CD9000E9684868FAF74CFB8046F1684868FAF79A
:10CDA00047FBB8EB00001BD504F1700801E0D8F890
:10CDB0000080D8F8000068B1D8F80010C968486849
:10CDC000FAF736FB8346E9684868FAF731FBBBEBB4
:10CDD0000000ECD4D8F800002860C8F8005006E045
:10CDE0003560366803E0FFE7284602F001FDE56E96
:10CDF00055B1E9684868FAF71BFB616C401A29894C
:10CE0000084448457FF63EAF00BFE06E10B90020F1
:10CE1000A4F8680000BF00BF608B4FF67F71084028
:10CE2000608300BF0020CCE62E2E2F4D6964646C19
:10CE30006577617265732F54686972645F506172BF
:10CE400074792F4C7749502F7372632F636F72651B
:10CE50002F7463705F6F75742E6300007463705F6E
:10CE60006F75747075743A20696E76616C696420B0
:10CE700070636200417373657274696F6E2022255E
:10CE80007322206661696C6564206174206C696E30
:10CE90006520256420696E2025730A00646F6E2763
:10CEA000742063616C6C207463705F6F757470754F
:10CEB0007420666F72206C697374656E2D70636286
:10CEC000730000006C010020525354206E6F7420D8
:10CED000657870656374656420686572652100001B
:10CEE0002DE9FF4104460E461746984600BF002C28
:10CEF00008D100BF10A340F242721CA125A0F6F792
:10CF000053FE00BF00BF608D1023218BE28ACDE964
:10CF100001130092039043463A463146606A00F09E
:10CF20004DF805461DB1618D606A0844E0622846EF
:10CF300004B0BDE8F08100002E2E2F4D6964646CB2
:10CF40006577617265732F54686972645F506172AE
:10CF500074792F4C7749502F7372632F636F72650A
:10CF60002F7463705F6F75742E6300007463705F5D
:10CF70006F75747075745F616C6C6F635F68656109
:10CF80006465723A20696E76616C696420706362D0
:10CF900000000000417373657274696F6E20222572
:10CFA0007322206661696C6564206174206C696E0F
:10CFB0006520256420696E2025730A002DE9F05F45
:10CFC00082460D4617469846DDF830B005F114004C
:10CFD000384481B24FF420722220FBF797FE0646B8
:10CFE000002E34D000BF718905F11400814208DAA7
:10CFF00000BF18A340F2237223A12FA0F6F7D4FD9F
:10D0000000BF00BF74680A98FAF71FFA20800B98D7
:10D01000FAF71BFA6080C4F804805046FAF708FA61
:10D02000A060A946E91705EB91718910491D4FF6DB
:10D03000FF7202EA013141EA0B00FAF706FAA08119
:10D040000D98FAF702FAE0810020208260823046D3
:10D05000BDE8F09F2E2E2F4D6964646C6577617278
:10D0600065732F54686972645F50617274792F4CD4
:10D070007749502F7372632F636F72652F746370DB
:10D080005F6F75742E630000636865636B2074685E
:10D0900061742066697273742070627566206361C2
:10D0A0006E20686F6C64207374727563742074638F
:10D0B000705F686472000000417373657274696F19
:10D0C0006E2022257322206661696C65642061747C
:10D0D000206C696E6520256420696E2025730A0026
:10D0E0002DE9FE4F04460E4692469B4600BF002E99
:10D0F00008D100BF17A340F2877223A12DA0F6F735
:10D1000053FD00BF00BF5A465146204602F072FA56
:10D11000054615B96FF0030715E024B194F80B80AC
:10D1200094F80A9003E04FF0FF084FF00009062042
:10D1300043465A465146CDE9009002953046F9F7EC
:10D1400033F9074600BF3046FCF776FA3846BDE8AB
:10D15000FE8F00002E2E2F4D6964646C657761721E
:10D1600065732F54686972645F50617274792F4CD3
:10D170007749502F7372632F636F72652F746370DA
:10D180005F6F75742E6300007463705F6F757470E9
:10D1900075745F636F6E74726F6C5F7365676D65D6
:10D1A0006E743A20696E76616C696420706275668F
:10D1B00000000000417373657274696F6E20222550
:10D1C0007322206661696C6564206174206C696EED
:10D1D0006520256420696E2025730A002DE9F0473B
:10D1E00081460D4614469A464FF0000800BF002DB8
:10D1F00008D100BF1CA340F2567228A131A0F6F757
:10D20000D3FC00BF00BF6E6806F1140700BF3846AC
:10D2100000EB880004F0010109B1042100E00021C5
:10D22000084404F0020109B1002100E00021084493
:10D2300004F0080109B1002100E00021084404F0D5
:10D24000100109B1002100E000210844B84208D0D3
:10D2500000BF05A340F2757224A11AA0F6F7A4FC42
:10D2600000BF00BFBDE8F0872E2E2F4D6964646CAF
:10D270006577617265732F54686972645F5061727B
:10D2800074792F4C7749502F7372632F636F7265D7
:10D290002F7463705F6F75742E6300007463705F2A
:10D2A0006F75747075745F66696C6C5F6F707469AC
:10D2B0006F6E733A20696E76616C69642070627576
:10D2C00066000000417373657274696F6E202225D9
:10D2D0007322206661696C6564206174206C696EDC
:10D2E0006520256420696E2025730A006F707469BB
:10D2F0006F6E73206E6F742066696C6C65640000DD
:10D300002DE9FE4F04460D46164600BF002C08D1FD
:10D3100000BF58A34FF4B76263A16BA0F6F744FCBB
:10D3200000BF00BF00BF002D08D100BF51A340F2D5
:10D33000B9526FA164A0F6F737FC00BF00BF00BF71
:10D34000002E08D100BF4BA340F2BA5270A15EA0DC
:10D35000F6F72AFC00BF00BF204600F0F7F810B136
:10D360000020BDE8FE8F686AFAF762F8E16888601D
:10D37000688DFAF76AF8E168C881698D686A0844BF
:10D38000E862E06800F11407A07A00F0010068B1DB
:10D390002A1D31464FF40670FDF7B6FF82464AF06B
:10D3A0000170FAF745F838603F1D00BFB5F930004D
:10D3B000002801DA00202886686B38B95D480068CB
:10D3C0006863E1684868FAF733F8A863A089616880
:10D3D0008988401A1FFA80F860684089A0EB08002D
:10D3E0006168488160680089A0EB08006168088175
:10D3F0006168E06848600020E168088200BFE0687A
:10D400001430A17A01F0010109B1042100E00021EA
:10D410000844A17A01F0020109B1002100E00021D5
:10D420000844A17A01F0080109B1002100E00021BF
:10D430000844A17A01F0100109B1002100E00021A7
:10D440000844B84208D000BF0AA340F21C623AA1C7
:10D450001DA0F6F7A9FB00BF00BF0621A87A8DE842
:10D460004300EB7A2A1D29466068F8F79DFF814644
:10D47000484676E72E2E2F4D6964646C657761729D
:10D4800065732F54686972645F50617274792F4CB0
:10D490007749502F7372632F636F72652F746370B7
:10D4A0005F6F75742E6300007463705F6F757470C6
:10D4B00075745F7365676D656E743A20696E766129
:10D4C0006C69642073656700417373657274696F7A
:10D4D0006E2022257322206661696C656420617468
:10D4E000206C696E6520256420696E2025730A0012
:10D4F0007463705F6F75747075745F7365676D6565
:10D500006E743A20696E76616C69642070636200A3
:10D510007463705F6F75747075745F7365676D6544
:10D520006E743A20696E76616C6964206E65746908
:10D53000660000002C0100206F7074696F6E73200C
:10D540006E6F742066696C6C6564000010B50446EB
:10D5500000BF002C08D100BF08A340F29A5214A1CA
:10D560001DA0F6F721FB00BF00BF6068807B01288B
:10D5700001D0012010BD0020FCE700002E2E2F4D11
:10D580006964646C6577617265732F54686972644D
:10D590005F50617274792F4C7749502F7372632FEB
:10D5A000636F72652F7463705F6F75742E63000014
:10D5B0007463705F6F75747075745F7365676D65A4
:10D5C0006E745F627573793A20696E76616C696416
:10D5D0002073656700000000417373657274696FA2
:10D5E0006E2022257322206661696C656420617457
:10D5F000206C696E6520256420696E2025730A0001
:10D600002DE9F041054600BF002D08D100BF28A339
:10D6100040F27D7233A13AA0F6F7C6FA00BF00BF10
:10D6200041480088002840D000204049088036E06A
:10D63000FEF7D2F9074627B1012F04D0022F1FD1E0
:10D6400002E0BDE8F08128E0FEF7C6F9042806D123
:10D6500036480088801C34490988884200DDF0E79C
:10D66000FEF7BAF90602FEF7B7F90643B6F5067FEC
:10D6700000DC16B94FF4067000E0304668860CE016
:10D68000FEF7AAF90446022C00DADAE7A01E2749C1
:10D69000098808442549088000BF00BF00BF23480F
:10D6A0000088214909888842C2DB00BFC9E7000021
:10D6B0002E2E2F4D6964646C6577617265732F54EB
:10D6C000686972645F50617274792F4C7749502F8A
:10D6D0007372632F636F72652F7463705F696E2E50
:10D6E000630000007463705F70617273656F7074C3
:10D6F0003A20696E76616C69642070636200000094
:10D70000417373657274696F6E20222573222066DF
:10D7100061696C6564206174206C696E65202564A4
:10D7200020696E2025730A004C010020540100205E
:10D7300010B5044600BF002C09D100BF16A340F667
:10D74000510221A127A0F6F72FFA00BF10BD00BF9C
:10D75000207DF8B1207D0A281CD0207D012819D019
:10D76000A06F20B1A06FFBF767FF0020A067606F7C
:10D7700010B12046FEF726F94FF0FF302086E06E0C
:10D7800002F043F8206F02F040F80020E0662067C6
:10D79000A4F8680000BFD9E72E2E2F4D6964646C91
:10D7A0006577617265732F54686972645F50617246
:10D7B00074792F4C7749502F7372632F636F7265A2
:10D7C0002F7463702E6300007463705F7063625F18
:10D7D00070757267653A20696E76616C6964207055
:10D7E00063620000417373657274696F6E20222555
:10D7F0007322206661696C6564206174206C696EB7
:10D800006520256420696E2025730A0070B50546E1
:10D810000C4600BF002C08D100BF3AA340F683029B
:10D8200044A14BA0F6F7C0F900BF00BF00BF002D18
:10D8300008D100BF33A340F684024FA144A0F6F7FD
:10D84000B3F900BF00BF00BF2868A04203D1286819
:10D85000C06828600CE0286806E0C168A14202D1D7
:10D86000E168C16002E0C0680028F6D100BF00BFD7
:10D870000020E06000BF2046FFF75AFF207D0A2805
:10D880000FD0207D01280CD0A07E00F0010040B117
:10D8900000BF608B40F00200608300BF2046FFF7AE
:10D8A0006DF9207D012826D000BFE06E40B100BF99
:10D8B00014A340F6930238A125A0F6F775F900BF2E
:10D8C00000BF00BF206F40B100BF0EA340F694021E
:10D8D00037A11FA0F6F768F900BF00BF00BF606F57
:10D8E00040B100BF07A340F6960238A118A0F6F792
:10D8F0005BF900BF00BF00202075E08200BF00BFC1
:10D9000070BD00002E2E2F4D6964646C65776172C6
:10D9100065732F54686972645F50617274792F4C1B
:10D920007749502F7372632F636F72652F74637022
:10D930002E6300007463705F7063625F72656D6F69
:10D9400076653A20696E76616C6964207063620066
:10D95000417373657274696F6E202225732220668D
:10D9600061696C6564206174206C696E6520256452
:10D9700020696E2025730A007463705F7063625FB4
:10D9800072656D6F76653A20696E76616C696420A8
:10D990007063626C69737400756E73656E74207366
:10D9A00065676D656E7473206C65616B696E670089
:10D9B000756E61636B6564207365676D656E747306
:10D9C000206C65616B696E67000000006F6F7365A6
:10D9D00071207365676D656E7473206C65616B692A
:10D9E0006E6700002DE9FE4304460027002600BFB5
:10D9F000002C08D100BFE5A34FF44772F0A1F7A0B7
:10DA0000F6F7D2F800BF00BFFE48007800F004002F
:10DA1000002845D0207D022806D1FB49206D0968E9
:10DA200088421BD1012719E0F849606A09688842D9
:10DA300001D1012712E0F549606A0968081A0DD47E
:10DA4000218D606A0844F1490968081A002805DC3C
:10DA500000BF608B40F00200608300BF002F1DD02C
:10DA600000BF207D40B900BFC8A34FF44E72E8A1AB
:10DA7000DAA0F6F799F800BF00BFED48007840F053
:10DA80000800EB49087000BF608B4FF6FE7108403C
:10DA9000608300BF6FF00D00BDE8FE830020FBE750
:10DAA000D848007800F0020068B1207D02280AD032
:10DAB000207D032807D000BF608B40F00200608308
:10DAC00000BF0020E8E7A07E00F0100010B9D948A0
:10DAD00000682062002084F89B0084F89A002046A9
:10DAE000FFF78EFD207D801E082875D2DFE800F04C
:10DAF00004CDF4F3F2F1F0EFC248007800F010002A
:10DB000000286AD0BF48007800F002000028F8D052
:10DB1000606C401CBC49096888425ED1BB48006803
:10DB2000401C6062606AE062B74800686064C24896
:10DB30000068C089A4F86000B4F86000A4F862002E
:10DB4000B2480068401E606504202075201DF8F76B
:10DB500093FE8046608E221D4146FDF7D5FB608610
:10DB6000608E8100400041F21C12904202D9608E0A
:10DB7000400001E041F21C10814202D2608E800020
:10DB80000AE0608E400041F21C11884202D9608E8A
:10DB9000400001E041F21C10A4F8480000BFB4F8B6
:10DBA0006600002808DC00BF78A34FF45B72A3A1D5
:10DBB0008AA0F5F7F9FF00BF00BFB4F86600401E69
:10DBC000A4F86600256F95B9E56E00BF5DB900BF8A
:10DBD0006EA34FF45D7201E08DE231E09DA17FA064
:10DBE000F5F7E2FF00BF00BF2868E06601E02868A3
:10DBF0002067284601F0FCFD206F18B94FF0FF3078
:10DC0000208603E00020208684F8420000BFD4F87C
:10DC1000880038B100222146D4F88830206998471E
:10DC2000064600E0002600BF06F10D0010B96FF0B7
:10DC30000C0031E700BF608B40F00200608323E0FE
:10DC40007048007800F01000F0B17B480068008850
:10DC5000794909684988844ACDE9002102906B48D6
:10DC600000688249098842187F4B1B1D664801687D
:10DC7000204601F0CFFC94F84200062804DA002088
:10DC80002086204601F07AFB36E25E48007800F0FC
:10DC90001000002876D0606C401C5B490968081AA7
:10DCA00071D45949206D0968081A00286BDC0420DA
:10DCB0002075E06F10B96FF0050623E000BFE06F3C
:10DCC000806978B900BF31A34FF46A7205E0FCE1C6
:10DCD000BCE107E17CE117E105E165A13FA0F5F7B3
:10DCE00063FF00BF00BF00BFE06F806938B1E16F24
:10DCF000206900228B6921469847064601E06FF0B3
:10DD00000F0600BF46B106F10D0010B12046FCF72A
:10DD1000D7FF6FF00C00BFE6204600F09FFA5C488A
:10DD2000008820B15A480088401E59490880608EFA
:10DD30008100400041F21C12904202D9608E4000E6
:10DD400001E041F21C10814202D2608E80000AE0A4
:10DD5000608E400041F21C11884202D9608E400062
:10DD600001E041F21C10A4F848003148007800F0AE
:10DD7000200048B100BF608B40F00200608300BF0C
:10DD8000072087E09FE087E0ABE000002E2E2F4DBC
:10DD90006964646C6577617265732F546869726435
:10DDA0005F50617274792F4C7749502F7372632FD3
:10DDB000636F72652F7463705F696E2E630000007D
:10DDC0007463705F70726F636573733A20696E7607
:10DDD000616C6964207063620000000041737365C8
:10DDE0007274696F6E2022257322206661696C65EA
:10DDF00064206174206C696E6520256420696E2042
:10DE000025730A00640100205C01002058010020F5
:10DE10007463705F696E7075743A207063622D3E32
:10DE2000737461746520213D20434C4F5345440079
:10DE3000650100202C010020480100207063622D44
:10DE40003E736E645F71756575656C656E203E200E
:10DE5000300000006E6F207365676D656E7420740E
:10DE60006F206672656500007890002062010020D6
:10DE70007063622D3E6C697374656E65722D3E61D0
:10DE8000636365707420213D204E554C4C000000AA
:10DE900060010020207524E09948006801889848B6
:10DEA00000684088974ACDE90020029196480068B2
:10DEB000964909884218934B1B1D954801682046D6
:10DEC00001F0A8FB0DE09348007800F0020040B19B
:10DED000606A401E8C490968884202D1204601F0E0
:10DEE00045F909E100BF204600F0B8F98A480078FA
:10DEF00000F0200038B100BF608B40F0020060836A
:10DF000000BF07202075F7E0204600F0A7F98248FF
:10DF1000007800F02000E8B37E48007800F01000A0
:10DF2000C8B37B49206D0968884239D1E06E90BB47
:10DF300000BF608B40F00200608300BF2046FFF707
:10DF4000F7FB00BF00BF75480068A04205D17348C9
:10DF50000068C068714908600DE07049086806E013
:10DF6000C168A14202D1E168C16002E0C068002836
:10DF7000F6D100BF00BF0020E06000BF012068496B
:10DF8000087000BF0A20207500BF66480068E06086
:10DF9000644801E00DE003E0046002F055FA16E089
:10DFA00000BF608B40F00200608300BF0820207536
:10DFB0000DE05848007800F0100040B15449206D41
:10DFC0000968884203D1E06E08B90620207593E005
:10DFD000204600F043F95048007800F02000A0B33C
:10DFE00000BF608B40F00200608300BF2046FFF757
:10DFF0009FFB00BF00BF49480068A04205D14748C9
:10E000000068C068454908600DE04449086806E0BA
:10E01000C168A14202D1E168C16002E0C068002885
:10E02000F6D100BF00BF0020E06000BF01203C49E6
:10E03000087000BF0A20207500BF3A480068E06001
:10E040003848046002F000FA00BF55E0204600F0B6
:10E0500005F93048007800F01000A8B32C49206D75
:10E060000968884230D1E06E70BB2046FFF760FB44
:10E0700000BF00BF29480068A04205D127480068BA
:10E08000C068264908600DE02449086806E0C168B8
:10E09000A14202D1E168C16002E0C0680028F6D167
:10E0A00000BF00BF0020E06000BF01201C490870D5
:10E0B00000BF0A20207500BF1A480068E0601948B8
:10E0C000046002F0C1F900BF16E0204600F0C6F877
:10E0D0001048007800F0100060B10D49206D09680B
:10E0E000884207D1E06E28B90B48007840F0100054
:10E0F0000949087000E000BF00BF0020CCE4000028
:10E100004801002078900020580100206201002082
:10E110005C0100206401002065010020380100201E
:10E12000400100203C0100202DE9F041044600BFE1
:10E13000002C0CD100BF29A340F2096233A13DA0FD
:10E14000F5F732FD00BF6FF00F00BDE8F08100BFB2
:10E15000A06F477BA66F0020A06700BFD4F88400A3
:10E1600040B1002332462146D4F884C02069E047FC
:10E17000054606E0002332462146184600F0ACFE74
:10E18000054600BFF5B907F0200028B3208DB0F593
:10E19000066F02D0208D401C208500BFD4F884007B
:10E1A00040B100231A462146D4F884C02069E047D4
:10E1B000054600E0002500BF05F10D0060B96FF0D5
:10E1C0000C00C2E705F10D0010B96FF00C00BCE7C0
:10E1D000A6676FF00400B8E70020B6E72E2E2F4D9B
:10E1E0006964646C6577617265732F5468697264E1
:10E1F0005F50617274792F4C7749502F7372632F7F
:10E20000636F72652F7463702E6300007463705FB8
:10E2100070726F636573735F726566757365645F53
:10E22000646174613A20696E76616C696420706320
:10E2300062000000417373657274696F6E2022255D
:10E240007322206661696C6564206174206C696E5C
:10E250006520256420696E2025730A002DE9F05F92
:10E2600004464FF0000900BF002C08D100BFE5A311
:10E2700040F27B42F0A1F7A0F5F796FC00BF00BF8B
:10E2800000BF207D042808DA00BFDEA340F27C42F4
:10E29000FAA1F0A0F5F788FC00BF00BFFE480078A7
:10E2A00000F01000002870D0B4F86000A16D00EB01
:10E2B0000108FA49606D0968401A15D4F749606D84
:10E2C0000968884204D1F649A06D0968401A0BD448
:10E2D000F349A06D096888421AD1F2480068C089E4
:10E2E000B4F86010884213D9EE480068C08924F859
:10E2F000600F608834F86019884203DAB4F860006F
:10E30000A4F86200E54800686065E5480068A0651B
:10E31000E349606C0968081A00284ADCE248008872
:10E3200090BBB4F86010A06D084440453AD1B4F9F0
:10E330003000002836DBDA49606C0968884231D148
:10E340004FF0010994F84300401CC0B294F8431008
:10E35000884204DD94F84300401C84F8430094F89C
:10E360004300032817DD00BFB4F84800618E08445D
:10E3700080B2B4F84810884208DBB4F84800618ED7
:10E380000844A4F8480005E00CE02AE14FF6FF70CD
:10E39000A4F8480000BF94F84300032802DB20469D
:10E3A00000F066FFB9F1000F02D1002084F84300AD
:10E3B000EBE0606C401CBA490968081A7ED4B84981
:10E3C000206D0968081A002878DCA07E00F004009F
:10E3D00060B100BF608B4FF6FB710840608300BFE7
:10E3E00048346088208000206084483C0020243429
:10E3F000A077608BB4F9181000EBE10000B2A083A5
:10E40000208CA7490988081A85B20020E077A44823
:10E410000068206214F8100C243C042865DBB4F872
:10E420004800B4F84A10884227DA628B02F400628E
:10E430000AB1012200E002221146628E4A4392B2E2
:10E44000AA4201DD2A4602E0628E4A4392B2104699
:10E4500000BFB4F84820024492B2B4F848309A425F
:10E4600005DBB4F848200244A4F8482003E04FF646
:10E47000FF72A4F8482000BF37E000BFB4F86A007C
:10E48000284480B2B4F86A10884205DBB4F86A0008
:10E490002844A4F86A0003E04FF6FF70A4F86A006D
:10E4A00000BFB4F86A00B4F8481088421DDB483455
:10E4B000608C2188401A6084483C00E062E000BF24
:10E4C000B4F84800618E084480B2B4F8481088421D
:10E4D00006DBB4F84800618E0844A4F8480003E065
:10E4E0004FF6FF70A4F8480000BF70A22046D4E9A0
:10E4F0001B31FDF76BF920676EA22046D4E91B1390
:10E50000FDF764F9E066206F18B94FF0FF30208600
:10E5100001E00020208600202077E06E10B9002066
:10E52000A4F86800B4F86400644909880844A4F8B1
:10E530006400608B00F4006018B3206F88B9E06E4F
:10E5400040B1E16EC9684868F8F772FFE16C081ADB
:10E55000002816DC00BF608B4FF2FF71084060831B
:10E560000FE0216FC9684868F8F762FFE16C081A8C
:10E57000002806DC00BF608B4FF2FF71084060830B
:10E5800000BF02E0204601F04DF9606B48B34449FA
:10E59000A06B0968401A24D5A08E49490988081A39
:10E5A00007B2B4F93C00A7EBE00007B2A08F3844F3
:10E5B00000B2A087002F01DA784207B2B4F93E001A
:10E5C000A7EBA00007B2E08F384400B2E087E08FED
:10E5D000B4F93C1000EBE10000B2A4F840000020C8
:10E5E00060633148008800286CDD207D072869DAE7
:10E5F0002A48616A0068401C081A7CD42748616A6E
:10E60000006860E02E2E2F4D6964646C657761723E
:10E6100065732F54686972645F50617274792F4C0E
:10E620007749502F7372632F636F72652F74637015
:10E630005F696E2E630000007463705F72656365CE
:10E640006976653A20696E76616C696420706362F0
:10E6500000000000417373657274696F6E2022259B
:10E660007322206661696C6564206174206C696E38
:10E670006520256420696E2025730A007463705F2D
:10E68000726563656976653A2077726F6E6720738D
:10E6900074617465000000006401002058010020CE
:10E6A0005C0100204801002062010020756E61635A
:10E6B0006B656400756E73656E7400006001002008
:10E6C0002C010020D4E3F74A12881044401E081A97
:10E6D00000285FDCF4484668F449606A0968A0EBEA
:10E6E000010A00BFF048406860B900BFAFF2EC0318
:10E6F00040F2945200E04DE0EDA1AFF2A800F5F732
:10E7000053FA00BF00BF00BF4FF6FF7082450AD327
:10E7100000BFAFF2101340F29552E9A1AFF2CC0066
:10E72000F5F742FA00BF00BF1FFA8AF500BFDE48C6
:10E7300040680089A8420ADA00BFAFF2381340F2FD
:10E740009752E3A1AFF2F400F5F72EFA00BF00BF35
:10E75000D5480089401BD449088108464068008993
:10E76000401B1FFA80FB07E07089281A85B2A6F8C3
:10E7700008B00020708136687089A842F4DB294611
:10E780003046FBF7BDF9C949606A0860C649C968E7
:10E7900048600AE0C549606A0968081A05D500BFE3
:10E7A000608B40F00200608300BFC049606A096866
:10E7B000081A7DD4218D606A0844401EBB4909684F
:10E7C000081A002874DCB949606A0968884270D167
:10E7D000B549C9688889F8F738FE00F0030008B128
:10E7E000012000E00020B04909890844AD490880B3
:10E7F000208D0988884256DAAB49C9688889F8F7BC
:10E8000024FE00F0010098B1A749C9688889F8F78B
:10E810001CFE00F03E052846F8F717FEA249C9681D
:10E8200089894CF2FF02114008439F49C9688881D9
:10E83000208D9D490881C9688889F8F706FE00F097
:10E84000020020B198480089401E97490881964AE5
:10E8500011895068FBF74CF89349C9688889F8F723
:10E86000F4FD00F0030008B1012000E000208E4913
:10E87000098908448B49088000BF218D606A0844DB
:10E880008A490968874A1288114488420AD000BF21
:10E89000AFF2902340F2CB5291A1AFF24820F5F7AE
:10E8A00083F900BF00BF606F002816D07E4901E0E9
:10E8B000DAE2D3E1C9688889F8F7C7FD00F0010002
:10E8C00060B107E0656F606F00686067284600F020
:10E8D0008FFF00BF606F0028F4D187E0656F2EE0E6
:10E8E000E9688889F8F7B1FD00F0010008B36E49C6
:10E8F000C9688889F8F7A9FD00F00200C8B90120AD
:10E90000F8F7A3FD6849C968898908436649C96859
:10E9100088816549C9688889F8F797FD00F0030088
:10E9200008B1012000E000205F49098908445D49E1
:10E9300008802E462D68304600F05AFF00BF55B1C2
:10E94000E86840682989084458490968554A128886
:10E950001144081AC4D5002D46D0544800685149C6
:10E9600009880844E9684968401A00283CDDE868DD
:10E9700080884E490988401A4B490881C9688889AE
:10E98000F8F763FD00F0020020B147480089401EFF
:10E9900045490881444A11895068FAF7A9FF42495C
:10E9A000C9688889F8F751FD00F0030008B101201B
:10E9B00000E000203C49098908443A49088000BF2A
:10E9C0003A48006809880844E968496888420AD0DA
:10E9D00000BFAFF2D03340F2FC524FA1AFF28C3007
:10E9E000F5F7E2F800BF00BF656700BF2F48006879
:10E9F0002C4909880844606200BF208D2949098894
:10EA000088420ADA00BFAFF2044340F2076251A124
:10EA1000AFF2C030F5F7C8F800BF00BF208D214924
:10EA20000988401A2085204601F0E8FD1E4840680C
:10EA30000089002806DD1C4840684E490860002017
:10EA4000194948601849C9688889F8F7FEFC00F040
:10EA5000010028B14848007840F02000464908707D
:10EA6000DAE0656F606FC068406810490860E96867
:10EA70008889F8F7EAFC00F0030008B1012000E003
:10EA8000002029890844616A0844606200BFE9687F
:10EA90008889F8F7DAFC00F0030008B101206EE085
:10EAA0006CE000006201002060C7002058010020D7
:10EAB000696E7365672E7020213D204E554C4C00C9
:10EAC000696E73616E65206F666673657421000000
:10EAD0007062756620746F6F2073686F72742100A6
:10EAE0007463705F726563656976653A2073656704
:10EAF0006D656E74206E6F74207472696D6D6564DF
:10EB000020636F72726563746C7920746F20726316
:10EB1000765F776E640A00007463705F7265636588
:10EB20006976653A207365676D656E74206E6F74E3
:10EB3000207472696D6D656420636F7272656374B1
:10EB40006C7920746F206F6F7365712071756575B6
:10EB5000650A00007463705F726563656976653A83
:10EB6000207463706C656E203E207263765F776EF2
:10EB7000640A000068010020650100200020298946
:10EB80000844218D88420AD900BFAFF2885340F271
:10EB90002B62C2A1AFF24450F5F706F800BF00BFE8
:10EBA000E9688889F8F751FC00F0030008B10120FA
:10EBB00000E0002029890844218D081A208520467C
:10EBC00001F01CFD6868008900280DDDBD48006863
:10EBD00028B1BC4869680068FAF770FA02E0B949E0
:10EBE0006868086000206860E9688889F8F72DFC8B
:10EBF00000F0010050B1B448007840F02000B24964
:10EC00000870207D042801D10720207528686067DE
:10EC1000284600F0EDFD00BF606F30B1606FC06846
:10EC20004068616A88423FF41CAF00BFA07E00F0DC
:10EC3000010060B100BF608B4FF6FE710840608339
:10EC400000BF00BF608B40F00200608305E000BFA2
:10EC5000608B40F00100608300BF1DE1606F20B950
:10EC60009A4800F06BFD6067FAE00026656FF2E0FD
:10EC7000E868406896490968884217D19348008936
:10EC80002989884211DD914800F058FD8246BAF189
:10EC9000000F09D016B1C6F800A001E0C4F874A0B6
:10ECA00029465046FDF7D4FED8E0D7E0A6B9E8687B
:10ECB000406887490968081A0DD5844800F03EFD70
:10ECC0008246BAF1000F05D0C4F874A02946504618
:10ECD000FDF7BEFEC2E030E0F0684068401C7C49B1
:10ECE0000968081A28D4E8684068401E784909680D
:10ECF000081A002820DC754800F020FD8246BAF191
:10ED0000000F18D0F06840683189084470490968DC
:10ED1000401A002809DDF06880886D490988081AC2
:10ED2000308131897068FAF7E3FDC6F800A0294602
:10ED30005046FDF78DFE91E000BF2E462868002862
:10ED40007DD1E868406862490968081A002876DDC4
:10ED5000E9688889F8F779FB00F0010000B17DE0EF
:10ED60005A4800F0EBFC28602868002871D0E86859
:10ED700040682989084456490968401A002809DD75
:10ED8000E868808852490988081A288129896868B2
:10ED9000FAF7AEFD218D606A08444E4909884C4A55
:10EDA00012681144081A002853DD2968C968888947
:10EDB000F8F74BFB00F0010098B12968C968888911
:10EDC000F8F743FB00F03E0A5046F8F73EFB29688F
:10EDD000C96889894CF2FF02114008432968C96853
:10EDE0008881A08C218D084439490988401A2968F6
:10EDF00008812A6811895068FAF77AFD2968C9687C
:10EE00008889F8F722FB00F0030008B1012000E038
:10EE100000202968098908442E49088000BF218DF7
:10EE2000606A01442A4800682A4A128810448142D4
:10EE30000ED000BFAFF634034FF4DF6201E009E00B
:10EE400007E0AFF26431AFF2F470F4F7ADFE00BF4B
:10EE500000BF03E02D68002D7FF40AAF00BF00BFA4
:10EE6000204600F0DFFC17E0204600F0DBFC13E05A
:10EE70001749606A0968081A08D4218D606A084435
:10EE8000401E13490968081A002805DD00BF608B81
:10EE900040F00200608300BFBDE8F09F7463705FC4
:10EEA000726563656976653A206F6F73657120746A
:10EEB00063706C656E203E207263765F776E640AC5
:10EEC00000000000680100206501002060C70020EC
:10EED00058010020620100202DE9F04107460D464F
:10EEE00014461E4600BF002D0CD100BF0EA34FF4E8
:10EEF000D36219A11FA0F4F757FE00BF6FF00F00F7
:10EF0000BDE8F08100BF3CB12189284600F046F8F9
:10EF10002046FAF791FB04E01EB92846FBF738FFBC
:10EF2000EEE70020ECE700002E2E2F4D6964646CA4
:10EF30006577617265732F54686972645F5061729E
:10EF400074792F4C7749502F7372632F636F7265FA
:10EF50002F7463702E6300007463705F7265637654
:10EF60005F6E756C6C3A20696E76616C69642070B6
:10EF700063620000417373657274696F6E202225AD
:10EF80007322206661696C6564206174206C696E0F
:10EF90006520256420696E2025730A002DE9F04163
:10EFA00004460F4600BF002C0AD100BF1CA340F24C
:10EFB000CF3227A12CA0F4F7F7FD00BFBDE8F08108
:10EFC00000BF00BF207D012808D100BF14A340F27C
:10EFD000D2322FA124A0F4F7E7FD00BF00BF208D9F
:10EFE000384485B2B5F5066F02DC208DA84203DDFA
:10EFF0004FF40660208500E02585204601F0FEFAEA
:10F000000646B6F5067F08D300BF608B40F00200CD
:10F01000608300BF2046FDF7B1FD00BFCEE70000D2
:10F020002E2E2F4D6964646C6577617265732F5461
:10F03000686972645F50617274792F4C7749502F00
:10F040007372632F636F72652F7463702E63000099
:10F050007463705F7265637665643A20696E766189
:10F060006C69642070636200417373657274696FC8
:10F070006E2022257322206661696C6564206174AC
:10F08000206C696E6520256420696E2025730A0056
:10F09000646F6E27742063616C6C207463705F72A0
:10F0A000656376656420666F72206C697374656E43
:10F0B0002D7063627300000070B506460D4600BFF8
:10F0C000002D07D100BF09A3FF2214A11DA0F4F752
:10F0D0006BFD00BF00BF344605E0E06FA84201D1E0
:10F0E0000020E067E468002CF7D170BD2E2E2F4D74
:10F0F0006964646C6577617265732F5468697264C2
:10F100005F50617274792F4C7749502F7372632F5F
:10F11000636F72652F7463702E6300007463705F99
:10F1200072656D6F76655F6C697374656E65723A52
:10F1300020696E76616C6964206C697374656E65B4
:10F1400072000000417373657274696F6E2022252E
:10F150007322206661696C6564206174206C696E3D
:10F160006520256420696E2025730A002DE9F04191
:10F17000044600BF002C08D100BF20A340F2C162AA
:10F180002BA131A0F4F710FD00BF00BF206F18B90C
:10F190006FF00500BDE8F081256F2846FEF7D6F92F
:10F1A00010B16FF00500F5E72868206704F16C06E0
:10F1B00000E03668306858B13168C9684868F8F7C7
:10F1C00037F90746E9684868F8F732F9381AF0D491
:10F1D000306828603560286810B90020A4F86800FD
:10F1E00094F84200FF2804DA94F84200401C84F8A6
:10F1F00042000020606300BFCCE700002E2E2F4DA0
:10F200006964646C6577617265732F5468697264B0
:10F210005F50617274792F4C7749502F7372632F4E
:10F22000636F72652F7463705F6F75742E63000077
:10F230007463705F7265786D69743A20696E766187
:10F240006C69642070636200417373657274696FE6
:10F250006E2022257322206661696C6564206174CA
:10F26000206C696E6520256420696E2025730A0074
:10F2700010B5044600BF002C08D100BF20A340F207
:10F28000F9622CA133A0F4F78FFC00BF00BF206F00
:10F29000A0B3A07E00F0040080BB2046FFF766FF0D
:10F2A00060BBB4F84810B4F86020914202DAB4F8B8
:10F2B000481001E0B4F86010084601EBD071C1F3CA
:10F2C0004F01A4F84A10B4F84A00618E4900884200
:10F2D00004D2608E4004000CA4F84A00B4F84A003E
:10F2E000618E032202FB0100A4F8480000BF608B7E
:10F2F00040F00400608300BF0020208610BD0000A5
:10F300002E2E2F4D6964646C6577617265732F547E
:10F31000686972645F50617274792F4C7749502F1D
:10F320007372632F636F72652F7463705F6F757490
:10F330002E6300007463705F7265786D69745F6638
:10F340006173743A20696E76616C696420706362DF
:10F3500000000000417373657274696F6E2022258E
:10F360007322206661696C6564206174206C696E2B
:10F370006520256420696E2025730A0010B50446B7
:10F3800000BF002C08D100BF08A340F2AD6214A159
:10F390001AA0F4F709FC00BF00BF204600F09EF859
:10F3A00010B9204600F03EF810BD00002E2E2F4D63
:10F3B0006964646C6577617265732F5468697264FF
:10F3C0005F50617274792F4C7749502F7372632F9D
:10F3D000636F72652F7463705F6F75742E630000C6
:10F3E0007463705F7265786D69745F72746F3A20D0
:10F3F000696E76616C696420706362004173736545
:10F400007274696F6E2022257322206661696C65B3
:10F4100064206174206C696E6520256420696E200B
:10F4200025730A0010B5044600BF002C08D100BFA8
:10F430000AA34FF4D36216A11EA0F4F7B5FB00BFD8
:10F4400000BF94F84200FF2804DA94F84200401C00
:10F4500084F842002046FDF791FB10BD2E2E2F4D63
:10F460006964646C6577617265732F54686972644E
:10F470005F50617274792F4C7749502F7372632FEC
:10F48000636F72652F7463705F6F75742E63000015
:10F490007463705F7265786D69745F72746F5F63B7
:10F4A0006F6D6D69743A20696E76616C6964207065
:10F4B00063620000417373657274696F6E20222568
:10F4C0007322206661696C6564206174206C696ECA
:10F4D0006520256420696E2025730A0070B50446F6
:10F4E00000BF002C08D100BF22A340F263622EA10E
:10F4F00036A0F4F759FB00BF00BF206F10B96FF0C2
:10F50000050070BD256F07E02846FEF71FF810B113
:10F510006FF00500F5E72D6828680028F4D128462B
:10F52000FEF714F810B16FF00500EAE7E06E28600E
:10F53000206FE0660020206700BF608B40F4006011
:10F54000608300BFE9684868F7F772FF0646E9681C
:10F550008889F7F77AFF00F0030008B1012000E086
:10F560000020298908443044E0640020606300BF23
:10F57000C7E700002E2E2F4D6964646C65776172B9
:10F5800065732F54686972645F50617274792F4C8F
:10F590007749502F7372632F636F72652F74637096
:10F5A0005F6F75742E6300007463705F7265786DB1
:10F5B00069745F72746F5F707265706172653A2012
:10F5C000696E76616C696420706362004173736573
:10F5D0007274696F6E2022257322206661696C65E2
:10F5E00064206174206C696E6520256420696E203A
:10F5F00025730A0070B504460E4615462CB1207AD4
:10F6000018B1207AF8F704FF70BD2846F7F734F9EF
:10F61000FAE700002DE9F04F85B083460F4690468B
:10F620001D46DDF8389000BF002D08D100BF1EA395
:10F6300040F2C47229A130A0F4F7B6FA00BF00BFAF
:10F6400000BFB9F1000F08D100BF17A340F2C57287
:10F6500033A129A0F4F7A8FA00BF00BF002646F2A4
:10F66000080A3846F7F7E4FE14220490DDE90F019A
:10F670008DE80704002231464046049BFDF79EFCBE
:10F68000044614B905B0BDE8F08F33460022214688
:10F690005846FDF7A3FD4B462A4621465846FDF73E
:10F6A0001FFD00BFEEE700002E2E2F4D6964646C35
:10F6B0006577617265732F54686972645F50617217
:10F6C00074792F4C7749502F7372632F636F726573
:10F6D0002F7463705F6F75742E6300007463705FC6
:10F6E0007273743A20696E76616C6964206C6F6322
:10F6F000616C5F6970000000417373657274696FBB
:10F700006E2022257322206661696C656420617415
:10F71000206C696E6520256420696E2025730A00BF
:10F720007463705F7273743A20696E76616C696499
:10F730002072656D6F74655F6970000070B5054675
:10F7400000BF002D08D100BF0CA340F2826217A1B8
:10F750001DA0F4F729FA00BF00BF0320F8F7F8FB5B
:10F7600004460CB9002070BD95E80F0084E80F0036
:10F770006068FAF771F92046F5E700002E2E2F4D4C
:10F780006964646C6577617265732F54686972642B
:10F790005F50617274792F4C7749502F7372632FC9
:10F7A000636F72652F7463702E6300007463705F03
:10F7B0007365675F636F70793A20696E76616C6913
:10F7C0006420736567000000417373657274696F2C
:10F7D0006E2022257322206661696C656420617445
:10F7E000206C696E6520256420696E2025730A00EF
:10F7F00010B5044644B1606810B16068F9F71CFFA9
:10F8000021460320F8F7D6FA10BD70B5044605E08E
:10F8100025682046FFF7ECFF2C4600BF002CF7D1EF
:10F8200070BD00002DE9F04704460025A94600BF41
:10F83000002C08D100BF2CA340F2EA7237A13FA0F0
:10F84000F4F7B2F900BF00BF05F0010008B10420D1
:10F8500000E0002005F0020109B1002100E00021D4
:10F86000084405F0080109B1002100E00021084426
:10F8700005F0100109B1002100E0002100EB0108B2
:10F88000206DF7F7D5FD82465346002241462046BB
:10F89000FDF726FB06464EB900BF608B40F0030023
:10F8A000608300BF6FF00100BDE8F0874B462A4639
:10F8B00031462046FDF792FC231D22463146204664
:10F8C000FDF70EFC07462FB100BF608B40F0030030
:10F8D000608306E000BF608B4FF6FC7108406083D8
:10F8E00000BF3846E0E700002E2E2F4D6964646C9F
:10F8F0006577617265732F54686972645F506172D5
:10F9000074792F4C7749502F7372632F636F726530
:10F910002F7463705F6F75742E6300007463705F83
:10F9200073656E645F656D7074795F61636B3A20B7
:10F93000696E76616C6964207063620041737365FF
:10F940007274696F6E2022257322206661696C656E
:10F9500064206174206C696E6520256420696E20C6
:10F9600025730A0070B5044600BF002C08D100BF03
:10F9700016A340F2EB3222A128A0F4F715F900BF3C
:10F9800000BFE06EE8B1E56E00E02D682868002851
:10F99000FBD1E9688889F7F758FD00F0070078B9CE
:10F9A0000120F7F752FDE96889890843E9688881F1
:10F9B00000BF608B40F02000608300BF002070BD5E
:10F9C00000BF01212046FBF709FDF8E72E2E2F4D41
:10F9D0006964646C6577617265732F5468697264D9
:10F9E0005F50617274792F4C7749502F7372632F77
:10F9F000636F72652F7463705F6F75742E630000A0
:10FA00007463705F73656E645F66696E3A20696ED9
:10FA100076616C69642070636200000041737365F5
:10FA20007274696F6E2022257322206661696C658D
:10FA300064206174206C696E6520256420696E20E5
:10FA400025730A002DE9F04F85B04FF00009E94811
:10FA50000068401CE7490860E7480078401CE64918
:10FA6000087000BF0025E5480468E3E200BF207D80
:10FA7000002808D100BFE2A340F2BE42ECA1F7A0EB
:10FA8000F4F792F800BF00BF00BF207D012808D125
:10FA900000BFDBA340F2BF42FAA1F0A0F4F784F864
:10FAA00000BF00BF00BF207D0A2808D100BFD4A33B
:10FAB0004FF49862FEA1E9A0F4F776F800BF00BF0A
:10FAC000A07FCD490978884202D12546E468B1E299
:10FAD000C9480078A0770026B046207D022806D1CC
:10FAE00094F84200062802DB701CC6B2D1E094F8FC
:10FAF00042000C2802DB701CC6B2CAE094F89900E0
:10FB000000285DDD00BF206F002808D000BFBCA327
:10FB100040F2D442F2A1D1A0F4F746F800BF00BFF2
:10FB200000BFE06E002808D100BFB5A340F2D54267
:10FB3000F8A1CAA0F4F738F800BF00BF94F89A0003
:10FB40000C2802DB701CC6B2A3E094F89900401E9A
:10FB5000FE490F5C94F89800B84204DA94F89800D3
:10FB6000401C84F8980094F89800B84227DB4FF0C6
:10FB7000010AB4F8600030B9204600F0CBFD70B146
:10FB80004FF0000A0BE0B4F86010204600F0F4FAE1
:10FB900028B92046FCF7F2FF08B94FF0000ABAF185
:10FBA000000F0BD0002084F8980094F899000728E3
:10FBB00004D294F89900401C84F8990000BF68E0D2
:10FBC000B4F93000002809DBB4F9300047F6FF71C2
:10FBD000884203DA208E401C00B22086B4F930003F
:10FBE000B4F94010884254DB2046FFF777FC18B187
:10FBF000206F70BBE06E60B3207D02281ED094F8A9
:10FC000042200C2A02D294F8422000E00C22114635
:10FC1000B4F93E20B4F93C3002EBE302CC4B5B5C20
:10FC200002FA03F047F6FF72904201DA024601E061
:10FC300047F6FF7212B2A4F8402000BF00202086D1
:10FC4000B4F84800B4F86010884203DAB4F8480009
:10FC500002E01EE0B4F86000049004984010A4F89C
:10FC60004A00B4F84A00618E4FF6FF7202EA410181
:10FC7000884205DA608E114601EA4000A4F84A0085
:10FC8000608EA4F848000020A4F86A002046FFF720
:10FC9000C9FB207D06280BD1A07E00F0100038B1F2
:10FCA0005449206A0968081A282801D9701CC6B26C
:10FCB000607A00F00800D0B3207D042802D0207DB7
:10FCC000072834D1A349D4F8940008444FF4FA71BA
:10FCD000B0FBF1F0474A216A1268511A884206D2F5
:10FCE000701CC6B208F1010000F0FF081FE094F894
:10FCF0009B1042F29F4211FB02F1D4F8940000EBFA
:10FD0000C1004FF4FA71B0FBF1F03A4A216A12686F
:10FD1000511A88420BD22046FCF728FB8146B9F1E4
:10FD2000000F04D194F89B00401C84F89B00606F86
:10FD300068B13049206A0968081AB4F9401001EB2B
:10FD40004101B0EB410F02D32046FBF73BFE207D83
:10FD5000032807D12749206A0968081A282801D9E9
:10FD6000701CC6B2207D092807D12249206A096883
:10FD7000081AF02801D9701CC6B2002E37D0D4F86A
:10FD800090A02046FDF7D4FC8DB100BF1B48006851
:10FD9000844208D100BF1AA340F26D526EA12FA079
:10FDA000F3F702FF00BF00BFE068E86011E000BFAA
:10FDB00012480068A04208D000BF11A340F271525F
:10FDC00070A126A0F3F7F0FE00BF00BF0B49E0686A
:10FDD0000860B8F1000F0BD0208BE18A221DCDE91D
:10FDE0000021029023462046626A216DE0E0FBE09C
:10FDF000E0E000002C01002042010020380100203A
:10FE00002E2E2F4D6964646C6577617265732F5473
:10FE1000686972645F50617274792F4C7749502F12
:10FE20007372632F636F72652F7463702E630000AB
:10FE30007463705F736C6F77746D723A2061637472
:10FE4000697665207063622D3E737461746520214C
:10FE50003D20434C4F5345440A00000041737365F5
:10FE60007274696F6E2022257322206661696C6549
:10FE700064206174206C696E6520256420696E20A1
:10FE800025730A007463705F736C6F77746D723AD8
:10FE900020616374697665207063622D3E737461BE
:10FEA000746520213D204C495354454E0A00000002
:10FEB0007463705F736C6F77746D723A20616374F2
:10FEC000697665207063622D3E73746174652021CC
:10FED0003D2054494D452D574149540A000000002A
:10FEE0007463705F736C6F7774696D723A207065BC
:10FEF0007273697374207469636B696E67207769C4
:10FF0000746820696E2D666C69676874206461741A
:10FF1000610000007463705F736C6F7774696D7259
:10FF20003A2070657273697374207469636B696ECB
:10FF300067207769746820656D7074792073656EC9
:10FF4000642062756666657200000000E12A01089F
:10FF5000D42A0108B84C0A007463705F736C6F7721
:10FF6000746D723A206D6964646C652074637020EE
:10FF7000213D207463705F6163746976655F7063AF
:10FF8000627300007463705F736C6F77746D723AA4
:10FF900020666972737420706362203D3D20746333
:10FFA000705F6163746976655F70636273000000FF
:10FFB000FFF730FBD4F810B0207D03902746E468AB
:10FFC0003846FBF7B9FB00204849087000BFBAF17A
:10FFD000000F03D06FF00C015846D04700BF4348D4
:10FFE000007800B13EE524E02546E468287F401C07
:10FFF0002877287F697F88421BDB002028773B49D0
:020000040801F1
:10000000087000BFD5F88C0030B12946D5F88C2097
:1000100028699047814601E04FF0000900BF33484E
:10002000007800B11EE5B9F1000F02D12846FCF7B7
:10003000A5FD00BF002C7FF419AD00252C480468F5
:100040004EE000BF207D0A280AD000BFAFF2502347
:1000500040F2A15227A1AFF2FC10F3F7A5FD00BFBB
:1000600000BF00262F49206A0968081AF02801D924
:10007000701CC6B2002E31D02046FDF759FB9DB151
:1000800000BF1B48006884420AD100BFAFF2902332
:1000900040F2AF5224A1AFF23C20F3F785FD00BF40
:1000A00000BFE068E86013E000BF11480068A042AC
:1000B0000AD000BFAFF2B82340F2B35224A1AFF28E
:1000C0006420F3F771FD00BF00BF0949E0680860D4
:1000D0002746E4683846FBF72FFB01E02546E46835
:1000E000002CAED105B0BDE8F08F0000400100202B
:1000F0003C0100207463705F736C6F77746D723AAB
:100100002054494D452D57414954207063622D3E7E
:100110007374617465203D3D2054494D452D574110
:10012000495400002C0100207463705F736C6F777A
:10013000746D723A206D6964646C6520746370201C
:10014000213D207463705F74775F70636273000099
:100150007463705F736C6F77746D723A2066697246
:10016000737420706362203D3D207463705F747708
:100170005F706362730000002DE9F04F85B00546A3
:100180000E4600270024A34600BF002D08D100BF63
:1001900079A340F24B3285A18DA0F3F705FD00BF96
:1001A00000BFEC6E24B94FF0FF3005B0BDE8F08F12
:1001B000002E0CD100BF00BF6FA340F253328EA1BE
:1001C00083A0F3F7F1FC00BF00BFB01FEDE720896B
:1001D000B04201DC0020E8E700BF688EB04208DAD8
:1001E00000BF65A340F25B328CA179A0F3F7DCFC81
:1001F00000BF00BF00BF2089002808DC00BF5EA34D
:100200004FF4577289A172A0F3F7CEFC00BF00BF74
:1002100094F80A8008F0010008B1042000E00020F2
:1002200008F0020109B1002100E00021084408F0B3
:10023000080109B1002100E00021084408F0100184
:1002400009B1002100E00021084404902089801BAE
:100250001FFA80FA0498504481B24FF4207236207D
:10026000F8F754FD8346BBF1000F00D16EE06068E3
:1002700000892189401A304480B20290DBF80430B2
:10028000049A991860685246029BF9F735F950456F
:1002900000D05BE0E1688889F7F7D7F800F03F0904
:1002A0000020039009F0080028B129F008090398FC
:1002B00040F00800039009F0010028B129F001097D
:1002C000039840F001000390E1684868F7F7B0F840
:1002D00030440346CDE9008059462846039AFAF790
:1002E00029FF074607B931E06068F8F78FFF35F856
:1002F000661F081A288062681289A2EB0A0291B26E
:100300006068F9F7F5FA2089A0EB0A0020814846D9
:10031000F7F79BF8E16889890843E168888160689C
:10032000F8F774FF2988084428807868F8F76EFF8A
:100330002988084425F866092068386027603868ED
:1003400010B90020A5F8680000202EE700BF47B1D3
:1003500000BF09A34FF4767238A11DA0F3F724FC67
:1003600000BF00BFBBF1000F02D05846F9F764F997
:100370004FF0FF3019E700002E2E2F4D6964646C9A
:100380006577617265732F54686972645F5061723A
:1003900074792F4C7749502F7372632F636F726596
:1003A0002F7463705F6F75742E6300007463705FE9
:1003B00073706C69745F756E73656E745F73656777
:1003C0003A20696E76616C69642070636200000097
:1003D000417373657274696F6E20222573222066E3
:1003E00061696C6564206174206C696E65202564A8
:1003F00020696E2025730A0043616E277420737094
:100400006C6974207365676D656E7420696E746FB6
:10041000206C656E677468203000000073706C6932
:1004200074203C3D206D7373000000007573656798
:100430002D3E6C656E203E20300000007365672005
:100440003D3D204E554C4C0010B50948006868B938
:100450000848006810B90848006838B1012004490C
:10046000086000220549FA20FAF7BEF910BD000025
:1004700078010020380100203C010020AD0A01086D
:100480003EB504462948007800F0040000B13EBDA6
:1004900000BF002C08D100BF25A340F2EE2231A1FD
:1004A00038A0F3F781FB00BF00BF2048007800F0C0
:1004B000020018B33D49606A0968081A26D4218DE4
:1004C000606A084439490968081A00281EDC38485F
:1004D00000680088364909684988364ACDE9002114
:1004E000029032480068344909884218314B1B1D7C
:1004F000324801682046FFF78DF8C8E70B480078BE
:1005000000F0010010B12E48006820622A480088DF
:10051000002808DD00BF608B40F00200608300BF50
:100520002046FCF72BFB00BFB1E700006401002070
:100530002E2E2F4D6964646C6577617265732F543C
:10054000686972645F50617274792F4C7749502FDB
:100550007372632F636F72652F7463705F696E2EA1
:10056000630000007463705F74696D65776169741E
:100570005F696E7075743A20696E76616C6964208B
:1005800070636200417373657274696F6E20222517
:100590007322206661696C6564206174206C696EE9
:1005A0006520256420696E2025730A00580100200B
:1005B0004801002078900020620100205C010020AA
:1005C0002C01002010B5FBF769F806480078401CA4
:1005D000C0B20449087000F0010008B1FFF732FA18
:1005E00010BD0000410100200348007840F01000D9
:1005F00001490870704700006501002070B504468D
:1006000000BF002C08D100BF1CA340F2A63227A1D6
:100610002FA0F3F7C9FA00BF00BF218D606A45180B
:10062000608EE16AB0F5866F02DD4FF4866000E00F
:10063000608E0844281A04D4208D6085E06A281A48
:1006400070BDE16A606A401A002802DD0020608502
:1006500012E0616AE06A461A00BFB6F5803F08D32F
:1006600000BF06A340F2B63223A119A0F3F79CFA0B
:1006700000BF00BF668500BF0020E1E72E2E2F4D92
:100680006964646C6577617265732F54686972641C
:100690005F50617274792F4C7749502F7372632FBA
:1006A000636F72652F7463702E6300007463705FF4
:1006B0007570646174655F7263765F616E6E5F779B
:1006C0006E643A20696E76616C69642070636200C2
:1006D000417373657274696F6E20222573222066E0
:1006E00061696C6564206174206C696E65202564A5
:1006F00020696E2025730A006E65775F7263765FEE
:10070000616E6E5F776E64203C3D20307866666671
:10071000660000002DE9FC5F04464FF0000A00BFB0
:10072000002C08D100BF37A340F64F0242A14BA0D6
:10073000F3F73AFA00BF00BFE56E15B90020BDE837
:10074000FC9F94F89A00FF2804DA94F89A00401C61
:1007500084F89A00E9688889F6F777FE00F00100CE
:1007600018B1288908B9012000E000208146B9F1BC
:10077000000F01D1012000E000208346E8684368B3
:100780005A4651462046FCF7ABFB064616B94FF0D9
:10079000FF30D4E77768B9F1000F09D01120F6F7E0
:1007A00054FEB9894CF2FF0211400843B8810DE0B4
:1007B000706814300090696809892A89891A8BB297
:1007C000012268680099F8F797FE00BFE968486859
:1007D000F6F72EFE00F10108206DB0EB080001D500
:1007E000C4F850805346002231462046FCF7F6FC00
:1007F000231D224631462046FCF772FC01900198E9
:100800009DE700002E2E2F4D6964646C6577617240
:1008100065732F54686972645F50617274792F4CEC
:100820007749502F7372632F636F72652F746370F3
:100830005F6F75742E6300007463705F7A65726F0A
:100840005F77696E646F775F70726F62653A206977
:100850006E76616C69642070636200004173736539
:100860007274696F6E2022257322206661696C653F
:1008700064206174206C696E6520256420696E2097
:1008800025730A0038B504460D46F6F7E5FD17480E
:1008900004601748056006211648F9F739FF00285B
:1008A0000AD000BF00BF14A340F261221EA127A0FE
:1008B000F3F77AF900BF00BF2E48F9F75FFF002871
:1008C0000AD000BF00BF0CA340F265222AA11FA0DE
:1008D000F3F76AF900BF00BF00204FF480630246BF
:1008E0002E4900902EA0F9F763FF38BDC800002004
:1008F000CC000020D00000202E2E2F4D6964646CA7
:100900006577617265732F54686972645F506172B4
:1009100074792F4C7749502F7372632F6170692F50
:1009200074637069702E63006661696C656420741D
:100930006F206372656174652074637069705F74A1
:100940006872656164206D626F7800004173736541
:100950007274696F6E2022257322206661696C654E
:1009600064206174206C696E6520256420696E20A6
:1009700025730A00D40000206661696C65642074E8
:100980006F20637265617465206C6F636B5F746365
:100990007069705F636F726500000000E50A01080E
:1009A00074637069705F7468726561640000000050
:1009B0002DE9F04105460E46174600BF1448F9F7E9
:1009C000CEFE38B900BF13A3FC221EA121A0F3F76D
:1009D000EBF800BF00BF0920F7F7BAFA04461CB9CC
:1009E0004FF0FF30BDE8F081002020706560A66008
:1009F000E76021460648F9F7A3FE30B121460920F9
:100A0000F7F7D8F94FF0FF30ECE70020EAE70000F5
:100A1000D00000202E2E2F4D6964646C65776172C2
:100A200065732F54686972645F50617274792F4CDA
:100A30007749502F7372632F6170692F74637069E7
:100A4000702E6300496E76616C6964206D626F7808
:100A500000000000417373657274696F6E20222577
:100A60007322206661696C6564206174206C696E14
:100A70006520256420696E2025730A0070B505463F
:100A80000C4694F82D0000F0180028B1054A2146C4
:100A90002846FFF78DFF70BD034A21462846FFF721
:100AA00087FFF8E725550008D961000810B504460E
:100AB000FFF788FD0748006810B90748006828B1AB
:100AC00000220649FA20F9F78FFE02E000200449CF
:100AD000086010BD380100203C010020AD0A01086B
:100AE0007801002008B51148F9F740FE1048006869
:100AF00020B1104800680E490968884715E069462A
:100B00000D4800F0C1F8009800280AD100BF00BFCE
:100B10000AA3912215A11DA0F3F746F800BF00BF5C
:100B200003E0009800F046F800BFE8E7D40000209A
:100B3000C8000020CC000020D00000202E2E2F4D19
:100B40006964646C6577617265732F546869726457
:100B50005F50617274792F4C7749502F7372632FF5
:100B60006170692F74637069702E630074637069BB
:100B7000705F7468726561643A20696E76616C6951
:100B800064206D6573736167650000004173736570
:100B90007274696F6E2022257322206661696C650C
:100BA00064206174206C696E6520256420696E2064
:100BB00025730A0010B50446207820B101280ED014
:100BC000022818D113E0201D07C8904710B16068B3
:100BD000F8F732FD21460920F7F7ECF816E0D4E9E2
:100BE0000110884721460820F7F7E4F80EE0D4E921
:100BF000011088470AE000BF00BF05A3CF2210A163
:100C000017A0F2F7D1FF00BF00BF00BF00BF10BDAB
:100C10002E2E2F4D6964646C6577617265732F5455
:100C2000686972645F50617274792F4C7749502FF4
:100C30007372632F6170692F74637069702E630023
:100C400074637069705F7468726561643A20696E7C
:100C500076616C6964206D6573736167650000007F
:100C6000417373657274696F6E202225732220664A
:100C700061696C6564206174206C696E652025640F
:100C800020696E2025730A002DE9F04106460F46C3
:100C900000BFF9F7C5FE0446601C60B91148F9F7BA
:100CA0007DFD002239463046F9F7B7FC0D48F9F7CB
:100CB0005DFDBDE8F08114B9F9F7F4FCE9E70948F6
:100CC000F9F76CFD224639463046F9F7A6FC054691
:100CD0000448F9F74BFD681C10B9F9F7E3FCD8E7B5
:100CE00000BFE6E7D400002070B505460E4600BF01
:100CF0001348F9F734FD40B900BF12A340F25D126A
:100D00001CA120A0F2F750FF00BF00BF0820F7F79A
:100D10001FF9044614B94FF0FF3070BD0120207058
:100D20006560A66021460648F9F70AFD30B1214604
:100D30000820F7F73FF84FF0FF30EEE70020ECE730
:100D4000D00000202E2E2F4D6964646C657761728F
:100D500065732F54686972645F50617274792F4CA7
:100D60007749502F7372632F6170692F74637069B4
:100D7000702E6300496E76616C6964206D626F78D5
:100D800000000000417373657274696F6E20222544
:100D90007322206661696C6564206174206C696EE1
:100DA0006520256420696E2025730A0010B5EFF7D1
:100DB0009BFAC0F30D0000F540400149088010BDCA
:100DC0007C0100202DE9FE4F05460E4600200190D3
:100DD00000BF002D07D100BF61A3CF226CA172A07C
:100DE000F2F7E2FE00BF00BF00BF002E07D100BF38
:100DF0005BA3D02276A16CA0F2F7D6FE00BF00BFA5
:100E00006889082803DA2846F8F716FCA6E0D5F822
:100E100004A0764A11685069F5F751F88146BAF88E
:100E20000000F6F712FB8346BAF80200F6F70DFB56
:100E3000029000240027A0466D48046838E0618ACB
:100E40000298814232D14A463146204600F0E0F80D
:100E500060B3207C00F00400A8B9B8F1000F01D104
:100E6000A04610E0B9F1000F0DD060484069401C69
:100E700048B9D8F800007168884204D020687168C9
:100E8000884200D1A046A08A58450FD1606820B1A1
:100E9000564960680969884208D137B1E068F8604E
:100EA00053480068E0605248046003E02746E46865
:100EB000002CC4D100BF04B9444614B101200190F4
:100EC00008E04A4970684969884201D1012000E080
:100ED00000200190019800283CD008212846F8F70E
:100EE0000FFE70B100BF00BF1DA34FF4B87241A147
:100EF0002DA0F2F759FE00BF00BF2846F8F79CFB73
:100F00002CE07CB1A06948B1CDF800B0374B10336C
:100F10002A462146D4E906C0E0471EE02846F8F7F5
:100F20008BFB1BE0B9F1000F10D13048007D00F0C1
:100F3000F000E0280AD02D488089083001B2284608
:100F4000F8F78BFC03212846F4F7D8FD2846F8F77C
:100F500073FB02E02846F8F76FFB00BFBDE8FE8F89
:100F60002E2E2F4D6964646C6577617265732F5402
:100F7000686972645F50617274792F4C7749502FA1
:100F80007372632F636F72652F7564702E63000038
:100F90007564705F696E7075743A20696E76616C05
:100FA0006964207062756600417373657274696F5D
:100FB0006E2022257322206661696C65642061744D
:100FC000206C696E6520256420696E2025730A00F7
:100FD0007564705F696E7075743A20696E76616CC5
:100FE0006964206E657469660000000068900020E6
:100FF00080010020706275665F72656D6F76655F57
:10100000686561646572206661696C65640A0000E8
:1010100070B504460D46164600BF002C07D100BF30
:101020001FA387222AA133A0F2F7BEFD00BF00BF95
:1010300000BF002D07D100BF19A3882237A12DA022
:10104000F2F7B2FD00BF00BF207A50B1217A3D48CF
:10105000406890F83000401CC0B2814201D00020AE
:1010600070BD8EB174B1206860B136484069401CD3
:1010700040B12068A968084032494969AA6811400E
:1010800088420BD10120EBE734B1206820B12D4913
:1010900020684969884201D10120E1E70020DFE7AB
:1010A0002E2E2F4D6964646C6577617265732F54C1
:1010B000686972645F50617274792F4C7749502F60
:1010C0007372632F636F72652F7564702E630000F7
:1010D0007564705F696E7075745F6C6F63616C5F6F
:1010E0006D617463683A20696E76616C6964207022
:1010F00063620000417373657274696F6E2022250C
:101100007322206661696C6564206174206C696E6D
:101110006520256420696E2025730A007564705F60
:10112000696E7075745F6C6F63616C5F6D61746321
:10113000683A20696E76616C6964206E65746966D0
:10114000000000006890002010B5024682B11368CC
:1011500073B169B10B685BB1064B186806E00368B0
:101160001468A34201D10B680360C0680028F6D15F
:1011700010BD00008001002001460A69D1E901305C
:101180009860D1E9010358605068884201D18868AD
:101190005060002008611068401E106010687047A1
:1011A000034B0360034B0B60802313607047000008
:1011B000A0010020FC01002000F1080141604FF077
:1011C000FF31816000F10801C1600161002101600F
:1011D000704700210161704710B502460B685C1C26
:1011E0000CB9106907E002F1080000E040684468AB
:1011F00024689C42FAD944684C604C68A1608860BD
:1012000041600A611468641C146010BD42684A6041
:1012100093688B60936859609160086103685B1CF8
:101220000360704700BF502080F31188BFF34F8FD9
:10123000BFF36F8F00BF0E480068401C0C49086068
:1012400008460068012812D10A480068C0B208B9EF
:10125000012000E0002050B900BF502080F3118829
:10126000BFF34F8FBFF36F8F00BF00BFFEE7704724
:10127000BC00002004ED00E00D48006850B900BF3C
:10128000502080F31188BFF34F8FBFF36F8F00BFE3
:1012900000BFFEE706480068401E05490860084692
:1012A000006820B9002080F3118800BF00BF70479C
:1012B000BC00002070B506463546002E44D0083DDF
:1012C0002C46224960680968084008B1012000E006
:1012D000002050B900BF502080F31188BFF34F8F1A
:1012E000BFF36F8F00BF00BFFEE7206808B9012081
:1012F00000E0002050B900BF502080F31188BFF3F8
:101300004F8FBFF36F8F00BF00BFFEE70F496068CC
:1013100009680840C0B12068B0B90C496068096824
:101320008843606000F008FA094960680968084469
:10133000074908602046F8F79BFF06480068401CF4
:101340000449086001F068FA70BD0000B800002090
:10135000A8000020B400002000204FF0E021086128
:101360008861064800684FF47A71B0FBF1F0401EC6
:101370004FF0E021486107200861704720000020FD
:1013800070B5EEF769FF0446102C16D304F1E02087
:1013900090F8F05315480078854201DB012000E009
:1013A000002050B900BF502080F31188BFF34F8F49
:1013B000BFF36F8F00BF00BFFEE70D48006800F469
:1013C000E0600C490968884201D8012000E0002053
:1013D00050B900BF502080F31188BFF34F8FBFF387
:1013E0006F8F00BF00BFFEE770BD0000C00000208F
:1013F0000CED00E0C400002070B504460025D4B117
:101400001248006808B9012000E0002050B900BF70
:10141000502080F31188BFF34F8FBFF36F8F00BF51
:1014200000BFFEE700F088F900212046F8F7CEFC67
:1014300001F0F2F905463DB94FF0805004490860CB
:10144000BFF34F8FBFF36F8F70BD00009800002077
:1014500004ED00E070B50546FFF7E4FE15B930482D
:10146000006800E028460446201DFFF785FE78B995
:10147000E06A00EB80002B4951F8200040B994F855
:101480002C100120884028490968814326480160C2
:10149000A06A18B104F11800FFF76EFE2348006837
:1014A000401C224908601E480068844209D1211D61
:1014B0001F48FFF7ABFE1F480068401C1D4908602D
:1014C00009E01D480068401E1B4908602046F8F7E7
:1014D0009BFDF8F71DFFFFF7CFFE18480068E8B145
:1014E0000F480068844219D11548006808B90120E6
:1014F00000E0002050B900BF502080F31188BFF3F6
:101500004F8FBFF36F8F00BF00BFFEE74FF08050DB
:101510000C490860BFF34F8FBFF36F8F70BD0000A1
:101520006000002084510020780000208C00002002
:10153000405400206C000020700000207C0000203F
:101540009800002004ED00E00349096801600349A8
:101550000968416070470000880000207400002086
:1015600001200149086070478400002070B50446DE
:101570000D4654B900BF502080F31188BFF34F8F40
:10158000BFF36F8F00BF00BFFEE705480168183149
:101590002046FFF721FE01212846F8F717FC70BD11
:1015A000600000202DE9F04706460F4634464FF014
:1015B0000109002E60D0206D50B900BF502080F38B
:1015C0001188BFF34F8FBFF36F8F00BF00BFFEE7DF
:1015D000E06CB84201D23D4600E0E56CE06AA8420A
:1015E0004AD0206D012847D124480068844201D0A8
:1015F000012000E0002050B900BF502080F3118886
:10160000BFF34F8FBFF36F8F00BF00BFFEE7D4F86B
:101610002C80E562A06900F0004010B9C5F12000FF
:10162000A06108EB8801164A02EB810160698842DB
:1016300001D1012000E00020F0B1201DFFF79CFD4A
:1016400040B994F82C10012088400E490968814364
:101650000C48016094F82C10012088400949096861
:10166000084308490860E16A01EB8101044A02EB82
:101670008100211DFFF7CAFDBDE8F0876000002052
:10168000845100207800002010B586B0002005901D
:10169000049003AA04A905A8FFF782FD0022DDE952
:1016A00004101346CDE9002102901CA11D48039AA5
:1016B00000F084FE1C4908600846006808B1012457
:1016C00000E00024012C15D100BF502080F31188C8
:1016D000BFF34F8FBFF36F8F00BF4FF0FF30134941
:1016E000086001201249086000201249086000F0DB
:1016F00071F810E0601C08B1012000E0002050B932
:1017000000BF502080F31188BFF34F8FBFF36F8F5E
:1017100000BF00BFFEE706B010BD000049444C45C5
:1017200000000000E9A000089400002090000020C4
:101730007C0000207400002002480068401C014921
:1017400008607047980000201D48006818B101200B
:101750001C49086032E000201A4908601A480068F5
:10176000B0FA80F0C0F11F0101EB8100174A52F876
:10177000200008B1012000E0002050B900BF502037
:1017800080F31188BFF34F8FBFF36F8F00BF00BF8F
:10179000FEE701EB81020D4B03EB820042685268C9
:1017A000426000F108024368934202D142685268E5
:1017B00042604268D268064B1A6000BF7047000062
:1017C0009800002084000020780000208451002030
:1017D000600000201CB5524800685249884201D080
:1017E000012000E0002050B900BF502080F3118894
:1017F000BFF34F8FBFF36F8F00BF00BFFEE74848B6
:1018000000684849491E884201D0012000E00020BC
:1018100050B900BF502080F31188BFF34F8FBFF342
:101820006F8F00BF00BFFEE73F4908460078019078
:10183000FF200A4610700846007800909DF80000CE
:1018400000F0F0009DF80020904201D1012000E05E
:10185000002050B900BF502080F31188BFF34F8F94
:10186000BFF36F8F00BF00BFFEE79DF8000000F0E0
:1018700050002E4A107007202D4A106009E02C48B5
:101880000068401E2A4A10609DF800004006000EC5
:1018900000909DF8000000F080008028EFD02448E0
:1018A0000068C0F10700042801D1012000E00020F9
:1018B00050B900BF502080F31188BFF34F8FBFF3A2
:1018C0006F8F00BF00BFFEE7194800680002184A8A
:1018D00010601046008800F4E0601060124A019821
:1018E00010700F482030006840F470000C4920311F
:1018F00008600846006840F070400860FFF72CFD63
:1019000000200C490860EEF76FFC0B48006840F0BF
:10191000404009490860EEF753FC00201CBD000060
:1019200000ED00E071C20F4100E400E0C0000020C3
:10193000C4000020BC00002034EF00E02DE9F0419D
:1019400004460126002722460021012000F01CF851
:1019500005462846F8F7DCFB2846BDE8F0812DE96E
:10196000F84304460D4601274FF000082B4600229D
:1019700011460120009400F034F806463046F8F78E
:10198000C7FB3046BDE8F8832DE9F84305460E460F
:1019900017460DB1012000E0002050B900BF5020D3
:1019A00080F31188BFF34F8FBFF36F8F00BF00BF6D
:1019B000FEE705FB06F808F14800F8F72BFD0446A2
:1019C00064B1A14609F14809002084F846003B466D
:1019D0004A46314628460094F8F7A9FB2046BDE860
:1019E000F8832DE9F84380460E4617461D46DDF87C
:1019F0002090B8F1000F01D0012000E0002050B984
:101A000000BF502080F31188BFF34F8FBFF36F8F5B
:101A100000BF00BFFEE70DB1012000E0002050B97B
:101A200000BF502080F31188BFF34F8FBFF36F8F3B
:101A300000BF00BFFEE707B10EB1012000E00020AB
:101A400050B900BF502080F31188BFF34F8FBFF310
:101A50006F8F00BF00BFFEE707B90EB9012000E09D
:101A6000002050B900BF502080F31188BFF34F8F82
:101A7000BFF36F8F00BF00BFFEE7482000900098C3
:101A8000482801D1012000E0002050B900BF5020BB
:101A900080F31188BFF34F8FBFF36F8F00BF00BF7C
:101AA000FEE700BF2C464CB1012084F846004B46AF
:101AB0003A46314640460094F8F739FB2046BDE8E7
:101AC000F883000070B505460E462C4654B900BF99
:101AD000502080F31188BFF34F8FBFF36F8F00BF8B
:101AE00000BFFEE7FFF79EFBD4E90F12206801FB61
:101AF0000200A0600020A06320686060E06B401ED0
:101B0000226C216800FB0211E160FF2084F8440090
:101B100084F845009EB9206908B9012000E0002042
:101B2000A8B904F1100000F02BFE80B14FF08050F6
:101B300009490860BFF34F8FBFF36F8F07E004F1CF
:101B40001000FFF739FB04F12400FFF735FBFFF726
:101B500093FB012070BD000004ED00E02DE9FF4380
:101B600083B0064688461D464FF00009344654B9F6
:101B700000BF502080F31188BFF34F8FBFF36F8FEA
:101B800000BF00BFFEE7B8F1000F01D1206C08B91B
:101B9000012000E0002050B900BF502080F31188E0
:101BA000BFF34F8FBFF36F8F00BF00BFFEE7022D63
:101BB00002D1E06B012801D1012000E0002050B9E2
:101BC00000BF502080F31188BFF34F8FBFF36F8F9A
:101BD00000BF00BFFEE700F04FFC08B9059808B948
:101BE000012000E0002050B900BF502080F3118890
:101BF000BFF34F8FBFF36F8F00BF00BFFEE700BF83
